:1000000000000120910100000D0200008BE60000BD
:1000100011020000130200001502000000000000A1
:1000200000000000000000000000000061A30000CC
:10003000190200000000000081A300001505010066
:1000400035D300003DD3000045D300004DD3000060
:1000500055D300005DD3000065D300006DD30000D0
:1000600075D300007DD3000085D300008DD3000040
:1000700095D300009DD30000A5D30000ADD30000B0
:10008000B5D30000BDD30000C5D30000CDD3000020
:10009000D5D30000DDD30000E5D30000EDD3000090
:1000A000F5D30000FDD3000005D400000DD40000FE
:1000B00015D400001DD40000D96200004969000079
:1000C00025D400002DD4000035D400003DD400001C
:1000D00045D400004DD4000055D400005DD400008C
:1000E00065D400006DD4000075D400007DD40000FC
:1000F00085D400008DD4000095D400009DD400006C
:10010000A5D40000ADD40000B5D40000BDD40000DB
:10011000C5D40000CDD40000D5D40000DDD400004B
:10012000E5D40000EDD40000F5D40000FDD40000BB
:1001300005D500000DD5000015D500001DD5000027
:1001400025D500002DD5000035D500003DD5000097
:1001500045D500004DD5000055D500005DD5000007
:1001600065D500006DD50000AC47010000000020FF
:100170008C000000AC4701000000FF1F00000000E1
:100180008C000020681300000000FF1F00600000CA
:1001900072B604F087FB0E4B07E003F10C049A687B
:1001A0005968186800F01AF823460A4A9342F4D3B3
:1001B00006E01C46596854F8080B00F01EF8234668
:1001C000054A9342F5D362B600F010FDFEE700BF8A
:1001D00068010000800100009001000000239342AC
:1001E0000AD210B450F8044B41F8044B0433934244
:1001F000F8D35DF8044B70477047002303E00022FA
:1002000040F8042B04338B42F9D37047FEE7FEE736
:10021000FEE7FEE7FEE7FEE7FEE7FEE7FEE7FEE7B6
:10022000FFFFFFFFFFFFFFFFFFFFFFFFFFFFFFFFDE
:10023000FFFFFFFFFFFFFFFFFFFFFFFFFFFFFFFFCE
:10024000FFFFFFFFFFFFFFFFFFFFFFFFFFFFFFFFBE
:10025000FFFFFFFFFFFFFFFFFFFFFFFFFFFFFFFFAE
:10026000FFFFFFFFFFFFFFFFFFFFFFFFFFFFFFFF9E
:10027000FFFFFFFFFFFFFFFFFFFFFFFFFFFFFFFF8E
:10028000FFFFFFFFFFFFFFFFFFFFFFFFFFFFFFFF7E
:10029000FFFFFFFFFFFFFFFFFFFFFFFFFFFFFFFF6E
:1002A000FFFFFFFFFFFFFFFFFFFFFFFFFFFFFFFF5E
:1002B000FFFFFFFFFFFFFFFFFFFFFFFFFFFFFFFF4E
:1002C000FFFFFFFFFFFFFFFFFFFFFFFFFFFFFFFF3E
:1002D000FFFFFFFFFFFFFFFFFFFFFFFFFFFFFFFF2E
:1002E000FFFFFFFFFFFFFFFFFFFFFFFFFFFFFFFF1E
:1002F000FFFFFFFFFFFFFFFFFFFFFFFFFFFFFFFF0E
:10030000FFFFFFFFFFFFFFFFFFFFFFFFFFFFFFFFFD
:10031000FFFFFFFFFFFFFFFFFFFFFFFFFFFFFFFFED
:10032000FFFFFFFFFFFFFFFFFFFFFFFFFFFFFFFFDD
:10033000FFFFFFFFFFFFFFFFFFFFFFFFFFFFFFFFCD
:10034000FFFFFFFFFFFFFFFFFFFFFFFFFFFFFFFFBD
:10035000FFFFFFFFFFFFFFFFFFFFFFFFFFFFFFFFAD
:10036000FFFFFFFFFFFFFFFFFFFFFFFFFFFFFFFF9D
:10037000FFFFFFFFFFFFFFFFFFFFFFFFFFFFFFFF8D
:10038000FFFFFFFFFFFFFFFFFFFFFFFFFFFFFFFF7D
:10039000FFFFFFFFFFFFFFFFFFFFFFFFFFFFFFFF6D
:1003A000FFFFFFFFFFFFFFFFFFFFFFFFFFFFFFFF5D
:1003B000FFFFFFFFFFFFFFFFFFFFFFFFFFFFFFFF4D
:1003C000FFFFFFFFFFFFFFFFFFFFFFFFFFFFFFFF3D
:1003D000FFFFFFFFFFFFFFFFFFFFFFFFFFFFFFFF2D
:1003E000FFFFFFFFFFFFFFFFFFFFFFFFFFFFFFFF1D
:1003F000FFFFFFFFFFFFFFFFFFFFFFFFFFFFFFFF0D
:10040000FFFFFFFFFFFFFFFFFFFFFFFFFEFFFFFFFD
:1004100001F0FF01102A2BDB10F0070F08D010F8B5
:10042000013B013A8B422DD010F0070F42B3F6D1B9
:10043000F0B441EA012141EA014122F007047FF0D2
:1004400000070023F0E80256083C85EA010586EA29
:10045000010685FA47F5A3FA87F586FA47F6A5FA65
:1004600087F68EB9EED1F0BC01F0FF0102F0070271
:1004700032B110F8013B013A83EA010313B1F8D11C
:100480000020704701387047002D06BF35460338FD
:10049000073815F0010F07D1013015F4807F02BF36
:1004A000013015F4C03F0130F0BC0138704700BF87
:1004B00080B586B002AFF860B9607A603B607B6857
:1004C0000093BB68FA68396802480CF091FC00BEE2
:1004D000FDE700BF681F010080B485B000AF034690
:1004E0003960FB710023FB6014E00F4AFB6812F8CF
:1004F0001330FA799A420AD10B4AFB685B00134425
:1005000093F901301A463B681A60002306E0FB6845
:100510000133FB60FB68262BE7D91B2318461437F1
:10052000BD465DF8047B7047A81F010080B586B00A
:1005300000AF3B1D184604F0A7FB01233B710023CD
:100540007B71144BBB60144BFB6002233B613B1D72
:10055000184604F0B7FB0346104A136000F0C8F8D1
:1005600000F086FB0E4B1B68184600F09DFB0C4B01
:100570005B68184600F098FB094B9B68184600F032
:1005800093FB074BDB68184600F08EFB00BF183763
:10059000BD4680BD80F00F4000B004408C000020BC
:1005A0009000002080B596B002AF7860354B4222B3
:1005B0003549022004F032FD02F02CF8B86407F14E
:1005C0001C0314221946B86C10F0CDFB0346012B16
:1005D00053D13B7F042B47D801A252F823F000BF30
:1005E000FB050000F50500000D060000690600008F
:1005F0005B06000000F090FB40E0BB6ADBB27A6A69
:10060000D2B21146184600F06DFC37E03B6A01217A
:1006100018460BF0D7FE0346FB643B6A59B207F15C
:100620001C030833FA6C18460DF09DF90346002BA5
:100630000CD1164B56221449022004F0EFFCF86C42
:1006400000F0E2FBF86C0CF095F817E0104B5A2222
:100650000D49042004F0E2FC10E00E4B5E220A4932
:10066000042004F0DBFC09E03B7F00930A4B61228D
:100670000549042004F0D2FC00E000BF142009F07A
:1006800099FF9CE7F81F01001420010024200100BD
:1006900034200100502001006C20010080B584B09E
:1006A00002AF0D4B0193002300930C4BE1220C4948
:1006B0000C4811F01DF878607B68012B06D00A4BBE
:1006C0009C220A49022004F0A9FCFEE70AF004F883
:1006D00000BF0837BD4680BDA000002000000020FC
:1006E000B0200100A5050000B82001001420010081
:1006F000B0B5ADF54C7D00AF07F53873184605F081
:100700001FFFD74BC7F8F032D64BC7F8F4320B2394
:10071000C7F8F832D24BC7F80033D24BC7F80433CE
:100720000A23C7F80833CE4BC7F81033CD4BC7F8B0
:1007300014330923C7F81833C94BC7F82033C94B02
:10074000C7F824330823C7F82833012387F8E13298
:1007500007F53373184604F057F9C34BC7F8D03286
:10076000C24BC7F8D4321323C7F8D832012387F815
:10077000CC32012387F8DC32002387F8C9320A2300
:1007800087F8C83207F52D7407F533750FCD0FC400
:100790002B68236007F5197307F538715022184646
:1007A00011F08FF907F51973184602F045F8034662
:1007B000AF4A136007F50573184605F0C1FE07F54B
:1007C0004C73A3F58E73AB4A1A6107F54C73A3F50E
:1007D0008E73A94A5A6107F54C73A3F58E730122F3
:1007E0009A6107F54C73A3F58E73A24A1A6207F556
:1007F0004C73A3F58E73A04A5A6207F54C73A3F5A8
:100800008E7302229A6207F54C73A3F58E73994A90
:100810001A6307F54C73A3F58E73974A5A6307F56D
:100820004C73A3F58E7305229A6307F54C73A3F5F9
:100830008E73904A1A6407F54C73A3F58E738E4A33
:100840005A6407F54C73A3F58E730C229A6407F56E
:100850004C73A3F58E7301225A7007F50073184686
:1008600004F0D2F807F54C73A3F598737E4A5A60EA
:1008700007F54C73A3F598737C4A9A6007F54C739F
:10088000A3F598731222DA6007F54C73A3F59873F9
:1008900001221A7007F54C73A3F5987301221A749C
:1008A00007F54C73A3F5CC73012283F8652007F597
:1008B0004C73A3F5CC73142283F8642007F54C73B2
:1008C000A3F5CC7307F54C72A2F5987203F15004AE
:1008D00015460FCD0FC42B68236007F54C73A3F5A5
:1008E000CC7207F54C73A3F58E731046194650234E
:1008F0001A4611F0E6F807F5CC73184601F09CFF94
:1009000003465B4A536007F5A473184605F018FECA
:1009100007F54C73A3F5F473584A1A6107F54C7345
:10092000A3F5F473564A5A6107F54C73A3F5F473B3
:1009300004229A6107F54C73A3F5F4734F4A1A62C7
:1009400007F54C73A3F5F4734D4A5A6207F54C73DF
:10095000A3F5F47305229A6207F54C73A3F5F473BB
:10096000464A1A6307F54C73A3F5F473444A5A6375
:1009700007F54C73A3F5F47306229A6307F54C73DD
:10098000A3F5F4733D4A1A6407F54C73A3F5F473A9
:100990003B4A5A6407F54C73A3F5F47307229A6433
:1009A00007F54C73A3F5F47301225A7007F59A7397
:1009B000184604F029F807F54C73A3F5FE732D4A89
:1009C0005A6007F54C73A3F5FE732B4A9A6007F53E
:1009D0004C73A3F5FE730D22DA6007F54C73A3F593
:1009E000FE7301221A7007F54C73A3F5FE73012202
:1009F0001A7407F54C73A3F51973022283F8652066
:100A000007F54C73A3F51973142283F8642007F5D6
:100A10004C73A3F5197307F54C72A2F5FE7203F13E
:100A2000500415460FCD0FC42B68236007F54C7397
:100A3000A3F5197207F54C73A3F5F4731046194624
:100A400050231A4611F03DF807F1CC03184601F087
:100A5000F3FE0346064A936007F17C03184611E053
:100A600080F00F4000B0044040F00F4000A0044070
:100A70009000002000F00F4000900440C0F00F40B4
:100A800000C0044005F05CFD07F54C73A3F52D7321
:100A9000514A1A6107F54C73A3F52D734F4A5A61F9
:100AA00007F54C73A3F52D7300229A6107F54C737B
:100AB000A3F52D73484A1A6207F54C73A3F52D73FD
:100AC000464A5A6207F54C73A3F52D7301229A62C8
:100AD00007F54C73A3F52D733F4A1A6307F54C7362
:100AE000A3F52D733D4A5A6307F54C73A3F52D7397
:100AF00002229A6307F54C73A3F52D73364A1A64E4
:100B000007F54C73A3F52D73344A5A6407F54C73FB
:100B1000A3F52D7303229A6407F54C73A3F52D7387
:100B200001225A7007F16803184603F06DFF07F5BC
:100B30004C73A3F532732A4A5A6007F54C73A3F538
:100B40003273284A9A6007F54C73A3F53273032277
:100B5000DA6007F54C73A3F5327301221A7007F5BA
:100B60004C73A3F5327301221A7407F54C73A3F585
:100B70004C73032283F8652007F54C73A3F54C737F
:100B8000142283F8642007F54C73A3F54C7307F522
:100B90004C72A2F5327203F1500415460FCD0FC40A
:100BA0002B68236007F54C73A3F54C7207F54C7363
:100BB000A3F52D731046194650231A4610F081FFF5
:100BC0003B46184601F038FE0346074AD36000BF93
:100BD00007F54C77BD46B0BDC0F00F4000C00440E3
:100BE00040F00F4000A004409000002080B500AF0E
:100BF0000DF05DFC0DF011FC0DF01CFC0DF0F2FB96
:100C0000154B3F221549022004F008FA00F0B0FB12
:100C1000134B42221149022004F000FAFFF786FC30
:100C2000104B46220D49022004F0F8F9FFF736FD7B
:100C30000D4B4A220949022004F0F0F90CF037FD6F
:100C40000A4B4E220549022004F0E8F90CF05EFD43
:100C50000023184680BD00BFDC200100F820010001
:100C6000002101001821010028210100402101007C
:100C700080B500AF0A4B00221A700CF07BFC0346D3
:100C8000084A1360074B1B6800221A60054B1B685B
:100C900000225A60034B1B6800229A6000BF80BD8F
:100CA000E8130020A400002080B584B002AF786073
:100CB000134B28221349022004F0B0F9124B1B6891
:100CC000124A12781146124A11447A6818460CF0FA
:100CD000BBFC0E4B1B7801330922019200930D4B94
:100CE0002A220849022004F099F9084B1B780133A5
:100CF000DAB2064B1A7000BF0837BD4680BD00BF90
:100D00006021010094210100A4000020E8130020CC
:100D100004000020A821010080B588B002AF00F0D7
:100D200033F90346BB73314B30223149022004F0C2
:100D300075F90023FB7510E02E4B1B681A68FB7DCC
:100D40002D490B44194610460CF01CFC786078685D
:100D50000CF07BFEFB7D0133FB75FA7DBB7B9A4279
:100D6000EAD30023BB7500233B6126E00123BB755A
:100D7000322009F01FFC0023FB7314E01D4B1B689D
:100D80001A68FB7B1C490B44194610460CF0FAFB11
:100D9000B860BB681B7D022B02D00023BB7506E048
:100DA000FB7B0133FB73FA7BBB7B9A42E6D3BB7DB3
:100DB000002B07D13B6901333B613B69B3F52F7FC2
:100DC000D4DB00E000BFBB7D002B01D00B4B00E06B
:100DD0000B4B00930B4B4E220549022004F01EF9E9
:100DE000BB7D18461837BD4680BD00BFC02101003D
:100DF00094210100A400002004000020082201002A
:100E0000102201001822010080B588B002AF78607E
:100E100000F0BAF803463B750023FB7525E02D4B27
:100E20001B681A68FB7D2C490B44194610460CF0D0
:100E3000A9FBF860FB7D7A6813441B78FB72FB7A90
:100E40001946F86801F068FFFB7D0133FA7A0192D8
:100E50000093224B5A222249022004F0DFF864203A
:100E600009F0A8FBFB7D0133FB75FA7D3B7D9A42BF
:100E7000D5D30023BB7521E0642009F09BFB01233F
:100E8000BB7500237B7515E0124B1B681A687B7DD0
:100E900011490B44194610460CF074FB386138694F
:100EA0000CF0FCFD0346032B01D10023BB757B7DB9
:100EB00001337B757A7D3B7D9A42E5D3BB7D83F020
:100EC0000103DBB2002BD7D1BB7D18461837BD46D6
:100ED00080BD00BFA40000200400002064220100A7
:100EE0009421010080B586B002AF03460A46FB712B
:100EF0001346BB71FB79082B09D9FB7900931C4B76
:100F000074221C49042004F089F800232BE000F02F
:100F10003BF803461A46FB79934209D3FB790093C9
:100F2000154B79221349042004F078F800231AE0C5
:100F3000124B1B681A68FB7911490B44194610467D
:100F40000CF020FBF860BB791946F86801F006FF49
:100F5000FB79BA79019200930A4B87220549022056
:100F600004F05CF8012318461037BD4680BD00BF71
:100F70009C22010094210100FC220100A400002019
:100F8000040000206023010080B400AF034B1B78F5
:100F90001846BD465DF8047B704700BFE81300208B
:100FA00080B582B000AF7860074B0122074908483E
:100FB00008F08CF80346DAB27B681A7000231846F2
:100FC0000837BD4680BD00BFAC230100BC23010033
:100FD000C423010080B582B000AF0346FB71FA79EB
:100FE000044B054905480FF050F90023184608370F
:100FF000BD4680BDAC230100BC230100C423010019
:1010000080B582B000AF7860074B002207490848DE
:1010100008F05CF803461A467B681A6000231846FD
:101020000837BD4680BD00BFAC230100CC230100C2
:10103000D423010080B582B000AF78607A68054B98
:10104000054906480FF021F9002318460837BD4628
:1010500080BD00BFAC230100CC230100D4230100DC
:1010600080B584B000AFF860B9601346FB71074AE1
:10107000B968F8680DF087FFFB791A46B968F86817
:101080000EF087F800BF1037BD4680BDD8230100A1
:1010900080B586B000AF03463960FB71FA7907F17D
:1010A000080310211846FFF7DBFF07F10800074B84
:1010B0004FF0FF32064908F009F803461AB23B68C0
:1010C0001A80002318461837BD4680BDAC230100A6
:1010D000E023010080B586B000AF03460A46FB71ED
:1010E0001346BB80FA7907F1080310211846FFF771
:1010F000B7FFBA8807F10800044B05490FF0C5F89F
:10110000002318461837BD4680BD00BFAC23010040
:10111000E023010080B596B000AF78607B685B6823
:101120001A46434943480DF083FD07F1130318465F
:10113000FFF736FF034687F8573097F85730002BF4
:1011400015D107F114033C4A402118460DF01BFF4E
:10115000FA7C07F11403402118460EF06DF807F1F0
:101160001403364A402118460DF032FF06E007F11D
:101170001403334A402118460DF005FF7B685A6876
:1011800007F1140319462F480DF052FD07F10C0327
:101190001846FFF735FF034687F8573097F8573062
:1011A000002B30D107F11403234A402118460DF0DB
:1011B000EAFEFA6807F11403402118460EF0D8F849
:1011C00007F11403204A402118460DF001FFFB6887
:1011D00003F00103002B07D007F114031B4A402141
:1011E00018460DF0F5FE06E007F11403184A4021F9
:1011F00018460DF0EDFE07F11403104A4021184681
:101200000DF0E6FE06E007F114030D4A40211846F2
:101210000DF0B9FE7B685A6807F1140319460D48B2
:101220000DF006FD002318465837BD4680BD00BFAF
:10123000E423010010240100B026010084410100D4
:10124000182401002024010030240100382401006A
:101250003C2401004024010080B582B000AF7860DA
:101260007B685B681A460B490B480DF0CFFC7B6826
:101270005B681A4609490A480DF0C8FC7B685B6840
:101280001A46084908480DF0C1FC002318460837E3
:10129000BD4680BD482401001024010064240100E3
:1012A0008824010098240100A424010080B586B0A0
:1012B00000AFF860B9607A602849F86810F013FD53
:1012C0000346002B06D02649F86810F00CFD0346B3
:1012D000002B07D1BB6801221A707868FFF7BCFFAA
:1012E000034637E01F49F86810F0FDFC0346002B69
:1012F00006D01D49F86810F0F6FC0346002B07D114
:10130000BB6801221A707868FFF704FF034621E0EA
:101310000A221649F86810F000FD0346002B18D188
:10132000BB6801221A70FB680B337B6107F1100266
:1013300007F11403114618460EF068F80346002B17
:1013400005D13B691846FFF775FE034602E01B23F3
:1013500000E0002318461837BD4680BDA8390100BB
:10136000B4240100B8390100C0240100CC240100DC
:1013700080B500AF1D480CF0AFF91D480CF0ACF97A
:101380001C480CF0A9F91C480CF0A6F90CF09DF9CA
:101390000EF056FB06F04CFF4FF400614FF4FF20B7
:1013A00006F012FD0DF096F90DF0BBF906F088F885
:1013B0000DF05DF90DF080F90DF0A8FD0DF0E9F9E3
:1013C00000F0DCFE0DF046FC05F09CF803F0DEFEBC
:1013D00004F062FC03460021184603F0F9FC01F01A
:1013E000B1F90DF09EF900BF80BD00BF09003810B3
:1013F0000A0038100B0038100C00381080B582B08D
:1014000000AF0346FB71044B5B68FA7910469847BE
:1014100000BF0837BD4680BD0C3D010080B582B0DD
:1014200000AF0346FB710C4B1B684FF0FF311846B1
:101430000FF05BFA0346012B09D1084B5B68FA7980
:1014400010469847044B1B6818460FF020FA00BF5F
:101450000837BD4680BD00BFA80000200C3D01003C
:1014600080B582B000AF78600B4B1B684FF0FF3146
:1014700018460FF03AFA0346012B08D1074B1B68B8
:1014800078689847044B1B6818460FF000FA00BFB5
:101490000837BD4680BD00BFA80000200C3D0100FC
:1014A00080B582B000AF0023FB710C4B1B684FF07E
:1014B000FF3118460FF019FA0346012B09D1084BEA
:1014C000DB6898470346FB71044B1B6818460FF016
:1014D000DEF9FB7918460837BD4680BDA80000201C
:1014E0000C3D010080B582B000AF786006E008498D
:1014F0007B685A1C7A601B78184688477B681B7883
:10150000002BF4D100BF00BF0837BD4680BD00BF2F
:10151000FD13000080B588B000AFF8607A603B60D2
:101520000B46FB72FB7A402B02D1FB6800221A703B
:10153000FB681B78052B00F2F68001A252F823F01D
:10154000591500007D15000087150000E515000005
:101550003F1600008B1600007B6800221A70FB7A91
:10156000402B09D1FB7A1A46396878680DF063FD83
:10157000FB6801221A70D7E00023D6E0FB68022244
:101580001A700023D1E0FB7A1A46396878680DF0AA
:1015900052FDFB7A202B1DD17B680133BB6107F123
:1015A000170207F11803114618460EF048F80346D3
:1015B000002B0BD10CF0CCF803461A46FB7D9A4267
:1015C00004D1FB6803221A700023AEE0FB680022FE
:1015D0001A7005E0FB7A0A2B02D1FB6800221A7010
:1015E0000023A2E0FB7A1A46396878680DF023FDE3
:1015F000FB7A202B1BD17B680433BB6107F11702F8
:1016000007F11803114618460EF019F80346002B8F
:1016100009D1FB7D97F828209A4204D1FB68042267
:101620001A70002381E0FB6800221A7005E0FB7A43
:101630000A2B02D1FB6800221A70002375E0FB7AA6
:101640001A46396878680DF0F6FCFB7A202B14D125
:101650007B680733BB6107F11803364918460DF064
:10166000EEFF0346002B04D1FB6805221A7000230D
:101670005BE0FB6800221A7005E0FB7A0A2B02D1BE
:10168000FB6800221A7000234FE0FB7A1A46396883
:1016900078680DF0D0FCFB7A0A2B42D17B680A33C4
:1016A000BB61BB692449184610F01DFB0346002BA3
:1016B00014D17B680C3300221A7078680CF0BBF8E8
:1016C0000346FB77FB6800221A701A4B1B78FA7FDF
:1016D0009A4201D1012328E0022326E017497868C5
:1016E00010F001FB0346002B14D17B680D33002260
:1016F0001A7078680CF09FF80346FB77FB680022AD
:101700001A700C4B1B78FA7F9A4201D102230CE02D
:1017100002230AE0FB7A0A2B03D1FB6800221A702D
:1017200002E0002301E000BF02E718462037BD4673
:1017300080BD00BFEA130020082501000C25010030
:1017400080B58EB002AFF8607A603B600B46FB72EA
:1017500000237B6107F1180300221A605A609A6027
:10176000DA601A610023BB74284B00221A703B68B0
:101770001B6807F1130210469847FB7C002B14D01E
:10178000FB7C1A464FF4007120480DF054FCFB7CA2
:101790000A2B0AD11D4B1B78402B03D079681B48BC
:1017A0000CF03DF9194B00221A70FB7C002BDED1A6
:1017B00005F04CF80346FB74FB7C002B17D0F97C3A
:1017C00007F1140207F11200FB7A00931823FFF7C8
:1017D000A1FE034687F82F3097F82F30012B03D056
:1017E00097F82F30022BBFD197F82F3009E0322025
:1017F00008F0E0FEFB68323BFB60FB68002BB3DCCB
:10180000032318463037BD4680BD00BFAC00002022
:1018100080B594B002AFB9607A603B600346FB7359
:10182000002387F847307B6D002B01D1644B7B652B
:1018300007F11403634A302118460DF0A4FBFA7B2C
:1018400007F11403302118460DF0F6FC07F11403DC
:101850002022302118460DF0EEFB0BF079FF0346F5
:101860001A4607F11403302118460DF0E5FC07F184
:1018700014032022302118460DF0DDFB07F114037C
:101880000022302118460DF0D7FC07F114034E4A10
:10189000302118460DF09CFB07F11403BA68302183
:1018A00018460DF095FB07F1140318460BF0C3FF23
:1018B000034687F8463097F846301B0987F84530CD
:1018C00097F84530092B01D8302200E0372297F8ED
:1018D00045301344DBB2FB7697F8463003F00F0334
:1018E00087F8453097F84530092B01D8302200E0C1
:1018F000372297F845301344DBB23B77334B1B68F4
:101900004FF0FF3118460EF0F0FF0346012B51D186
:1019100004F090FF2E4B1B78002B09D007F1140325
:1019200000932C4B40F259122B49002003F076FB18
:1019300007F114031846FFF7D5FD2848FFF7D2FD3D
:10194000FB7B002B03D1002387F847302DE0642078
:1019500008F030FEF97B7B6D3A6D7868FFF7F0FE9A
:10196000034687F8443097F84430012B03D1002315
:1019700087F8473019E097F84430032B03D10C2344
:1019800087F8473006E097F84430022B02D1142341
:1019900087F847303B68002B03D11B2387F847307B
:1019A00003E03B68013B3B60B2E7084B1B6818460D
:1019B0000EF06DFF97F8473018464837BD4680BD9A
:1019C000F82401001425010018250100A8000020BA
:1019D000E91300202025010028250100D03B01004B
:1019E00080B586B000AF78607B685B681A461B499B
:1019F0001B480DF01DF907F108031A4A102118467B
:101A00000DF0C1FA0BF0A4FE03461A4607F10803D5
:101A1000102118460DF010FC07F10803124A10219E
:101A200018460DF0D5FA7B685A6807F10803194685
:101A30000E480DF0FDF80E4B1B78002B01D00D4920
:101A400000E00D497B685B681A460C480DF0F0F821
:101A5000002318461837BD4680BD00BF3025010061
:101A600044250100B0260100844101004825010001
:101A7000E91300208C450100502501005825010084
:101A800080B582B000AF78607B685B681A46164903
:101A900016480DF0BBF87B685B681A461449154878
:101AA0000DF0B4F87B685B681A46134913480DF0D3
:101AB000ADF87B685B681A46114912480DF0A6F82C
:101AC0007B685B681A46104910480DF09FF87B68E8
:101AD0005B681A460E490F480DF098F80023184627
:101AE0000837BD4680BD00BF6025010044250100C8
:101AF00064240100882401007C2501009425010054
:101B0000A4250100C4250100D425010014260100EC
:101B10002C2601005026010080B594B002AFF86079
:101B2000B9607A606D49F86810F0DDF80346002B63
:101B300006D06B49F86810F0D6F80346002B07D1A1
:101B4000BB6801221A707868FFF79AFF0346C1E06C
:101B50006449F86810F0C7F80346002B06D06249C4
:101B6000F86810F0C0F80346002B07D1BB680122CB
:101B70001A707868FFF734FF0346ABE007225B4931
:101B8000F86810F0CAF80346002B21D1BB68012287
:101B90001A70FB6807337B647B6C5549184610F05C
:101BA000A2F80346002B04D1524B01221A700023E5
:101BB00090E07B6C5049184610F095F80346002BD6
:101BC00004D14C4B00221A70002383E01B2381E0D8
:101BD00008224A49F86810F0A0F80346002B1FD1EC
:101BE000BB6801221A70FB6808337B6407F140026E
:101BF00007F14403114618460DF008FC0346002B7C
:101C00000CD13B6C002B09DB3B6CFF2B06DC3B6CE7
:101C1000DBB21846FFF7DEF903465BE01B2359E011
:101C200008223749F86810F078F80346002B0BD1EA
:101C3000BB6801221A70FB6808331846FFF752FC94
:101C40003048FFF74FFC44E00B222F49F86810F0B2
:101C500064F80346002B3CD1BB6801221A70FB6874
:101C60000B337B6407F1400207F144031146184629
:101C70000DF0CCFB0346002B29D102E07B6C013335
:101C80007B647B6C1B78202BF8D07B6C1B78222B21
:101C90000FD107F1100107F14403302218460DF06F
:101CA00012FD0346002B01D01B2313E007F11003A4
:101CB0007B643B6CD8B2796C144B01937B680093C6
:101CC000002342F21072FFF7A3FD034602E01B233C
:101CD00000E0002318464837BD4680BDA839010002
:101CE00060260100B8390100682601007426010051
:101CF0007C260100E91300208026010084260100D3
:101D000090260100D03B01009C260100F824010030
:101D100080B592B000AFF860B9607A603B607B68D4
:101D200000221A703B6800221A70BB68FA681A60B9
:101D3000FB681B78402B40F09380FB6801333B64C9
:101D400007F13F0207F14003114618460DF077FCFA
:101D50000346002B40F084800BF0FAFC03461A4641
:101D600097F83F309A4203D097F83F30002B77D155
:101D700007F13E0207F14003114618460DF05FFCE3
:101D80000346002B6CD197F83E207B681A7097F8B9
:101D90003F203B681A7007F13D0207F140031146EE
:101DA00018460DF04CFC034687F8473097F847304B
:101DB000002B01D0142354E0F8680BF03CFD0346DF
:101DC00087F8463097F83D3097F846209A4242D03F
:101DD00097F83F30002B3CD007F11003234A2A210B
:101DE00018460DF0D0F80BF0B3FC03461A4607F185
:101DF00010032A2118460DF01FFA07F110031C4AA0
:101E00002A2118460DF0E4F897F83D2007F1100359
:101E10002A2118460DF010FA07F11003154A2A215D
:101E200018460DF0D5F897F8462007F110032A213F
:101E300018460DF001FA07F110030A222A2118466C
:101E40000DF0F9F80C4A07F11003114618460CF092
:101E5000A6FC142305E03A6CBB681A60002300E07E
:101E60001B2318464837BD4680BD00BFA826010089
:101E7000B4260100BC260100FD13000080B590B01F
:101E800002AF7860AC4B40F20322AC49002003F073
:101E9000C5F8AB4B00221A7002E00A2008F08AFB5A
:101EA000A84BDB689847034683F00103DBB2002BA5
:101EB000F3D1A54A3021A2480CF000FE0346002BC6
:101EC000EED1002387F83630FF2387F82F30FF2329
:101ED00087F82E309A4B1B78402B40F09C80984816
:101EE0000FF013FF03460A2B40F29580974B1B78A7
:101EF000002B08D0924B0093954B40F215228F494E
:101F0000002003F08BF8002387F8363007F12E030A
:101F100007F12F0207F130018948FFF7F9FE034668
:101F200087F8373097F83730142B06D1894B1422B5
:101F30001A70012387F8363076E097F83730002B97
:101F400072D11B2387F837303B6B834918460FF05B
:101F5000CAFE0346002B0AD1012387F836307D4B99
:101F60001B7887F837307B4B00221A705CE03B6BA4
:101F70007A4918460FF0B7FE0346002B06D101231D
:101F800087F836301B2387F837304DE03B6B05224E
:101F9000734918460FF0C1FE0346002B23D104F00D
:101FA00049FC3B6B05333B6397F82E30002B09D17E
:101FB0003B6B01226B49184600F038FB034687F85B
:101FC000373008E03B6B01226749184600F02EFBD2
:101FD000034687F837305F4A97F83730137001238C
:101FE00087F8363020E03B6B604918460FF07BFEE7
:101FF0000346002B03D1002387F8363014E03B6BF7
:102000005B4918460FF06FFE0346002B0CD10023EE
:1020100087F8363008E0574A302149480CF0D8FF9D
:10202000474800F01DFB00E000BF454B00221A703E
:1020300097F83630002B3FF433AF97F82E30002B53
:102040003FF42EAF07F10C034B4A202118460CF049
:102050009AFF97F82F2007F10C03202118460DF066
:10206000EBF807F10C032022202118460CF0E3FFC7
:102070000BF06EFB03461A4607F10C0320211846AD
:102080000DF0DAF807F10C032022202118460CF09D
:10209000D2FF07F10C030022202118460DF0CCF8E6
:1020A00097F83730002B07D107F10C032F4A202176
:1020B00018460CF08DFF06E007F10C032C4A202196
:1020C00018460CF085FF07F10C0318460BF0B3FB24
:1020D000034687F8353097F835301B0987F83430D8
:1020E00097F83430092B01D8302200E0372297F8D6
:1020F00034301344DBB2FB7497F8353003F00F0330
:1021000087F8343097F83430092B01D8302200E0BA
:10211000372297F834301344DBB23B7507F10C03D8
:102120000A22202118460CF086FF07F10C031846FE
:10213000FFF7D8F9B4E600BFCC260100282501003E
:10214000AC0200200C3D0100F8240100E91300203E
:10215000E0260100EB130020E8260100F82601002C
:1021600018250100E8240100D824010004270100FB
:1021700008270100844101001425010080B582B0C8
:1021800002AF04F0EFFE0023019304230093002329
:1021900040F24512144915480FF0AAFA0346012BE4
:1021A00007D0134B40F26B221249052002F036FF94
:1021B000FEE704200EF053FB03460F4A13600E4B5C
:1021C0001B68002B07D10D4B4FF41C7209490520E9
:1021D00002F024FFFEE7084B1B680949184608F087
:1021E0002DF900BFBD4680BD102701007D1E0000F7
:1021F0001827010028250100A8000020342701002D
:102200006027010080B582B000AF78607B685B68B2
:102210001A46164916480CF0F9FC7B685B681A46AA
:10222000144915480CF0F2FC7B685B681A461349A8
:1022300013480CF0EBFC7B685B681A4611491248A6
:102240000CF0E4FC7B685B681A46104910480CF0FF
:10225000DDFC7B685B681A460E490F480CF0D6FC23
:10226000002318460837BD4680BD00BF7027010017
:102270008C2701006424010098270100A027010099
:10228000DC270100F8270100102801001C280100AC
:10229000582801006C2801008828010080B584B00E
:1022A00000AFF860B9607A607B689B681946134894
:1022B0000CF075FA7B689B681946F8680CF06FFAA9
:1022C0007B689B6819460E480CF069FA7B689B682E
:1022D00019460C480CF063FA7B689B681946B8688D
:1022E0000CF05DFA7B689B68194605480CF057FABC
:1022F0001B2318461037BD4680BD00BFA028010033
:1023000084410100B828010084B080B500AF07F116
:10231000080C8CE80F000B4B18680023642207F1AF
:1023200008010EF012FB0346012B05D0064B3522A7
:102330000649032002F072FE00BFBD46BDE88040A2
:1023400004B07047DC020020C8280100F828010012
:10235000B0B59EB008AFF860B9607A60FB687B6585
:10236000FB68A14918460FF0BEFC0346002B07D0BE
:10237000FB689E4918460FF0B6FC0346002B07D1B8
:10238000BB6801221A707868FFF73CFF034626E11C
:10239000FB680F22964918460FF0BFFC0346002B3E
:1023A0006AD100233B650023FB64BB6801221A70DD
:1023B000FB680F33FB6007F14C0207F10C03114679
:1023C00018460DF023F80346002B09D1FB6C092BAE
:1023D0000DDD7A688749786DFFF760FF0346FEE000
:1023E0007A688549786DFFF759FF0346F7E0FB6887
:1023F0000133FB6007F1500207F10C031146184648
:102400000DF004F80346002B13D10023BB643B6D91
:10241000DBB207F1480211461846FEF75DF80346A5
:10242000002B0DD07A687549786DFFF737FF0346AA
:10243000D5E07A687249786DFFF730FF0346CEE049
:1024400007F114032C22002118460FF048FB022349
:10245000BB613B6DFB61FB6C3B626D4607F1240485
:102460000FCC0FC594E8070085E8070007F11403B7
:102470000FCBFFF749FFB1E0FB68624918460FF048
:1024800032FC0346002B1AD1BB6801221A7007F1F7
:1024900014032C22002118460FF021FB01233B7569
:1024A0006D4607F124040FCC0FC594E8070085E8BA
:1024B000070007F114030FCBFFF726FF8EE0FB6840
:1024C0001122514918460FF028FC0346002B2ED14B
:1024D000BB6801221A7007F114032C220021184650
:1024E0000FF0FDFA02233B750923BB61FB68113332
:1024F000FB6007F1140303F1080107F10C03092243
:1025000018460BF0B9F90346002B01D01B2366E0F7
:102510006D4607F124040FCC0FC594E8070085E849
:10252000070007F114030FCBFFF7EEFE56E0FB6840
:102530000F22364918460FF0F0FB0346002B4DD111
:1025400000237B6400233B64BB6801221A70FB6894
:102550000F33FB6007F1440207F10C0311461846E4
:102560000CF054FF0346002B06D07A682449786D9E
:10257000FFF794FE034632E0FB680133FB6007F18E
:10258000400207F10C03114618460CF03FFF0346CA
:10259000002B06D07A681E49786DFFF77FFE034650
:1025A0001DE007F114032C22002118460FF097FAC2
:1025B00004233B750223BB617B6CFB613B6C3B627C
:1025C0006D4607F124040FCC0FC594E8070085E899
:1025D000070007F114030FCBFFF796FE0023184600
:1025E0005837BD46B0BD00BFA83901000029010021
:1025F000102901002029010038290100502901007B
:102600007829010090290100A4290100B8290100BE
:10261000C829010080B400AF034B1B681846BD46B3
:102620005DF8047B704700BFDC02002080B584B0F9
:1026300000AFF860B9601346FB71BB68002B02D194
:1026400003F08CFCB860FB79044AB968F8680CF0B8
:1026500077F9034618461037BD4680BDE0290100D2
:1026600080B584B000AF78600023FB600FE00C49B8
:10267000FA6813465B0013449B000B441B685B68BD
:10268000194678680CF08BF8FB680133FB60FB6837
:10269000012BECD900BF00BF1037BD4680BD00BF85
:1026A000082A010090B585B000AF7860214BE52283
:1026B0002149022002F0B2FC0023FB600DE01F491B
:1026C000FA6813465B0013449B000B4404331B68F9
:1026D00000221A70FB680133FB60FB68012BEED906
:1026E0000023FB601FE01549FA6813465B001344A2
:1026F0009B000B44043318681049FA6813465B00CA
:1027000013449B000B44083319680C4CFA681346B9
:102710005B0013449B0023441A68094B0CF026FA13
:10272000FB680133FB60FB68012BDCD9142007F048
:1027300041FFD5E7202A0100F8280100082A0100FE
:10274000E029010080B582B002AF0023019302238B
:1027500000930023C8222C492C480EF0C9FF0346E1
:10276000012B06D02A4BFC222A49052002F056FCF8
:10277000FEE7294803F0E2FB0346002B1FD0274B5E
:102780004FF481722349032002F048FC03F084FADD
:102790000346184603F0D2FB0346002B07D0204B1C
:1027A00040F205121B49052002F038FCFEE71D4BE4
:1027B0004FF484721749022002F030FC06E01A4BF5
:1027C00040F20B121349022002F028FC00222C21B7
:1027D00005200DF0C0FF0346144A1360134B1B681D
:1027E000002B07D1124B40F20F120A49052002F0CC
:1027F00015FCFEE70D4B1B680E49184607F01EFE40
:1028000000BFBD4680BD00BF342A0100A5260000E0
:102810003C2A0100F8280100D83B0100582A010099
:10282000842A0100AC2A0100C02A0100DC02002039
:10283000D42A0100F82A010080B588B002AF786080
:10284000182007F071FA78617B685033184602F05F
:10285000F9F802467B699A607B68184603F08EFEA1
:1028600002467B695A6004200DF0F9FF02467B693D
:10287000DA600022012105200DF06DFF02467B6920
:102880001A617B6893F865207B691A707B6893F8FE
:1028900064207B695A707B6900221A754FF6FF73BA
:1028A000FB817B6893F8653007F10E0211461846EC
:1028B000FEF7EEFB0346002B09D1B7F90E30002BD3
:1028C00005DBB7F90E30DAB27B695A7020E07B691C
:1028D0001B780093314B3B223149032002F09EFBD1
:1028E0007B6893F865207B6893F864309BB2194647
:1028F0001046FEF7EFFB0346002B09D07B6893F8E8
:1029000065300093274B3E222549042002F086FBC8
:102910007B691B69002B09D17B691B780093224BD3
:1029200044221F49042002F079FBFEE77B691B6902
:102930001E49184607F082FD7B69DB68002B09D130
:102940007B691B7800931A4B4C221549042002F036
:1029500065FBFEE77B69DB681649184607F06EFDEC
:1029600000230193002300937B69C8221249134876
:102970000EF0BEFE38613B69012B09D07B691B78E4
:1029800000930F4B5B220649042002F047FBFEE751
:102990007B6918461837BD4680BD00BF082B010073
:1029A0005C2B0100682B0100AC2B0100DC2B01002B
:1029B000E82B0100202C0100342C0100A92D00007F
:1029C000382C010080B58AB004AF786000237B61A9
:1029D0000023FB607B685B7807F10C021146184608
:1029E000FDF77AFD0346002B0ED1FB687A6812785A
:1029F00011467A685278029201910093644B7922D1
:102A00006449022002F00AFBFB68002B0ADA7B68AB
:102A10005B780093604B7E225E49022002F0FEFA52
:102A20000023FB607B681B7D022B0AD17B681B782F
:102A300000935A4B83225749032002F0EFFA0123F7
:102A4000A2E07B681B7D032B0AD17B681B78009377
:102A5000534B87224F49032002F0E0FA002393E012
:102A600078680BF027F80346002B61D07B680122C1
:102A70001A7507E07B685B6818460CF001FA1420B1
:102A800007F098FD78680AF0EDFF0346002BF1D1BE
:102A90007B685B6818460CF0C3F90EE07B685B68E6
:102AA000012118460CF07EF90346002B02D07B6909
:102AB00001337B61012007F07DFD78680AF0D2FFC9
:102AC000034683F00103DBB2002B03D07B69B3F52F
:102AD000007FE3DB7B685B6818460CF0BFF97B691D
:102AE000B3F5007F11DA00233B610AE07B685B6885
:102AF00018460CF0C5F9142007F05CFD3B69013362
:102B00003B61FB683A699A42F0DB7B685B680021B5
:102B100018460CF0D8F97B685B68184603F0B8FDDE
:102B2000786800F007FA7B69B3F5007F10DA0DE0F2
:102B30007B6800221A757B681B780093194BB822BA
:102B40001449042002F06AFA00231DE0022200E08A
:102B500000227B681A757B681B781A467B681B7D90
:102B6000022B01D1104B00E0104B01930092104B4F
:102B7000BE220849022002F051FA7B681B7D022B1D
:102B80000CBF01230023DBB218461837BD4680BDB9
:102B9000642C01005C2B0100B42C0100182D0100F5
:102BA0006C2D0100C02D010008220100102201003F
:102BB0001C2E010080B584B002AF786039607B685C
:102BC0001B7D022B3BD178680AF074FF0346002B73
:102BD0002BD07B6803221A757B685B6818460CF063
:102BE0001FF90EE07B685B68012118460CF0DAF8EB
:102BF0000346002B02D03B68013B3B60012007F0FD
:102C0000D9FC3B68002BEDD17B685B6818460CF063
:102C100025F97B685B68184603F03AFD7B68022261
:102C20001A75786800F086F912E07B681B780093CB
:102C3000094BE6220949042002F0F0F908E07B681C
:102C40001B780093064BE9220449042002F0E6F9C0
:102C500000BF0837BD4680BD602E01005C2B01001F
:102C6000B02E010080B588B002AF78600B46FB70D3
:102C700078680AF01FFF0346002B46D007F10E02CA
:102C8000FB781146184600F075F903461B2B0BD153
:102C9000FB7800931E4BF7221E49042002F0BEF978
:102CA000786800F047F930E078680AF0E9FE0346FA
:102CB0005A42C3F30803C2F3080258BF53423B61B0
:102CC00000237B61FB891A463B6993421AD0FB893A
:102CD0001A463B69934206DD3B69C3F50073FA89E6
:102CE00013447B6109E0FB891A463B69934204DA8D
:102CF000FB891A463B69D31A7B617B691946786860
:102D0000FFF758FF786800F015F91837BD4680BD09
:102D1000042F01005C2B010080B584B002AF786005
:102D20000B46FB707B681869F91C002364220DF0C8
:102D30000CFE0346012B09D07B681B780093054BE2
:102D400040F20F120449042002F068F900BF08376E
:102D5000BD4680BD382F01005C2B010080B584B0DA
:102D600002AF78600B46FB707B68FA785A707B681C
:102D70001B78FA7892B211461846FEF7ABF9034673
:102D8000002B09D07B681B780093054B40F217128B
:102D90000449042002F042F900BF0837BD4680BD57
:102DA0007C2F01005C2B010080B588B002AF7860F9
:102DB0007B687B617B693B612023BB730023FB73D2
:102DC0003B691B780093504B4FF497724F49022098
:102DD00002F024F9322007F0EDFB3B691B7D022B4A
:102DE00029D0022B00F38180002B00F08680012B7C
:102DF0007BD13B691B780093454B4FF49E7243494E
:102E0000022002F00BF97869FFF7DCFD0346FB7343
:102E10003B691B781A46FB7B002B01D03D4B00E041
:102E20003D4B019300923D4B4FF49F723749022076
:102E300002F0F4F866E03B691B6907F10E0100221D
:102E400018460EF034F90346012B58D13B691B7824
:102E5000BA7B01920093324B40F249122B49022077
:102E600002F0DCF878690AF025FE0346002B48D012
:102E70003B691B6907F10E01002218460DF073FF34
:102E80000346012B0DD03B691B780093254B40F284
:102E900051121E49042002F0C1F8786900F04AF886
:102EA00030E03B691B78BA7B019200931E4B40F2E5
:102EB00057121649022002F0B1F8BB7B1946786917
:102EC000FFF7D0FE3B691B78BA7B01920093174B4A
:102ED00040F259120D49022002F0A0F8642007F0D8
:102EE00069FB786900F026F80BE0114B4FF4B172E2
:102EF0000649032002F092F804E000BF6AE700BF31
:102F000068E700BF66E700BFD42F01005C2B01001B
:102F100000300100082201001022010050300100A1
:102F200084300100C4300100F43001001831010088
:102F30004031010080B584B002AF78607B68DB6807
:102F400018460DF0A4FC0346012B0AD07B681B78C1
:102F50000093064B4FF4BC720549042002F05EF862
:102F6000FEE700BF0837BD4680BD00BF64310100E9
:102F70005C2B010080B485B000AF03463960FB7163
:102F80000023FB6012E00E4AFB6812F82330FA7946
:102F90009A4208D10A4AFB689B0013445A883B684E
:102FA0001A80002306E0FB680133FB60FB68272BD7
:102FB000E9D91B2318461437BD465DF8047B7047DA
:102FC0009C31010080B483B000AF7860084B1B686F
:102FD00023F440227B689B0403F4402304491343F9
:102FE0000B6000BF0C37BD465DF8047B704700BF27
:102FF0000070044080B483B000AF78600A4B03F5E2
:1030000080535B6823F440327B681B0403F4403335
:103010000549134301F58052536000BF0C37BD468C
:103020005DF8047B704700BF0070044080B582B03B
:1030300000AF1A4B1B7BDBB203F00303022B22D041
:10304000022B23D8002B02D0012B0ED01EE0144BF4
:103050001B68002B05D1134B134ADA211348FDF7E7
:1030600027FA0F4B1B687B6013E0114B1B68002B8A
:1030700005D1104B0C4ADF210C48FDF719FA0C4B17
:103080001B687B6005E00C4B7B6002E000237B60EB
:1030900000BF7B6818460837BD4680BD004006402B
:1030A000E00200203C320100983201005032010061
:1030B000E40200205C320100006CDC0280B582B0CA
:1030C00000AFFFF7B3FF7860254B1B78DBB2DB085E
:1030D000DBB203F00703FB70FB787A6822FA03F394
:1030E0007B601F4B5B78DBB21B09DBB203F0030391
:1030F000BB701B4B1B7BDBB203F003037B70BB7805
:10310000002B02D07B78002B02D07B78022B21D1C0
:10311000FB78072B14D0072B19DC052B02DC002BC6
:1031200003DA14E0062B04D011E07B685B097B60B6
:1031300011E07B680B4AA2FB03231B097B600AE0BA
:103140007B68094AA2FB0323DB087B6003E00023C2
:103150007B6000E000BF7B6818460837BD4680BD35
:1031600000400640CDCCCCCCABAAAAAA80B483B098
:1031700000AF0E4B9B79DBB203F00103002B03D1B0
:103180000B4B1B687B600AE00A4B1A68074B1B7AE3
:10319000DBB25B0803F0070322FA03F37B607B6872
:1031A00018460C37BD465DF8047B7047004006406A
:1031B000100000201400002080B582B000AF094B41
:1031C0009B79DBB203F01003002B03D1FFF776FFEE
:1031D000786002E0044B1B687B607B681846083708
:1031E000BD4680BD004006401000002080B500AF05
:1031F0000B4B1B78DBB25BB2002B0DDA094B1B6863
:10320000002B06D1084B094A4FF4B3710848FDF76B
:103210004FF9044B1B6800E00023184680BD00BF37
:1032200000500640E002002070320100B032010080
:103230005032010080B582B000AF134B1B78DBB277
:103240005BB2002B18DA114B1B68002B06D1104B18
:10325000104A40F27B111048FDF72AF90A4B9B787F
:10326000DBB223F03F03FB70084B1B68FA7892092E
:10327000D2B2D3407B6001E000237B607B681846BC
:103280000837BD4680BD00BF00500640E002002068
:1032900070320100CC3201005032010080B582B0A2
:1032A00000AF1A4B1B689B0C03F00303032B21D0C8
:1032B000032B23D8002B02D0022B0CD01EE0FFF7EB
:1032C00095FF0346B3F5004F02D14FF4004300E0F1
:1032D00000237B6015E00E4B1B68002B06D10D4BC5
:1032E0000D4A4FF4CB710D48FDF7E2F8084B1B680F
:1032F0007B6006E04FF47A737B6002E000237B6022
:1033000000BF7B6818460837BD4680BD007004408A
:10331000E40200207C320100E8320100503201005A
:1033200080B582B000AF114B03F580535B681B0C76
:1033300003F00303032B0ED0032B0FD8002B02D076
:10334000012B04D00AE000F005F9786009E000F0F4
:103350005BF9786005E0064B7B6002E000237B6050
:1033600000BF7B6818460837BD4680BD007004402A
:10337000006CDC0280B584B000AF0346FB71FB79C2
:10338000132B00F28E8001A252F823F0DD330000EF
:10339000DD330000FB330000193400003734000037
:1033A000A3340000553400005D3400009B3400005D
:1033B000A334000093340000653400006D34000035
:1033C000753400007D340000A3340000A3340000F5
:1033D000A3340000853400008B34000000F088F82E
:1033E0000246344B03F580535B6C1B0F03F00F0355
:1033F0000133B2FBF3F3FB6056E000F079F80246CC
:103400002C4B03F580535B6C1B0E03F00F03013351
:10341000B2FBF3F3FB6047E000F06AF80246254B8D
:1034200003F580535B6C1B0D03F00F030133B2FBFC
:10343000F3F3FB6038E000F05BF802461D4B03F548
:1034400080535B6C1B0C03F00F030133B2FBF3F3EF
:10345000FB6029E0FFF764FFF86025E0FFF71EFF3F
:10346000F86021E00AF041FBF8601DE000F0B4F8DC
:10347000F86019E000F06EF8F86015E000F0C4F8AC
:10348000F86011E00C4BFB600EE04FF47A73FB60C8
:103490000AE0FFF7ABFEF86006E0FFF7CBFEF8604E
:1034A00002E00023FB6000BFFB6818461037BD46F2
:1034B00080BD00BF00700440006CDC0280B582B0AB
:1034C00000AF7860094A7B685B6802F580525364FC
:1034D0007B681B781846FFF78DFD7B685B78184684
:1034E000FFF770FD00BF0837BD4680BD0070044087
:1034F00080B582B000AF164B9B79DBB29B0803F01E
:1035000003033B603B68032B1AD801A252F823F057
:103510002935000031350000393500002135000023
:1035200000F072F878600EE000F014F878600AE0BD
:10353000FFF71CFE786006E0FFF778FD786002E098
:1035400000237B6000BF7B6818460837BD4680BDFE
:103550000040064080B584B000AF1D4B5B78DBB205
:1035600003F00203002B06D1194B9B79DBB203F069
:103570002003002B02D00023FB6024E0FFF71CFE99
:10358000B860BB68002B02D1BB68FB601BE0104B2E
:10359000DB78DBB25B09DBB203F00303FB710C4B9E
:1035A000DB78DBB2DB09DBB203F00103BB71FA7934
:1035B000BB7908495200134431F813301A46BB68EE
:1035C00002FB03F3FB60FB6818461037BD4680BD65
:1035D000004006400033010080B582B000AF094BC7
:1035E0001B78DBB203F00203002B02D100237B60C7
:1035F00002E0FFF7BBFD78607B6818460837BD46E0
:1036000080BD00BF0040064080B584B000AF1C4BB9
:103610009B79DBB203F04003002B02D10023FB6057
:1036200028E00AF05BFAB860BB68002B06D1154BA6
:10363000154A40F21A311548FCF73AFF104B1B7936
:10364000DBB203F01F03DBB20133FB71FB79BA6815
:10365000B2FBF3F3BB600A4B5B79DBB203F01F03F1
:10366000DBB21833BB71BA79BB6802FB03F3BB60F2
:10367000BB68FB60FB6818461037BD4680BD00BFC5
:10368000004006408C32010010330100503201002E
:1036900080B485B000AF0346FB710B46BB71134687
:1036A0007B713B4B9B79DBB29B0803F00303FB6010
:1036B000374B9B79DBB203F00103FB72344B1B7A6F
:1036C000DBB25B08DBB203F00703BB727A79BB7A2B
:1036D0009A422CD02E4B1B78DBB203F00203002B56
:1036E00002D1FB68012B12D1FB7A012B0FD1284BA1
:1036F0005B78DBB2264A23F00103DBB2537000BFD4
:10370000234B9B79DBB203F00103002BF8D1204B54
:103710001B7ADBB223F02F03DAB27B795B00DBB2DA
:1037200003F00E03DBB21A491343DBB20B72184BE2
:103730005B78DBB223F00103DAB2BB7903F001035B
:10374000DBB213491343DBB24B70114B1B78DBB276
:1037500023F00303DAB20E49FB791343DBB20B709B
:10376000FB68012B04D0FB7903F00203002B08D087
:1037700000BF074B9B79DBB203F00102BB799A4291
:10378000F7D1002318461437BD465DF8047B704717
:103790000040064080B584B000AF03463A60FB713C
:1037A0000B46BB710023FB73294BDB78BB73284BA3
:1037B0009B79DBB203F01003002B09D10123FB73CB
:1037C000234BDB78DBB2224A83F02003DBB2D370D9
:1037D0001F4B1B78DBB203F03B03DBB21C4A43F008
:1037E0000403DBB2137000BF194B9B79DBB21B09DA
:1037F00003F00103012BF7D1FB7B002B02D0144A0D
:10380000BB7BD370BB7B03F01F03DAB2FB79DB0118
:10381000D9B2BB795B01DBB203F06003DBB20B43CF
:10382000DBB20B491343DBB2CB7000BF084B9B7973
:10383000DBB29B0803F00303002BF7D13B68002B9E
:1038400001D03B689847002318461037BD4680BD1D
:103850000040064080B582B000AF7860396078687B
:103860000AF070F90346002B05D0094B1B68396834
:103870007868984704E0074B1B6839687868984770
:10388000BFF34F8F00BF00BF0837BD4680BD00BFEC
:10389000F0020020F402002080B500AF094B1B6845
:1038A000002B06D1084B094A40F694010848FCF762
:1038B000FFFD044B1B6819460648FFF7CBFF00BF0E
:1038C00080BD00BFE80200205433010084330100B2
:1038D0004833010000C0024080B500AF094B5B686F
:1038E000002B06D1084B094A40F69D010848FCF719
:1038F000DFFD044B5B6819460648FFF7ABFF00BFCE
:1039000080BD00BFE80200206C3301009C33010041
:103910004833010000D0024080B582B000AF78602B
:103920007B68002B14D07B6800229A647B6800229D
:10393000DA637B6800221A64074A7B689A647B68B2
:103940009B6C184600F048F978680AF00EF900E020
:1039500000BF0837BD4680BDF802002080B58AB0A0
:1039600000AFF860B9607A603B60FB6893F8343070
:103970007A68B968F8680AF028F938623B6A002B5F
:1039800001D03B6A43E0386800F06CF938623B6A6A
:10399000002B01D03B6A3AE0FB681B6BFB61FB68C4
:1039A0001B69BB61FA697B681344013B7B627B6ADC
:1039B000BA69B3FBF2F2B96901FB02F29B1A002B60
:1039C0001ED07A6ABB69B2FBF3F301337B617B697A
:1039D000BA6902FB03F3013B7B6211E0FB6923F050
:1039E0007F430D4A43F010631360F86800F004F958
:1039F00038623B6A002B08D1FA69BB691344FB614A
:103A0000FA697B6A9A42E9D900E000BF3B6A18462E
:103A10002837BD4680BD00BF0400024090B589B084
:103A200000AFF860B9607A603B60FB6893F83930AA
:103A3000FB747B68002B01D1042353E0FB7C3A68C4
:103A4000B968F8680AF0C1F8F861FB69002B01D089
:103A5000FB6947E0FB681B6BBB613B687B613BE03C
:103A6000224B1C1D78680AF0E3F8034623607B684C
:103A700004337B60FB7C042B07D1BB6923F07F43BD
:103A80001A4A43F0C063136017E0FB7C082B12D185
:103A9000164B03F1080478680AF0CAF8034623605D
:103AA0007B6804337B60BB6923F07F430F4A43F09C
:103AB000E063136001E0042314E0F86800F09CF870
:103AC000F861FB69002B0BD1FB7CBA691344BB6125
:103AD000FB7C7A69D31A7B617B69002BC0D100E043
:103AE00000BFFB6918462437BD4690BD0400024064
:103AF00080B58CB000AFF860B9607A60FB70FB688D
:103B000093F83530FB77FB7F7A68B968F8680AF07C
:103B10005CF8B861BB69002B01D0BB6955E0FB685C
:103B20001B6B7B62FB68DA68FB685B69B2FBF3F3D3
:103B30007B617A6A7B6913445A1E7B695B4213403E
:103B4000FB62FA6A7B6A9A4203D1FA6A7B69134480
:103B5000FB627B68BB6234E0FA6A7B6AD31A3B6221
:103B60003A6ABB6A9A4201D9BB6A3B62FB7F3A6AF6
:103B7000B2FBF3F33B617B6A23F07F43154A43F0CA
:103B8000807313603B691A04FB781B021A43114BC4
:103B9000043342F0FF021A60F86800F02DF8B861B3
:103BA000BB69002B01D0BB690FE0BA6A3B6AD31A2C
:103BB000BB627A6A3B6A13447B62FA6A7B6913448C
:103BC000FB62BB6A002BC7D1002318463037BD46C5
:103BD00080BD00BF0400024080B582B000AF7860B5
:103BE0000C22044978680DF06CFF00BF0837BD4611
:103BF00080BD00BFB433010080B584B000AF7860F1
:103C0000174B70221A707B689B6C5A1C7B689A64F5
:103C10007B689B6CFB60FB68114898477B689B6CDA
:103C20005A1E7B689A640E4B1B78FB72FB7A03F07A
:103C30002003002B01D067230EE0FB7A03F0100372
:103C4000002B01D0682307E0FB7A03F00103002B6F
:103C500001D0692300E0002318461037BD4680BD1F
:103C60000000024080B483B000AF78607B68064AF1
:103C7000934201D06B2300E0002318460C37BD4669
:103C80005DF8047B704700BF6B66656B80B487B0DE
:103C900000AFF8600B467A60FB72FB68002B02D025
:103CA0007B68002B01D104238AE000237B61FB7A2F
:103CB000212B00F2818001A252F823F0453D000043
:103CC0004F3D0000593D00006B3D0000753D000078
:103CD0007F3D0000913D00009B3D0000B93D00008C
:103CE000B93D0000B93D0000B93D0000B93D0000FC
:103CF000B93D0000B93D0000B93D0000B93D0000EC
:103D0000B93D0000B93D0000B93D0000B93D0000DB
:103D1000B93D0000B93D0000B93D0000B93D0000CB
:103D2000B93D0000B93D0000B93D0000B93D0000BB
:103D3000B93D0000B93D0000B93D0000A53D0000BF
:103D4000AF3D0000FB681A697B681A6037E0FB68CA
:103D5000DA687B681A6032E0FB68DA68FB685B69E6
:103D6000B2FBF3F27B681A6029E0FB685A697B6852
:103D70001A6024E0FB689A687B681A601FE0FB68A1
:103D80001B79C3F30013DBB21A467B681A6016E096
:103D9000FB68DA697B681A6011E0FB681A6A7B6865
:103DA0001A600CE0FB68DA6B7B681A6007E0FB685E
:103DB0001A6C7B681A6002E06A237B6100BF7B6932
:103DC00018461C37BD465DF8047B704780B485B04B
:103DD00000AF78600B46FB707B681833FB607B6834
:103DE0009A68FB681A600C4B93F82830DBB21A46CD
:103DF0004FF4807303FA02F2FB685A60064B93F8A3
:103E00002B30DBB21A46FB689A6000BF1437BD4600
:103E10005DF8047B704700BF0000024080B487B0AB
:103E200000AFF860B9607A603B60104B03F58053D7
:103E3000DA6C7B681A403B6822FA03F3FB74FB7C64
:103E40000F2B05D1FB68BA6802FB03F37B6105E029
:103E5000FB7C074A32F813309B027B617B69184672
:103E60001C37BD465DF8047B704700BF00700440FE
:103E7000C033010080B584B000AFF860B9607A60EB
:103E80007B68002B05D1144B144A64211448FCF7BD
:103E90000FFB7B681B78002B0AD1FB685A69012154
:103EA000BB6801FA03F3DB431A40FB685A610FE079
:103EB0007B685B781A46B968F8680AF01CF9FB68F9
:103EC0005A690121BB6801FA03F31A43FB685A617E
:103ED00000BF1037BD4680BD103401002034010002
:103EE0000434010080B584B000AF786039607B682D
:103EF000DB78FB737B689B78BB73BB7B03F0200391
:103F0000002B04D1FB7B03F01003002B05D0094BE1
:103F10001B6839687868984704E0074B1B68396864
:103F200078689847BFF34F8F00BF00BF1037BD467A
:103F300080BD00BF400300204403002080B500AFD7
:103F4000034B1B6819460348FFF7CCFF00BF80BD39
:103F5000380300200060064080B500AF034B5B686B
:103F600019460348FFF7BEFF00BF80BD380300209D
:103F70000070064080B584B000AF78600023FB601D
:103F800006E00D4A7B68934206D0FB680133FB6074
:103F9000FB68002BF5D000E000BFFB68002B05D0CC
:103FA000064B074A7B210748FCF782FAFB68184654
:103FB0001037BD4680BD00BF00A002403034010074
:103FC000943401005834010080B58CB000AFF86023
:103FD000B9607A60BB68002B05D19F4B9F4AF221E4
:103FE0009F48FCF765FABB681B68002B05D19D4B09
:103FF0009A4AF3219A48FCF75BFA0023FB62BB68FC
:104000001B68FB61002387F823300023FB84042313
:1040100087F8223041E07A6813469B0013445B0026
:104020001946BB681B6897F8222002FB03F3B1FB1B
:10403000F3F305338C4AA2FB0323DB08BB84BB8C60
:10404000002B01D10123BB8497F82230BA8C02FBEC
:1040500003F37A68B2FBF3F37B61BB681B687A6990
:104060009A4204D9BB681B687A69D31A03E0BB681B
:104070001A687B69D31A3B613A69FB699A4207D88F
:104080003B69FB6197F8223087F82330BB8CFB84B7
:1040900097F82230013387F8223097F82230202B0E
:1040A000B9D9BB681B68714AA2FB03235A0913469E
:1040B0005B001344FA699A4203D940F22153FB6230
:1040C000C5E0F868FFF756FFB861694B18460AF07B
:1040D0002DF8FB689B6823F44022FB689A60FB681C
:1040E0001B68BB6297F82330032B07D997F823305E
:1040F000072B03D8BB6A43F40033BB62BB6A23F0CF
:10410000F853BB6297F82330013B1B0603F0F853CA
:10411000BA6A1343BB62BB6A23F4FF5323F01F0345
:10412000BB62FB8CC3F30C02BB6A1A43FB681A60C8
:10413000FB681B6823F00052FB681A60FB689B68F1
:1041400023F4E26323F00703BB62BB681B791A46C2
:10415000BB685B7B1B0203F4E0631A43BB681B7BF9
:104160009B0003F004031343BA6A1343BB62BB68AA
:104170001B79002B03D0BB6A43F01003BB62FB68C2
:10418000BA6A9A60FB681B6823F40053BB62BB6881
:10419000DB795B0303F40052BB6A1A43FB681A60C5
:1041A000344BBB62BB6A43F00043BB62BB6A43F45F
:1041B0004043BB62FB685A69BB68DB7A1B0103F0B2
:1041C0001001BB689B7A5B0103F020030B431A4389
:1041D000FB685A61BB681B7A002B05D0FB685B69E2
:1041E00043F00802FB685A61BB685B7A002B05D07C
:1041F000FB685B6943F00102FB685A61BB689B790D
:10420000002B04D0BB6A43F00053BB6203E0BB6ADF
:1042100023F00053BB62FB685A68BB6A1A43FB6811
:104220005A60FB689B68BB62BB689B7B002B03D01A
:10423000BB6A43F40023BB62BB68DB7B002B03D06B
:10424000BB6A43F48023BB62FB68BA6A9A60FB6A6C
:1042500018463037BD4680BD10340100A834010037
:104260005834010078340100CDCCCCCC1F85EB5103
:104270000A003C1000001F4080B582B000AF78609B
:104280007B68002B06D11C4B1C4A40F206211C48BF
:10429000FCF70EF91022002178680DF020FC7B68F5
:1042A0004FF4E1321A607B6800221A717B680022A9
:1042B0005A717B6800229A717B680022DA717B68F0
:1042C00000221A727B6800225A727B680022DA721E
:1042D0007B6800229A727B6800221A737B68002236
:1042E0005A737B6800229A737B680022DA7300BFDE
:1042F0000837BD4680BD00BF10340100B434010052
:104300005834010080B485B000AF786039603A68F5
:10431000154B13403B607B681B68FB603B681B02CE
:1043200003F40043FA681343FB603B6823F0800307
:104330003B603B681B0203F48043FA681343FB6055
:104340003B6823F040033B607B68FA681A607B6837
:104350009A683B681A437B689A6000BF1437BD4671
:104360005DF8047B704700BFC0C0F00F80B485B01B
:1043700000AF78607B685B68FB60FA68044B1340B1
:10438000FB60FB6818461437BD465DF8047B704738
:1043900000C0FFC180B584B000AF786039603A6872
:1043A0000F4B13403B607B685B6803F078533A68BF
:1043B0001343BB607B68BA685A607868FFF7D6FF22
:1043C00002463B681340002B03D040F21A53FB60B7
:1043D00001E00023FB60FB6818461037BD4680BD36
:1043E00000C01FC080B586B000AFF860B9607A60C9
:1043F000BB68002B06D1164B164A40F29631164880
:10440000FCF756F8BB687B617B683B6111E000BF3D
:10441000FB685B6803F40003002BF9D07B691B7811
:104420001A46FB68DA607B6901337B613B69013BBB
:104430003B613B69002BEAD100BFFB685B6803F47A
:104440008003002BF9D0002318461837BD4680BDE5
:1044500068340100CC3401005834010080B584B0C8
:1044600000AF78600323BB600023FB6009E00F4AC4
:10447000FB6852F823307A689A4207D0FB68013310
:10448000FB60FA68BB689A42F1D300E000BFFA68AB
:10449000BB689A4205D3064B064A8E210648FCF7B4
:1044A00007F8FB6818461037BD4680BDE4340100AC
:1044B000FC340100E03501001835010080B58AB0F8
:1044C00000AFF860B9607A60BB68002B05D19D4BE6
:1044D0009D4AD7219D48FBF7EBFFBB681B68002B6B
:1044E00005D19B4B984AD8219848FBF7E1FFFB6820
:1044F000984A93420DD0FB68974A934207D0FB68D5
:10450000964A934201D1012304E0FF2302E00123F4
:1045100000E00823BA685279934205DA904B8A4A40
:10452000DA218A48FBF7C4FFFB688A4A93420DD020
:10453000FB68894A934207D0FB68884A934201D1BD
:10454000012304E0FF2302E0012300E00823BA680E
:104550009279934205DA834B7B4ADB217B48FBF758
:10456000A7FF00237B62002387F823300023FB6131
:10457000BB681B681B017A68B2FBF3F37B627B6A42
:10458000002B01D101237B620023BB617B685A00B1
:10459000BB681B68B2FBF3F27B6A5B01D31A7B61D9
:1045A0007B685A007B6A59017B690B44B2FBF3F3C9
:1045B000BB61BB681B68BA699A4204D9BB681B68B7
:1045C000BA69D31A03E0BB681A68BB69D31AFB61E6
:1045D000BB681B68644AA2FB03235A0913465B00AD
:1045E0001344FA699A4202D940F2F533A5E0F8681B
:1045F000FFF734FF03465D4A52F82330184609F0AE
:10460000DDFDFB68DB78DBB223F00C03DAB2FB687C
:10461000DA70FB681B78DBB25BB223F01F035AB27F
:104620007B6A1B0A5BB213435BB2DAB2FB681A7097
:104630007B6ADAB2FB685A70FB689B7ADBB223F0C4
:104640001F03DAB27B69DBB203F01F03DBB2134353
:10465000DAB2FB689A72FB689B78DBB223F017032F
:1046600087F82330BB685B7A9B00DBB203F004035E
:10467000DAB297F82330134387F82330BB681B79ED
:10468000002B09D0BB681A7997F823301343DBB2AB
:1046900043F0100387F82330FB6897F823209A70C3
:1046A000BB685A79FB68DA74BB689A79FB685A75FB
:1046B000FB681B7CDBB263F07703DAB2FB681A7429
:1046C000FB685B7CDBB263F03F03DAB2FB685A74D1
:1046D000BB68DB79002B07D0FB685B7BDBB243F068
:1046E0000803DAB2FB685A73BB681B7A002B07D049
:1046F000FB685B7BDBB243F00103DAB2FB685A7301
:10470000FB68DB7887F82330BB689B7A002B05D0E9
:1047100097F8233043F0080387F82330BB68DB7A2F
:10472000002B05D097F8233043F0040387F823309B
:10473000FB6897F82320DA70002318462837BD4617
:1047400080BD00BF24350100F4350100183501009B
:104750003435010000A0064000B0064000C006400D
:1047600050350100983501001F85EB51F0340100F0
:1047700080B582B000AF78607B68002B06D1164B05
:10478000164A40F28F111648FBF792FE0C220021C8
:1047900078680DF0A4F97B684FF4E1321A607B6809
:1047A00000221A717B6800225A717B6801229A717B
:1047B0007B680022DA717B6800221A727B68002213
:1047C0005A727B6800229A727B680022DA7200BFFC
:1047D0000837BD4680BD00BF24350100003601000A
:1047E0001835010080B483B000AF786039603A6852
:1047F000174B13403B607B681B78DAB23B68DBB237
:104800001343DAB27B681A707B68DB78DAB23B68F4
:104810001B0ADBB21343DAB27B68DA707B689B79E0
:10482000DAB23B681B0CDBB21343DAB27B689A71D5
:104830007B685B7CDAB23B681B0EDBB21343DAB2F7
:104840007B685A7400BF0C37BD465DF8047B704727
:10485000C0F00F0780B500AF054B1B68054A5268D2
:10486000114605489847BFF34F8F00BF00BF80BD7A
:10487000540300204803002000B0064080B500AF7C
:10488000054B1B68054A9268114605489847BFF3D7
:104890004F8F00BF00BF80BD54030020480300209D
:1048A00000C0064080B500AF0B4BD3F888300A4AF1
:1048B00043F47003C2F88830084B4CF22052DA817E
:1048C000064B4DF62812DA81044B4FF4E9721A8038
:1048D00009F081FD00BF80BD00ED00E00020054033
:1048E00080B483B000AF78600A4B03F580535B68F7
:1048F00023F040627B689B0603F040630549134345
:1049000001F58052536000BF0C37BD465DF8047B53
:10491000704700BF0070044080B400AF054B03F542
:1049200080531A46044B536400BFBD465DF8047BB8
:10493000704700BF007004400000230180B500AF45
:10494000FFF7EAFF0023002101221846FEF7A0FE30
:1049500000230021074A184609F0E1F80648FEF74F
:10496000ADFD064B4FF0A0721A600120FFF7B8FFB3
:1049700000BF80BDF3E300001836010018000020DE
:1049800080B500AF1D4809F05BFD032210211C48D3
:1049900009F070FD1A4B1B6C23F0807323F00303A6
:1049A000174A43F00303136403221121144809F04A
:1049B00061FD134B5B6C23F0807323F00303104AFB
:1049C00043F003035364032202210D4809F052FD12
:1049D0000B4B9B6823F0807323F00303084A43F0DA
:1049E00003039360074B03F580531B69054A23F0CB
:1049F000030302F58052136100BF80BD0A00381026
:104A000000A004400070044080B582B000AF786020
:104A10007B68002B05D1074B074A67210748FBF746
:104A200047FD1422064978680DF04BF800BF08379F
:104A3000BD4680BD343601006C36010044360100AD
:104A40002036010080B584B000AF78607B68002B11
:104A500005D1214B214AE0212148FBF729FD1420F3
:104A600005F062F9F860FB68002B05D11D4B1B4A6D
:104A7000E7211B48FBF71CFDFB68002B10D014221C
:104A80000021F8680DF02BF87B681A78FB681A7023
:104A9000FB68181D7B680433102219460DF011F8CD
:104AA0007B6819787B685B781A46F86809F050FDD6
:104AB0007B681B7C1946F86809F087FD7B6898685D
:104AC0007B68DB680122194609F025FDFB68184662
:104AD0001037BD4680BD00BF343601008836010066
:104AE000443601005C36010080B584B000AF7860C8
:104AF0000B46FB707B68002B06D1134B134A40F228
:104B000097111348FBF7D4FC7B68FB60FB78002B04
:104B10000BD0FB685A68FB68DB68012101FA03F3DC
:104B20001946104609F0C9FC0AE0FB685A68FB68A0
:104B3000DB68012101FA03F31946104609F0CBFCAA
:104B400000BF1037BD4680BD503601009C360100C5
:104B50004436010080B584B000AF78607B68002BDC
:104B600006D10D4B0D4A4FF4E5710D48FBF7A0FC43
:104B70007B68FB60FB685A68FB68DB681946104677
:104B800009F0B7FC0346002B14BF01230023DBB25E
:104B900018461037BD4680BD50360100B0360100C2
:104BA0004436010080B483B000AF78607B681B6836
:104BB000214A13607B6804331B68204A13607B68BA
:104BC00008331B681E4A13607B680C331B681D4A40
:104BD00013607B6810331B681B4A13607B681433B7
:104BE0001B681A4A13607B6818331B68184A1360E5
:104BF0007B681C331B68174A1360174B1B68174AE6
:104C00001360174B1B68174A1360174B1B68174A32
:104C10001360174B1B68174A1360174B1B68174A22
:104C20001360174B1B68174A136000BE00BF0C3798
:104C3000BD465DF8047B7047580300205C030020EC
:104C40006003002064030020680300206C03002040
:104C5000700300207403002028ED00E0780300209A
:104C60002CED00E07C03002030ED00E0800300200C
:104C70003CED00E08403002034ED00E088030020D8
:104C800038ED00E08C03002080B582B000AF786082
:104C90007B68002B05D1074B074A3E210748FBF7ED
:104CA00007FC1422064978680CF00BFF00BF083798
:104CB000BD4680BD34360100E0360100D436010027
:104CC000C036010080B58AB000AF78607B68002BE9
:104CD00005D1294B294A47212948FBF7E9FB07F170
:104CE0000C031846FFF790FE00233B737B68191DE9
:104CF00007F10C030433102218460CF0E2FE7B6827
:104D00001B78002B0ED07B685B78002B14BF01232F
:104D10000023DBB283F00103DBB203F00103DBB25B
:104D20007B7302E07B685B787B7307F10C031846AA
:104D3000FFF788FE7862082004F0F6FF38623B6ACD
:104D4000002B05D10F4B0D4A56210D48FBF7B0FB48
:104D50003B6A002B0BD008220021386A0CF0BFFE02
:104D60003B6A7A6A1A607B681A783B6A1A713B6AF6
:104D700018462837BD4680BD34360100F83601009C
:104D8000D43601005C36010080B500AF064B9B684D
:104D9000002B06D0044B9B68034AD26801211046C1
:104DA000984700BF80BD00BF9003002080B500AFD2
:104DB000064B9B68002B06D0044B9B68034AD268C5
:104DC00000211046984700BF80BD00BF900300201F
:104DD00080B582B000AF78600B46FB70FB78002B8B
:104DE00005D0084B084A64210848FBF761FBFB78B3
:104DF000074904337A6841F8232000BF0837BD46CD
:104E000080BD00BF98370100E4370100C0370100C2
:104E10009003002080B483B000AF7860044A7B68C0
:104E2000936000BF0C37BD465DF8047B704700BF40
:104E30009003002080B483B000AF0346FB71044AA6
:104E4000FB79137000BF0C37BD465DF8047B7047DB
:104E50009003002080B483B000AF0346FB71044A86
:104E6000FB79537500BF0C37BD465DF8047B704776
:104E70009003002080B584B000AF78600B46FB70D3
:104E80007B68FB60FB68094A934206D1002004F06E
:104E900021FFB860BB68002B04D0FA78FB6810468D
:104EA000984700E000BF1037BD4680BD215C000080
:104EB00080B590B002AFF860B96011461A460B4653
:104EC000FB711346BB7100233B74BB79002B0DD0E3
:104ED0004D4B5B7D002B09D0FB794C4A52F82320C7
:104EE00007F11003202118460AF072F8FB79484AAE
:104EF00052F8232007F110000623009320232021DD
:104F00000AF02EFCBB79002B0AD03F4B5B7D002BB7
:104F100006D007F110033F4A202118460AF058F83E
:104F200007F11003FA6CB96C184609F0E1FB3B6C11
:104F30007B637B6B1B782E2B0CD102E07B6B0133E8
:104F40007B637B6B1B78202BF8D07B6B1B782E2B25
:104F5000F4D031E0386C0CF0D8FE0346013B3B63E3
:104F600002E03B6B013B3B633B6B012B0DD93B6B81
:104F7000013B3A6C13441B782F2B06D03B6B013B53
:104F80003A6C13441B785C2BEBD13B6B012B0FD19C
:104F90003B6B013B3A6C13441B782F2B08D03B6BC7
:104FA000013B3A6C13441B785C2B01D000233B631C
:104FB0003A6C3B6B13447B63FA6CB96C786B09F009
:104FC00097FB00233B7407F110033A222021184677
:104FD0000AF031F87A6C07F11003202118460AF024
:104FE000FDF907F110030C4A2021184609F0F0FFE3
:104FF00007F11003FA6CB96C184609F079FB00BF91
:105000003837BD4680BD00BF9003002080370100C7
:1050100068370100CC3701003424010008B480B5A2
:105020008BB004AF0346B9607A60FB73294B1B78E1
:10503000FA7B9A4247D3FFF7A7FE264B1B7D83F0EE
:105040000103DBB2002B3BD000237B6135E0214A1A
:105050007B69043352F82330002B2BD01D4A7B6927
:10506000043352F823309B68FA7B03931A4B029364
:105070007B680193BB680093012300210020FFF7A8
:1050800017FF07F128033B61124A7B69043352F88A
:10509000233099683B697A6A0F4802F0ADFA0D4AED
:1050A0007B69043352F823309B681A460A490B483F
:1050B00009F01EFB7B6901337B617B69002BC6DD38
:1050C000FFF774FE00E000BF1C37BD46BDE880401E
:1050D00001B0704790030020754E0000D03B0100E6
:1050E00080B588B000AF78600B46FB700023FB6092
:1050F000FB78002B23D0EFF30583FB61FB69002BCA
:1051000002D10023BB6101E00123BB61BB69002B1D
:105110000DD01D4B5B6807F10C02002118460CF006
:1051200087F8FB68002B2BD005F0D8F828E0164B49
:105130005B684FF0FF3118460BF0D7FB20E0EFF330
:1051400005837B617B69002B02D100233B6101E079
:1051500001233B613B69002B0DD00B4B5B6807F1D2
:105160000C02114618460BF075FDFB68002B07D0AA
:1051700005F0B4F804E0044B5B6818460BF087FBBD
:1051800000BF2037BD4680BD9003002080B500AF32
:1051900004200BF064FB03460E4A53600D4B5B6822
:1051A000002B00D1FEE70B4B5B680B49184605F05E
:1051B00045F90A48FFF72EFE0120FFF74BFE00F0ED
:1051C000CDFE0346034A13610020FFF733FE00BF04
:1051D00080BD00BF90030020D4370100E1500000E3
:1051E00080B500AF064B5B6818460CF0AAF8044B7C
:1051F00000225A600020FFF70DFE00BF80BD00BFF7
:105200009003002090B5B9B002AF7860002387F812
:10521000D33000233B7307F10C00042300932023B9
:10522000B54A20210AF09CFA7B685A6807F10C0302
:105230001146184609F0B3FA00233B7307F10C003E
:10524000072300932023AD4A20210AF089FA7B68C6
:105250005A6807F10C031146184609F0A0FA00231A
:105260003B7307F10C000B2300932023A44A202159
:105270000AF076FA7B685A6807F10C031146184663
:1052800009F08DFA00233B7307F10C000D23009306
:1052900020239C4A20210AF063FA7B685A6807F1B0
:1052A0000C031146184609F07AFA00233B7307F104
:1052B0000C00092300932023934A20210AF050FA7E
:1052C0007B685A6807F10C031146184609F067FA23
:1052D00000233B7307F10C000823009320238B4A23
:1052E00020210AF03DFA7B685A6807F10C03114649
:1052F000184609F054FA00233B7307F10C000B2306
:1053000000932023824A20210AF02AFA7B685A68F7
:1053100007F10C031146184609F041FA00233B73CC
:1053200007F10C000B23009320237A4A20210AF076
:1053300017FA7B685A6807F10C031146184609F002
:105340002EFA00233B7307F10C000823009320235F
:10535000714A20210AF004FA7B685A6807F10C03AD
:105360001146184609F01BFA00233B7307F10C00A5
:10537000152300932023694A20210AF0F1F97B6864
:105380005A6807F10C031146184609F008FA002381
:105390003B7307F10C00082300932023604A20216F
:1053A0000AF0DEF97B685A6807F10C0311461846CB
:1053B00009F0F5F900233B7307F10C00112300936A
:1053C0002023584A20210AF0CBF97B685A6807F15C
:1053D0000C031146184609F0E2F97B685B68194630
:1053E000514809F0DCF905F067FAC7F8CC00D7F8A6
:1053F000CC304E4AA2FB03235B09C7F8CC3005F042
:105400006DFAC7F8C800D7F8C830102B11D907F1CA
:105410000C03474A2021184609F0B5FD7B689A68BD
:1054200007F10C031146184609F0B9F91023C7F823
:10543000C83007F180031021184605F0C5FFC7F8F2
:10544000C8000023C7F8D430CFE2D7F8D4309B008F
:10545000D8333B4453F8583C002B00F0C182D7F8B6
:10546000D4309B00D8333B4453F8580C07F12C013F
:105470000523012205F04AFDD7F8D4309B00D8332C
:105480003B4453F8580C07F1740407F1780207F114
:105490007C0107F173030093234605F0E3FF00232B
:1054A00087F850307A6B07F150032021184609F035
:1054B00095FF00233B7307F1500207F10C00042312
:1054C0000093202320210AF04BF97B685A6807F1EA
:1054D0000C031146184609F062F9002387F8503092
:1054E00097F87330002B27D107F15003114A202180
:1054F000184609F048FD35E0FC370100003801008E
:105500000838010010380100183801002038010067
:1055100028380100343801004038010048380100C3
:10552000543801005C380100844101001F85EB51B3
:1055300064380100A038010007F15003584A2021C7
:10554000184609F020FD97F8732007F15003202139
:10555000184609F01EFE07F15003524A2021184652
:1055600009F036FD00233B7307F1500207F10C00F0
:1055700007230093202320210AF0F2F87B685A6861
:1055800007F10C031146184609F009F907F1500319
:10559000454A2021184609F0F6FCD7F8D4309B0084
:1055A000D8333B4453F8583C1A4607F150032021A6
:1055B000184609F0DDFE00233B7307F1500207F1A6
:1055C0000C000B230093202320210AF0C9F87B68EC
:1055D0005A6807F10C031146184609F0E0F8002359
:1055E0003B73D7F8D4309B00D8333B4453F8583C36
:1055F000184605F07FF9024607F10C000D230093D1
:10560000202320210AF0ACF87B685A6807F10C03CC
:105610001146184609F0C3F897F83830052B51D8D1
:1056200001A252F823F000BF41560000515600007D
:10563000715600006156000081560000915600002E
:1056400007F15003194A2021184609F09CFC41E05B
:1056500007F15003164A2021184609F094FC39E05E
:1056600007F15003134A2021184609F08CFC31E061
:1056700007F15003104A2021184609F084FC29E064
:1056800007F150030D4A2021184609F07CFC21E067
:1056900007F150030A4A2021184609F074FC19E06A
:1056A000A8380100B0380100B0260100B43801006C
:1056B000BC380100C4380100D0380100D8380100DE
:1056C000E038010007F15003CE4A2021184609F0C6
:1056D0005AFC00BF00233B7307F1500207F10C0096
:1056E00009230093202320210AF03AF87B685A68A6
:1056F00007F10C031146184609F051F8002387F80A
:10570000503007F1500328222021184609F093FC5D
:105710003A6C07F150032021184609F05FFE07F1AB
:1057200050032C222021184609F085FCFA6B07F162
:1057300050032021184609F051FE07F15003292299
:105740002021184609F077FC00233B7307F1500233
:1057500007F10C0008230093202320210AF000F811
:105760007B685A6807F10C031146184609F017F8D0
:1057700007F15003A44A2021184609F004FCFB6FEE
:105780001A4607F150032021184609F0F1FD0023C5
:105790003B7307F1500207F10C000B230093202309
:1057A000202109F0DDFF7B685A6807F10C031146E0
:1057B000184608F0F4FF07F15003934A20211846D9
:1057C00009F0E1FBBB6F1A4607F150032021184690
:1057D00009F0CEFD00233B7307F1500207F10C00E6
:1057E0000B2300932023202109F0BAFF7B685A681D
:1057F00007F10C031146184608F0D1FFFB6F1A465B
:10580000BB6FD31A9BB20833A7F8C630002387F8C2
:105810005030B7F8C62007F150000523009320232D
:10582000202109F0E8FC07F15003784A20211846AE
:1058300009F0CEFB00233B7307F1500207F10C0087
:10584000082300932023202109F08AFF7B685A68EF
:1058500007F10C031146184608F0A1FF07F15003A9
:10586000694A2021184609F08EFB7B6F1A4607F122
:1058700050032021184609F07BFD07F15003644ACC
:105880002021184609F0A4FBFB6F1A467B6FD31A40
:105890009BB204339AB207F15000052300932023F2
:1058A000202109F0A8FC07F150035A4A202118468C
:1058B00009F08EFB00233B7307F1500207F10C0047
:1058C000152300932023202109F04AFF7B685A68A2
:1058D00007F10C031146184608F061FF002387F812
:1058E0005030B7F84C309B009AB207F150000523B6
:1058F00000932023202109F07EFC07F15003434A46
:105900002021184609F064FB00233B7307F1500285
:1059100007F10C00082300932023202109F020FF29
:105920007B685A6807F10C031146184608F037FFE8
:1059300007F15003344A2021184609F024FB7A6C01
:1059400007F150032021184609F012FDD7F8CC309A
:10595000002B2BD07A6CD7F8CC30B2FBF3F3C7F81E
:10596000C030D7F8C030002B19D007F15003284AB7
:105970002021184609F02CFBD7F8C0309AB207F165
:105980005000032300932023202109F034FC07F169
:105990005003214A2021184609F01AFB06E007F1BE
:1059A00050031E4A2021184609F012FB00233B73C6
:1059B00007F1500207F10C0011230093202320214E
:1059C00009F0CEFE7B685A6807F10C0311461846B1
:1059D00008F0E5FE7B685B681946114808F0DFFEB9
:1059E000D7F8D4300133C7F8D430D7F8D420D7F85B
:1059F000C8309A42FFF429AD97F8D3301846DC3707
:105A0000BD4690BDE8380100B0260100F438010021
:105A1000F8380100FC3801000039010004390100A8
:105A20008441010080B586B000AF78607B685B6818
:105A30001A463349334809F0FBF87B685B681A461D
:105A40003149324809F0F4F87B685B681946304800
:105A500008F0A5FE7B685B681A462E492E4809F0BF
:105A6000E7F807F108034FF47A721021184601F0A5
:105A700039FB7B685A6807F108031146184608F09D
:105A80008EFE7B685B681946244808F088FE07F1A3
:105A9000080301221021184601F024FB7B685A6894
:105AA00007F108031146184608F079FE7B685B6829
:105AB00019461B4808F073FE7B685B681A46154957
:105AC000184809F0B5F804F04BFA024607F108034C
:105AD0001021184601F0A6FB7B685A6807F10803FD
:105AE0001146184608F05BFE7B685B6819460E4855
:105AF00008F055FE002318461837BD4680BD00BF8C
:105B00000C3901002C390100343901003C39010005
:105B100084410100A83B01004839010058390100C7
:105B200060390100683901007439010080B582B024
:105B300000AF78607B685B681A460B490B4809F038
:105B400065F87B685B681A4609490A4809F05EF8FF
:105B50007B685B681A460849084809F057F8002333
:105B600018460837BD4680BD702701002C3901005A
:105B70006424010088240100803901009439010067
:105B800080B584B000AFF860B9607A601F49F868EA
:105B90000CF0A9F80346002B06D01D49F8680CF05C
:105BA000A2F80346002B07D1BB6801221A7078685F
:105BB000FFF7BCFF034625E01649F8680CF093F8A0
:105BC0000346002B06D01449F8680CF08CF8034605
:105BD000002B07D1BB6801221A707868FFF722FFFB
:105BE00003460FE00D49F8680CF07DF80346002BE2
:105BF00007D1BB6801221A707868FFF703FB0346E0
:105C000000E0002318461037BD4680BDA8390100CA
:105C1000A0390100B8390100B0390100C0390100D4
:105C200080B584B000AF0346FB710A23FB60FB1D07
:105C300001221946002004F003F80346012B0AD183
:105C4000144B1B78002B1ED0124B1B78013BDAB291
:105C5000104B1A7017E00F4B1B780133DAB20D4B63
:105C60001A700C4B1B78632B03D90A4B64221A70F1
:105C70000CE0052004F09EFCFB68002B05DDFB68B2
:105C8000053BFB60D3E700BF00E000BF1037BD4617
:105C900080BD00BFEC13002080B400AF024B18465B
:105CA000BD465DF8047B7047D439010080B584B0EF
:105CB00000AFF860B9607A603249F8680CF013F808
:105CC0000346002B06D03049F8680CF00CF8034668
:105CD000002B3CD17B685B6819462C4808F05FFDBF
:105CE0007B685B6819462A4808F059FD7B685B6849
:105CF0001946264808F053FD7B685B68194625481D
:105D000008F04DFD7B685B681946204808F047FDA8
:105D10007B685B6819461E4808F041FD7B685B683C
:105D200019461A4808F03BFD7B685B681A461A4919
:105D30001A4808F06BFF7B685B681A4618491948D7
:105D400008F064FFBB6801221A70002316E01649B0
:105D5000F8680BF0C8FF0346002B06D01349F8681B
:105D60000BF0C1FF0346002B07D1BB6801221A705C
:105D7000786800F035F8034600E000231846103735
:105D8000BD4680BDA8390100E4390100844101000D
:105D9000F4390100343A0100403A0100603A010050
:105DA0006424010088240100B83901006C3A010024
:105DB00080B582B000AF78607B685B6819460648A2
:105DC00008F0EDFC7B685B681946044808F0E7FCC6
:105DD00000BF0837BD4680BD844101007C3A010008
:105DE00080B58AB000AF78607B685B681A462B4943
:105DF0002B4808F01DFF7B685B681A4629492A4832
:105E000008F016FF7B685B681946284808F0C7FC55
:105E10007B685B681946264808F0C1FC7B685B68B4
:105E20001946244808F0BBFC00233B7207F1080325
:105E300023222021184609F0FEF807F108031D4A25
:105E40002021184609F0C4F87B685A6807F1080356
:105E50001946194808F0ECFE7B685B681A4617493A
:105E6000174808F0E5FE07F1080330222021184604
:105E700001F0D8F907F10803124A2021184609F069
:105E8000A7F87B685A6807F1080319460E4808F01E
:105E9000CFFE002318462837BD4680BD843A010056
:105EA000603A0100A03A0100AC3A01005C390100FF
:105EB000B43A010084410100C03A0100CC3A01002B
:105EC000D43A0100E03A0100F83A010080B582B00E
:105ED00000AF786039603B689B681946124808F04B
:105EE0005EFC3B689B681946786808F058FC3B6884
:105EF0009B6819460D4808F052FC3B689B681946A0
:105F00000B4808F04CFC3B689B681946094808F0B0
:105F100046FC3B689B681946074808F040FC00BFF8
:105F20000837BD4680BD00BF003B01008441010031
:105F3000203B0100A83901002C3B010080B483B054
:105F400000AF7860044A7B681360002318460C3762
:105F5000BD465DF8047B7047D803002080B400AFD5
:105F6000034B1B681846BD465DF8047B704700BFB5
:105F7000D803002090B5A9B000AFF860B9607A608E
:105F8000FB70002387F899307A68BB689A4208D280
:105F9000D7F8B8309B681946854808F000FC022302
:105FA00001E1BB68C7F89C30F6E07A68D7F89C300E
:105FB000D31A5A1C97F8B0309A4204D397F8B030ED
:105FC00087F89A3009E07B68DAB2D7F89C30DBB208
:105FD000D31ADBB2013387F89A3097F89A3007F179
:105FE0007802D7F8B440D7F89C10F868A047034669
:105FF000002B08D0D7F8B8309B6819466D4808F0D8
:10600000CEFB1B23CFE097F89930002B08D0D7F8B0
:10601000B8309B681946684808F0C1FB1223C2E0FB
:1060200007F11003654A6521184608F0ACFFFB78BC
:1060300007F11000D7F89C20652109F0ECFB07F16F
:1060400010033A226521184608F0F5FFD7F8B8305A
:106050005A6807F110031146184608F0A0FB002308
:106060003B74002387F89B3022E097F89B30002B8D
:1060700006D107F1100320226521184608F0DBFF46
:1060800097F89B30A0333B4413F8282C07F11003FA
:106090006521184609F0D0F807F110032022652188
:1060A000184608F0C8FF97F89B30013387F89B30FB
:1060B00097F89B2097F89A309A42D6D30BE007F1D5
:1060C00010033F4A6521184608F082FF97F89B307D
:1060D000013387F89B3097F89B2097F8B0309A42AD
:1060E000EDD3D7F8B8305A6807F1100311461846B7
:1060F00008F055FBD7F8B8305B682020984700239C
:1061000087F89B3021E097F89B30A0333B4413F88D
:10611000283C87F8983097F898301F2B0BD997F9BF
:106120009830002B07DBD7F8B8305B6897F89820D9
:106130001046984704E0D7F8B8305B682E2098479F
:1061400097F89B30013387F89B3097F89B2097F89E
:106150009A309A42D7D30BE007F11003184A652111
:10616000184608F035FF97F89B30013387F89B30CD
:1061700097F89B2097F8B0309A42EDD3D7F8B83013
:106180005B6819460F4808F00AFB97F8B030D7F85B
:106190009C201344C7F89C30D7F89C207B689A4217
:1061A0007FF603AF00231846A437BD4690BD00BF5D
:1061B000543B0100943B0100AC3B0100B0260100C0
:1061C000D43B01008441010080B483B000AF03469A
:1061D000FB7197F90730002B0BDBFB7903F01F02F3
:1061E000074997F907305B09012000FA02F241F8EC
:1061F000232000BF0C37BD465DF8047B704700BF0D
:1062000000E100E080B483B000AF03463960FB7169
:1062100097F90730002B0ADB3B68DAB20C4997F993
:1062200007301201D2B20B4483F800230AE03B6826
:10623000DAB20849FB7903F00F03043B1201D2B232
:106240000B441A7600BF0C37BD465DF8047B7047DF
:1062500000E100E000ED00E080B582B000AF034651
:10626000FB71FB1D012219460348FEF7BBF800BF76
:106270000837BD4680BD00BF00A0024080B584B095
:1062800000AF78600A4B1B6807F10F010022184627
:106290000AF069FD0346012B03D1FA7B7B681A7073
:1062A00002E07B6800221A7000BF1037BD4680BD37
:1062B000DC03002080B500AF064B1B6818460BF0CE
:1062C00028F80346002B14BF01230023DBB2184635
:1062D00080BD00BFDC03002080B584B000AF002388
:1062E0003B601748FEF742F8B860BB6803F4201320
:1062F000002B14D00123FB730EE0114808F0EBFCD7
:106300000346FB710F4B18683A46F91D00230AF04B
:1063100004FCFB7B013BFB73FB7B002BEDD1B968DD
:106320000748FEF737F83B68002B01D003F0D6FF93
:10633000BFF34F8F00BF00BF1037BD4680BD00BF09
:1063400000A00240DC03002080B582B000AF78607E
:106350007B68062B58D07B68062B00F381807B6816
:10636000042B03D07B68052B22D079E03F4808F04E
:106370007FFC072203213E4808F0BAFC3C4BDB6857
:1063800023F0807323F00303394A43F00303D360FF
:1063900007220421364808F0ABFC354B1B6923F07B
:1063A000807323F00303324A43F00303136158E080
:1063B000304808F05DFC032210212F4808F098FCBB
:1063C0002D4B1B6C23F0807323F003032A4A43F008
:1063D0000303136403221121274808F089FC264B8C
:1063E0005B6C23F0807323F00303234A43F0030321
:1063F0005364224B03F580531B69204A23F00303A7
:1064000002F5805213612CE01D4808F031FC032294
:1064100000211C4808F06CFC1A4B1B6823F08073A9
:1064200023F00303174A43F00303136003220121FF
:10643000144808F05DFC134B5B6823F0807323F075
:106440000303104A43F0030353600C4B03F58053DE
:106450001B690A4A23F0330302F58052136100E0FE
:10646000FEE700BF0837BD4680BD00BF0B003810F7
:1064700000B004400A00381000A00440007004403E
:106480000D00381000D0044080B586B000AF08F091
:106490004CFC3B1D1846FDF7EFFE4FF4E1337B60EB
:1064A0000123FB740123BB740620FCF763FF024643
:1064B0003B1D19460B48FDF787FD78617B69002B72
:1064C00000D0FEE74FF400110648FDF71BFF052141
:1064D0001E20FFF797FE1E2008F0E4FB00BF1837D0
:1064E000BD4680BD00A0024080B500AF044B1B68D4
:1064F00018460AF026FF024B00221A6000BF80BD3A
:10650000DC03002080B500AF0022012130200AF01A
:1065100022F90346084A1360074B1B68002B00D181
:10652000FEE7054B1B680549184603F087FFFFF798
:10653000ABFF00BF80BD00BFDC030020E83B0100D3
:1065400080B582B000AF78607B68002B05D1074B27
:10655000074AA1210748F9F7ABFF5022064978689E
:106560000BF0AFFA00BF0837BD4680BD34360100DE
:10657000D83C0100C83C0100783C010080B58AB0DD
:1065800000AF78607B68002B05D13B4B3B4ABE21B6
:106590003B48F9F78DFF2C2003F0C6FB38623B6ABD
:1065A000002B05D1374B354AC4213548F9F780FF18
:1065B0003B6A002B5AD02C220021386A0BF08FFA4C
:1065C0003149386A08F0B8FB7B685A683B6A9A60C0
:1065D0003B6A00221A607B681A783B6A1A717B68F2
:1065E0005A783B6A5A713B6A00229A717B681A7A20
:1065F0003B6A1A737B68DA683B6A9A613B6A9B69FB
:10660000002B02D13B6A214A9A617B681B7A83F096
:106610000103DBB2002B29D007F10C031846FEF76B
:10662000F3F900237B621EE000233B737B6A013396
:106630001B017A68D11807F10C03043310221846A5
:106640000BF03FFA00237B7307F10C031846FEF7AB
:10665000F9F901463A6A7B6A06339B001344596094
:106660007B6A01337B627B6A032BDDDD3B6A184664
:106670002837BD4680BD00BF34360100F43C010020
:10668000C83C01005C3601000C3C010065ED0000D7
:1066900080B584B000AF78607B68FB60FB689B6965
:1066A000044978689847FB6800229A7100BF103748
:1066B000BD4680BD143C010080B586B000AF786057
:1066C0000B46FB707B68FB60FB681B79022B1BD1C0
:1066D000FB78002B06D0FB685B7983F00103DBB20B
:1066E000002B09D1FB7883F00103DBB2002B06D02D
:1066F000FB685B79002B02D0264B7B6101E0264BC7
:106700007B6108233B611AE0FB78002B06D0FB6815
:106710005B7983F00103DBB2002B09D1FB7883F0B6
:106720000103DBB2002B06D0FB685B79002B02D0A3
:106730001A4B7B6101E01A4B7B6104233B61FB68D0
:106740009B69FA689279920079690A441146F8685F
:106750009847FB689B790133DAB2FB689A71FB6852
:106760009B791A463B69934210D8FB6800229A71C4
:10677000FB78002B05D0FB681B685A1CFB681A606D
:1067800004E0FB681B685A1EFB681A6000BF1837DC
:10679000BD4680BD183C0100383C0100583C01005A
:1067A000683C010080B483B000AF0346FB7197F9E9
:1067B0000730002B0BDBFB7903F01F02074997F929
:1067C00007305B09012000FA02F241F8232000BFE4
:1067D0000C37BD465DF8047B704700BF00E100E068
:1067E00080B483B000AF03463960FB7197F907307E
:1067F000002B0ADB3B68DAB20C4997F9073012012B
:10680000D2B20B4483F800230AE03B68DAB20849AD
:10681000FB7903F00F03043B1201D2B20B441A764A
:1068200000BF0C37BD465DF8047B704700E100E017
:1068300000ED00E080B500AF034B1B680021184657
:1068400009F02FFF00BF80BD1404002080B582B086
:1068500000AF084B1B68F91D002218460AF083FAA6
:106860000346012B01D00023FB71FB791846083742
:10687000BD4680BD1404002080B582B000AF7860B2
:1068800039603A687968034807F016FD00BF083799
:10689000BD4680BD00A0064080B582B000AF034673
:1068A000FB71104B1B685A1C0E490A600E49FA799D
:1068B000CA54FB790A2B03D00A4B1B682F2B0DD12E
:1068C000084B1B68084A0021D154074808F04BFBCD
:1068D000054B00221A70034B00221A6000BF0837D4
:1068E000BD4680BD180400201C04002080B584B083
:1068F00000AF78600A4B1B6807F10F0100221846B1
:106900000AF031FA0346012B03D1FA7B7B681A7037
:1069100002E07B6800221A7000BF1037BD4680BDC0
:106920001004002080B500AF064B1B6818460AF023
:10693000F0FC0346002B14BF01230023DBB21846F2
:1069400080BD00BF1004002080B586B000AF0023DA
:10695000BB6000237B60334807F04AFC38613B6929
:1069600003F08063002B01D00023FB753B6903F02B
:106970002803002B3DD02B4B9B7DFB7536E029482F
:1069800008F0E4FA0346FB73FB7B002B2BD0264B6D
:106990001B780A2B05D1FB7B402B02D1234B012214
:1069A0001A70224B1B78002B08D0214B186807F176
:1069B000080207F10F0100230AF0AFF8FA7B1A4B27
:1069C0001A701A4B1B78002B05D0FB7B0A2B02D1C7
:1069D000164B00221A70174B18683A1D07F10F0169
:1069E00000230AF09AF8FB7D013BFB75FB7D002B31
:1069F000C5D13B6943F0806343F008033B613969CB
:106A0000084807F019FCBB68002B02D17B68002BFB
:106A100001D003F063FCBFF34F8F00BF00BF1837F6
:106A2000BD4680BD00A0064088000020ED13002078
:106A3000140400201004002080B584B000AF3B4651
:106A40001846FDF795FE4FF461433B600123FB724E
:106A50000123BB720123FB7100233B720620FCF76C
:106A600089FC02463B4619461848FDF727FDF860A9
:106A7000FB68002B07D0164B4FF48D72154905208B
:106A8000FEF7CCFAFEE7114B5B7BDBB20F4A43F01B
:106A90000403DBB253730D4B5B7BDBB20B4A43F059
:106AA0000203DBB253730121084807F02DFC0A49A9
:106AB0000648FDF797FE05211F20FFF791FE1F20D6
:106AC00008F02BFA00BF1037BD4680BD00A006407D
:106AD0001C3D0100383D01000020080480B582B053
:106AE00000AF786039607B6803F08003002B06D02C
:106AF0003B685B681A466949694808F099F87B6801
:106B000003F04003002B06D03B685B681A466549DA
:106B1000634808F08DF87B6803F02003002B06D053
:106B20003B685B681A4660495D4808F081F87B68FD
:106B300003F01003002B06D03B685B681A465B49E4
:106B4000574808F075F87B6803F00803002B06D05F
:106B50003B685B681A465649514808F069F87B68FB
:106B600003F00403002B06D03B685B681A465149CA
:106B70004B4808F05DF87B6803F00203002B06D059
:106B80003B685B681A464C49454808F051F87B68F9
:106B900003F00103002B06D03B685B681A464749A7
:106BA0003F4808F045F87B6803F40043002B06D00B
:106BB0003B685B681A464249394808F039F87B68F7
:106BC00003F48043002B06D03B685B681A463D49BE
:106BD000334808F02DF87B6803F48073002B06D04F
:106BE0003B685B681A4638492D4808F021F87B68F5
:106BF00003F40003002B06D03B685B681A46334958
:106C0000274808F015F87B6803F48003002B06D0B2
:106C10003B685B681A462E49214808F009F87B68F2
:106C2000002B06DA3B685B681A462A491C4807F0C5
:106C3000FFFF7B6803F08043002B06D03B685B6856
:106C40001A462549164807F0F3FF7B6803F00073E6
:106C5000002B06D03B685B681A462049104807F0B5
:106C6000E7FF7B6803F08063002B06D03B685B681E
:106C70001A461B490A4807F0DBFF7B6803F0806374
:106C8000002B06D03B685B681A461549044807F09C
:106C9000CFFF00BF0837BD4680BD00BF483D0100A3
:106CA000A83B0100643D0100883D0100A43D0100B6
:106CB000BC3D0100D43D0100EC3D0100083E010057
:106CC000203E0100383E0100543E01006C3E0100B0
:106CD000903E0100B43E0100CC3E0100E43E0100C4
:106CE000003F010080B59CB000AF78607B685B68B6
:106CF0001A463C493C4807F09BFF7B685B681A4694
:106D00003A493B4807F094FF3A4807F071FAF866B1
:106D100007F10C03384A6021184608F034F907F1EE
:106D20000C03FA6E6021184608F022FB07F10C03F1
:106D3000324A6021184608F04BF97B685A6807F11F
:106D40000C0319462E4807F073FF7968F86EFFF7B9
:106D5000C5FE07F10C034FF461426021184600F0B4
:106D600061FA07F10C03254A6021184608F030F952
:106D70007B685A6807F10C031946224807F058FF50
:106D800007F10C03204A6021184608F0FCF807F1CF
:106D90000C034FF440626021184608F01FFB07F116
:106DA0000C031A4A6021184608F012F907F10C0387
:106DB00060226021184608F011FB07F10C030F4A0E
:106DC0006021184608F004F97B685A6807F10C0343
:106DD00019460F4807F02CFF002318467037BD46B0
:106DE00080BD00BF1C3F0100343F0100403F010057
:106DF000483F010000A00640B02601008441010088
:106E000040240100543F01005C3F0100643F010049
:106E1000743F010080B582B000AF78607B685B682A
:106E20001A460B490B4807F0F1FE7B685B681A466F
:106E300009490A4807F0EAFE7B685B681A46084978
:106E4000084807F0E3FE002318460837BD4680BD1A
:106E500060250100343F0100642401008824010002
:106E6000803F0100983F010080B588B000AFF86016
:106E7000B9607A603349F8680AF035FF0346002BA1
:106E800006D03149F8680AF02EFF0346002B07D1DF
:106E9000BB6801221A707868FFF7BCFF03464CE01C
:106EA0002A49F8680AF01FFF0346002B06D028493C
:106EB000F8680AF018FF0346002B07D1BB680122CF
:106EC0001A707868FFF70EFF034636E01122214959
:106ED000F8680AF022FF0346002B2DD1BB6801227F
:106EE0001A70FB6811337B6107F1180207F1140374
:106EF0001146184608F08AFA0346002B1AD1BB69DE
:106F00001946154807F098F9F8617B685B681946DF
:106F1000124807F044FCFA697B685B681946104622
:106F200007F056FC7B685B6819460D4807F037FC94
:106F3000002302E01B2300E0002318462037BD4653
:106F400080BD00BFA8390100A83F0100B839010089
:106F5000B83F0100CC3F010000A00640E03F010027
:106F60008441010080B500AFFFF766FD00220121DA
:106F70004FF4406009F0EFFB0346184A1360174BCB
:106F80001B68002B07D1164B4FF4087215490520DA
:106F9000FEF744F8FEE7114B1B681349184603F04F
:106FA0004DFA00220121602009F0D5FB03460F4A6B
:106FB00013600E4B1B68002B07D10D4B40F22722AC
:106FC00008490520FEF72AF8FEE7084B1B68094927
:106FD000184603F033FA00BF80BD00BF1004002044
:106FE000EC3F0100383D01000C400100140400207A
:106FF000204001004840010080B489B000AFF86033
:10700000B9601346FB80FB68BB610023FB77BB685C
:10701000013BBB60FB88002B2CD1BB68002B29D027
:10702000FB7F5A1CFA771A46BB69134430221A7048
:10703000BB68013BBB601DE0FA88294BA3FB021330
:10704000D9080B469B000B445B00D31A9BB2DAB203
:10705000FB7F591CF9771946BB690B443032D2B219
:107060001A70BB68013BBB60FB881D4AA2FB03236F
:10707000DB08FB80FB88002B02D0BB68002BDBD138
:107080000023BB771AE0BB7FBA6913441B78FB75FA
:10709000FA7FBB7FD31A013BBA691A44BB7FB96937
:1070A0000B4412781A70FA7FBB7FD31A013BBA697E
:1070B0001344FA7D1A70BB7F0133BB77FB7F5B08FB
:1070C000DBB2BA7F9A42DED3FB7FBA691344002257
:1070D0001A7000BF2437BD465DF8047B704700BFBF
:1070E000CDCCCCCC80B588B000AFF860B960134689
:1070F000FB80FB68BB610023FB77FB88DB0BDBB20B
:10710000FB75B7F9063013F5004F05D1434AB9684E
:10711000F86807F038FF7EE0BB68013BBB60FB7D91
:10712000002B03D0FB885B429BB2FB80B7F9063093
:10713000002B32D1BB68002B2FD0FB7F5A1CFA7773
:107140001A46BB69134430221A70BB68013BBB600E
:1071500023E0B7F90620324B83FB02139910D317B3
:10716000C91A0B469B000B445B00D31A1BB2DAB260
:10717000FB7F591CF9771946BB690B443032D2B2F8
:107180001A70BB68013BBB60B7F90630244A82FB2A
:1071900003129210DB17D31AFB80B7F90630002BCD
:1071A00002DDBB68002BD4D1FB7D002B0AD0BB686D
:1071B000002B07D0FB7F5A1CFA771A46BB69134491
:1071C0002D221A700023BB771AE0BB7FBA691344E3
:1071D0001B78BB75FA7FBB7FD31A013BBA691A448F
:1071E000BB7FB9690B4412781A70FA7FBB7FD31A40
:1071F000013BBA691344BA7D1A70BB7F0133BB7778
:10720000FB7F5B08DBB2BA7F9A42DED3FB7FBA69B1
:10721000134400221A702037BD4680BD6040010033
:107220006766666680B489B000AFF860B9607A605E
:10723000FB68BB610023FB77BB68013BBB607B68DD
:10724000002B2BD1BB68002B28D0FB7F5A1CFA7770
:107250001A46BB69134430221A70BB68013BBB60FD
:107260001CE07968284BA3FB0123DA0813469B0036
:1072700013445B00CA1AD2B2FB7F591CF977194636
:10728000BB690B443032D2B21A70BB68013BBB60A1
:107290007B681D4AA2FB0323DB087B607B68002B15
:1072A00002D0BB68002BDCD10023BB771AE0BB7F88
:1072B000BA6913441B78FB75FA7FBB7FD31A013B75
:1072C000BA691A44BB7FB9690B4412781A70FA7F05
:1072D000BB7FD31A013BBA691344FA7D1A70BB7F96
:1072E0000133BB77FB7F5B08DBB2BA7F9A42DED308
:1072F000FB7FBA69134400221A7000BF2437BD46D1
:107300005DF8047B704700BFCDCCCCCC80B588B095
:1073100000AFF860B9607A603B600023FB61002336
:10732000BB610023FB750023BB75FB68002B05D0F8
:10733000BB68002B04D07B68002B01D11B2380E0AD
:10734000FB681B78222B07D1FB680133FB60BB690C
:107350000133BB610123FB75FB6A002B01D13B4B61
:10736000FB62FB7D002B14D0FB681B78222B09D11C
:10737000FB680133FB60BB690133BB61FB681B78B1
:10738000222B47D1FB681B78002B27D10123BB752B
:1073900041E0FB681B78202B3DD0FB681B78092B54
:1073A00039D0FB681B780A2B35D0FB681B780B2B78
:1073B00031D0FB681B780C2B2DD0FB681B780D2B74
:1073C00029D0FB681B78002B25D0FB681B78194659
:1073D000F86A0AF07BFC0346002B1CD1BB68002B2B
:1073E00011D0FB6901337A689A4207D9FB681A7891
:1073F000BB681A70BB680133BB6004E0BB68002245
:107400001A700023BB60FB690133FB61FB68013329
:10741000FB60A6E700BFBB68002B02D0BB68002260
:107420001A703B68002B04D0FA69BB691A443B68A8
:107430001A60BB6A002B03D0FB695A1CBB6A1A6036
:10744000BB7D18462037BD4680BD00BFA83B01006C
:1074500080B485B000AF78607B68FB60084B1B6828
:10746000FA681344FB6000BF054B1B68FA689A4238
:10747000FAD800BF00BF1437BD465DF8047B7047E3
:10748000041000E080B584B000AF78600A4B1B6840
:107490000A4AA2FB03239B09FB6005E0F868FFF79B
:1074A000D7FF7B68013B7B607B68002BF6D100BF78
:1074B00000BF1037BD4680BD18000020D34D6210BC
:1074C00080B400AF094B1B68084A43F08073136017
:1074D000074B00221A60074B1B68064A43F0010362
:1074E000136000BFBD465DF8047B7047FCED00E013
:1074F000041000E0001000E080B400AF054B1B68F2
:10750000044A23F00103136000BFBD465DF8047B0D
:10751000704700BF001000E080B485B000AF786015
:1075200053E07B6893F85730102B1ED0102B28DCCB
:10753000022B02D0082B0CD023E07B681B68DBB247
:1075400003F00103FB737B681B685A087B681A60B1
:107550002DE07B681B68DBB203F00703FB737B68DD
:107560001B68DA087B681A6021E07B681B68DBB265
:1075700003F00F03FB737B681B681A097B681A60B2
:1075800015E07B6819681A4BA3FB0123DA08134640
:107590009B0013445B00CA1A1346FB737B681B688D
:1075A000134AA2FB0323DA087B681A6000BFFA7B48
:1075B0007B689B68581E796888600E498A5C1A70DF
:1075C0007B68DB695A1C7B68DA617B681B6A591E21
:1075D0007A681162002BA4DC7B681B68002BA0D1A9
:1075E00000BF00BF1437BD465DF8047B704700BF85
:1075F000CDCCCCCC804001002DE9B043A0B002AF8F
:10760000F860B9607A603B600023BB63002387F8B1
:107610006930CEE37B685A1C7A601B7887F8733038
:1076200097F873301F2B03D997F873307A2B02D950
:1076300000237B6707E097F87330203BC44AD35C94
:1076400003F00F037B677B6FDB0097F8692013441F
:10765000BF4AD35C1B09DBB287F8693097F8693001
:10766000013B062B10D801A252F823F09D760000B2
:107670004D770000B9760000B37D0000E57600008C
:1076800019770000D577000097F87320FB68114642
:10769000B8689847BB6B0133BB638AE300233B6345
:1076A0003B6B7B637B6B3B643B6CFB62FB6AFB630A
:1076B000202387F868307CE397F873302A2B05D1B4
:1076C0003B681A1D3A601B687B6372E37A6B134652
:1076D0009B0013445B001A4697F87330303B134409
:1076E0007B6366E3FB6B43F00403FB6397F8733043
:1076F0002A2B05D13B681A1D3A601B683B6358E38F
:107700003A6B13469B0013445B001A4697F873309C
:10771000303B13443B634CE397F873306C2B0AD037
:107720007A2B11D1FB6B23F00303FB63FB6B43F05C
:107730000203FB6309E0FB6B23F00303FB63FB6BBA
:1077400043F00103FB6300E000BF32E397F87330BE
:10775000203B102B3CD801A252F823F0B377000055
:10776000D1770000D1770000BD770000D17700000D
:10777000D1770000D1770000D1770000D1770000E9
:10778000D1770000D1770000C7770000D1770000E3
:10779000A1770000D1770000D1770000AB7700001F
:1077A000FB6B43F00803FB6313E0302387F868307A
:1077B0000FE0FB6B43F01003FB630AE0FB6B43F04D
:1077C0002003FB6305E0FB6B43F04003FB6300E039
:1077D00000BFEEE297F87330423B362B70D801A21F
:1077E00052F823F0857B0000D3790000C1780000B7
:1077F000C1780000C1780000C1780000C1780000A5
:10780000C1780000C1780000C1780000C178000094
:10781000C1780000C1780000C1780000C77800007E
:10782000C1780000C1780000A9790000C17800008B
:10783000C1780000C1780000C178000055790000CF
:10784000C1780000C1780000C1780000C178000054
:10785000C1780000C1780000C1780000C178000044
:10786000C1780000FF780000DB7900008979000012
:10787000C1780000F7790000C1780000C1780000ED
:1078800089790000C1780000C1780000C17800004B
:10789000C1780000C17800002B790000CF7800008B
:1078A000C1780000C1780000B1790000C178000003
:1078B00099790000C1780000C17800005D7900006E
:1078C0000023FB6275E1FB6B43F08003FB63FB6B02
:1078D00023F00303FB63FB6B43F4007343F00203E9
:1078E000FB63102387F8673008233B632D2387F859
:1078F00044303E2387F8453002233B6459E1FB6B5B
:1079000043F40073FB63022387F86730FB6B03F0DB
:107910002003002B00F04881302387F84430622395
:1079200087F8453002233B643EE1FB6B43F4007370
:10793000FB63082387F86730FB6B03F02003002B01
:1079400000F03481302387F8443001233B642DE17B
:1079500094400100FB6B43F08003FB63FB6B43F43B
:107960000073FB63102387F86730FB6B03F0200381
:10797000002B00F01D81302387F84430782387F8EE
:10798000453002233B6413E1FB6B43F44073FB631C
:107990000A2387F867300CE1FB6B43F40073FB6349
:1079A0000A2387F8673004E1FB6B43F08003FB6335
:1079B0003B681A1D3A601B68BB61BB69002B01D193
:1079C0009F4BBB61BB69184607F06AFF0346FB6229
:1079D000EFE0FB6B43F08003FB6307F110033633EA
:1079E000BB613B681A1D3A601B68DBB287F8463002
:1079F0000123FB62DDE0FB6B03F00403002B01D1EC
:107A000006233B633B68073323F0070303F10802B7
:107A10003A60D3E90023C7E908234FF00002894BFD
:107A2000C7E9042300237B670DE0D7E904014FF089
:107A30000002854B04F00EFB02460B46C7E9042307
:107A40007B6F01337B673B6B7A6F9A42EDDBD7E943
:107A500008014FF000024FF0000304F043FC03461E
:107A6000002B2DD0FB6B43F48063FB63D7E9080147
:107A7000D7E9042304F00CF802460B46C7E90823B3
:107A8000D7E908231046194604F054FC0346BB62AC
:107A9000D7E90889BB6A184604F048F902460B4644
:107AA0004046494603F0F4FF02460B46C7E9082367
:107AB000D7E90823144683F00045C7E9084521E0CB
:107AC000D7E90801D7E9042303F0E4FF02460B4697
:107AD000C7E90823D7E908231046194604F02AFC11
:107AE0000346BB62D7E90889BB6A184604F00EF961
:107AF00002460B464046494603F0CAFF02460B4683
:107B0000C7E9082300237B670DE0D7E908014FF0A0
:107B100000024D4B04F074F902460B46C7E90823F6
:107B20007B6F01337B673B6B7A6F9A42EDDBD7E962
:107B300008231046194604F025FC03463B6107F173
:107B4000100336332033BB610A2387F867303B6B61
:107B5000002B0CD007F110031846FFF7DDFCBB69C2
:107B60005A1EBA612E221A70FB6A0133FB62FB6B4C
:107B700043F4D85343F00103FB6300233B63BB6A28
:107B80003B6116E03B681A1D3A601B68002B02D06F
:107B90002E4BBB6101E02E4BBB61BB69184607F061
:107BA0007FFE0346FB6204E000BF02E000BF00E08E
:107BB00000BFFB6B03F40073002B00F0AB803B6B4A
:107BC000002B01D101233B63FB6B03F40063002B0B
:107BD00033D1FB6B03F00303022B06D0022B39D801
:107BE000002B19D0012B06D034E03B681A1D3A60F7
:107BF0001B683B612FE0FB6B03F48073002B05D007
:107C00003B681A1D3A601B683B6124E03B681A1D03
:107C10003A601B683B611EE0FB6B03F48073002B32
:107C200005D03B681A1D3A601B683B6113E03B6856
:107C30001A1D3A601B683B610DE000BF0BE000BFFE
:107C4000684001000000E03F000024407040010057
:107C50007840010000BFFB6B03F02003002B04D031
:107C60003B69002B01D100233B64FB6B03F4807361
:107C7000002B18D03B69002B06DA3B695B423B6165
:107C8000FB6B43F48063FB63FB6B03F48063002BAB
:107C900009D1FB6B03F01003002B04D0202387F8DD
:107CA000443001233B64FB6B03F48053002B04D16D
:107CB00007F1100336332033BB6107F11003184678
:107CC000FFF72AFCBB690133BB61FB6B03F48863DC
:107CD000002B28D0FB6B03F48063002B01D02D23F5
:107CE00000E02B2387F8733097F86830302B06D1EB
:107CF00001233B6497F8733087F8443013E0BB6985
:107D0000013BBB61BB6997F873201A70FB6A0133B2
:107D1000FB6208E07B6B002B05D0FA6A7B6B9A4212
:107D200001DD7B6BFB627A6BF96A3B6C0B44D31A07
:107D30007B63396CFB6B03F0800307F11002343274
:107D400000930B46B968F86807F0C1FD0246BB6BAB
:107D50001344BB63FB6B03F00803002B0AD197F8B5
:107D600068207B6BB968F86807F0E2FD0246BB6BE0
:107D70001344BB63BA69F96AFB6B03F08003009399
:107D80000B46B968F86807F0A2FD0246BB6B1344C6
:107D9000BB63FB6B03F00803002B0AD097F8682045
:107DA0007B6BB968F86807F0C3FD0246BB6B1344F0
:107DB000BB637B681B78002B7FF42CACBB6B184635
:107DC0007837BD46BDE8B08380B483B000AF78603B
:107DD00039607B68054A1360044A3B68536000BF02
:107DE0000C37BD465DF8047B704700BF4C04002093
:107DF00080B586B000AFF860B9607A600023FB758B
:107E00007968F86800F032F80346002B01D01B2394
:107E100023E0144806F0A4F938613B69002B01D037
:107E20001B231AE00120FFF72DFBF9687B68BA6875
:107E30000D4805F0B0FF38613B69002B02D01B23D1
:107E4000FB7500E000BF074806F09FF938613B6909
:107E5000002B01D01B23FB75FB7D18461837BD4650
:107E600080BD00BF00E007405404002080B586B00C
:107E700000AF786039600023FB600023FB75396830
:107E8000786807F07EFD0346002B01D0002343E015
:107E9000234806F065F938613B69002B01D01B23AC
:107EA0003AE00120FFF7EEFA07F10C031A46002131
:107EB0001C48FBF7EBFE38613B69002B01D01B230C
:107EC0002AE0FB68B3F5006F01D01B2324E079683A
:107ED000154B3A68134805F02EFF38613B69002BBB
:107EE00002D01B23FB750DE0796801233A680D4829
:107EF00005F081FF38613B69002B02D01B23FB7525
:107F000000E000BF064806F040F938613B69002BED
:107F100001D01B23FB75FB7D18461837BD4680BD7D
:107F200000E00740540400206B66656B80B58EB09E
:107F300000AF78607B685B681A462A492A4806F0D9
:107F400077FE07F10803294A3021184607F01BF88D
:107F500007F108034FF400623021184607F09BF93F
:107F600007F10803224A3021184607F031F87B68F0
:107F70005A6807F1080319461E4806F059FE07F132
:107F800008031D4A3021184606F0FDFF1B4B1A68F6
:107F900007F108033021184607F0EAF907F1080352
:107FA000174A3021184607F013F8144B5A6807F1A6
:107FB00008033021184607F0DBF907F108030C4AE3
:107FC0003021184607F004F87B685A6807F1080367
:107FD00019460C4806F02CFE002318463837BD46DB
:107FE00080BD00BFF04001000441010010410100CC
:107FF0008441010018410100204101004C0400208F
:10800000284101003441010080B58CB004AFF86014
:10801000B9607A607249F86809F065FE0346002B82
:1080200006D07049F86809F05EFE0346002B20D1A7
:108030007B685B681A466C496C4806F0E7FD7B6814
:108040005B681A466A496B4806F0E0FD7B685B682E
:108050001A466949694806F0D9FD7B685B681A468B
:108060006749684806F0D2FDBB6801221A700023F8
:10807000B1E06549F86809F036FE0346002B06D0EA
:108080006249F86809F02FFE0346002B07D1BB6850
:1080900001221A707868FFF749FF03469BE00E2221
:1080A0005B49F86809F039FE0346002B50D1BB68E4
:1080B00001221A70FB680E33FB6107F1180207F109
:1080C0001C031146184607F0A1F90346002B37D1CF
:1080D00007F1140207F11C031146184607F096F940
:1080E0000346002B24D17B69002B21DDBB691A4696
:1080F0007B691946104607F038FC0346002B0FD069
:10810000B969BB697A6913445A1E7B680293414B73
:1081100001931023009304230020FDF72BFF59E067
:108120007B689B6819463C4806F039FB1B2352E0EC
:108130007B689B681946394806F031FB1B234AE0EF
:108140007B689B681946364806F029FB1B2342E0F2
:108150000F223449F86809F0E0FD0346002B39D1BD
:10816000BB6801221A70FB680F33FB6107F118022C
:1081700007F11C031146184607F048F90346002B87
:1081800028D1BB69C3F30A03002B07D07B689B6827
:108190001946254806F003FB1B231CE007F11402D7
:1081A00007F11C031146184607F030F90346002B6F
:1081B00008D1BB691A467B6919461046FFF756FE7F
:1081C000034608E07B689B681946184806F0E7FA02
:1081D0001B2300E0002318462037BD4680BD00BFAA
:1081E000A83901004441010054410100044101004B
:1081F00064240100882401007441010088410100C9
:10820000A0410100BC410100B8390100D441010086
:10821000E4410100DFF90000F441010010420100D7
:108220002842010044420100544201008042010002
:1082300080B582B000AF642200210B4809F04FFCEA
:10824000094805F023FD78607B68002B07D0074BB9
:108250004FF4117206490520FCF7E0FEFEE700BF6F
:108260000837BD4680BD00BF540400209C42010079
:10827000B042010080B586B000AF78607B685B6873
:108280001A462649264806F0D3FC07F10803402287
:1082900010211846FEF7C6FF07F10803214A1021F6
:1082A000184606F095FE7B685A6807F108031946E0
:1082B0001D4806F0BDFC07F108031C4A10211846B2
:1082C00006F061FE7B685A6807F1080319461848F2
:1082D00006F0AEFC07F10803164A1021184606F016
:1082E00052FE7B685A6807F108031946124806F0E7
:1082F0009FFC07F10803114A1021184606F043FEBF
:1083000000BF7B685A6807F1080319460C4806F05D
:108310008FFC002318461837BD4680BDBC420100C3
:10832000CC42010074390100D8420100E44201004E
:10833000F4420100FC4201000C430100144301001F
:108340001C43010080B5C8B002AF07F58C73A3F5DC
:108350008673186007F58C73A3F58873196007F5A9
:108360008C73A3F58A731A6007F58C73A3F5867373
:10837000AD49186809F0B7FC0346002B0AD007F591
:108380008C73A3F58673A949186809F0ACFC034601
:10839000002B4AD107F58C73A3F58A731B685B68C1
:1083A0001A46A349A34806F031FC07F58C73A3F5E0
:1083B0008A731B685B681A469F49A04806F026FC32
:1083C00007F58C73A3F58A731B685B681A469C4992
:1083D0009C4806F01BFC07F58C73A3F58A731B6899
:1083E0005B681A469849994806F010FC07F58C73AB
:1083F000A3F58A731B685B681A469549954806F091
:1084000005FC07F58C73A3F58A731B685B681A4635
:108410009149924806F0FAFB07F58C73A3F588732F
:108420001B6801221A7000231DE307F58C73A3F566
:1084300086738B49186809F056FC0346002B0AD056
:1084400007F58C73A3F586738649186809F04BFC11
:108450000346002B0FD107F58C73A3F588731B68B7
:1084600001221A7007F58C73A3F58A731868FFF759
:1084700001FF0346F7E207F58C73A3F586730F221D
:108480007949186809F049FC0346002B40F0F48054
:1084900007F58C73A3F588731B6801221A7007F522
:1084A0008C73A3F586731B680F33C7F81431D7F8A4
:1084B000140107F1100307F11401002201920022B8
:1084C00000924022FEF722FF0346002B06D107F55B
:1084D0008C73A3F584731B68002B01D11B23C2E2AC
:1084E000D7F8142107F58C73A3F584731B68134424
:1084F000C7F8143107F58A73184607F0BBF9D7F8A7
:10850000140107F1100307F1E40100220192002297
:1085100000923022FEF7FAFE0346002B06D107F543
:108520008C73A3F584731B68002B01D11B239AE283
:10853000D7F8142107F58C73A3F584731B681344D3
:10854000C7F8143107F58A73184607F093F9D7F87E
:10855000140107F1100307F1B40100220192002277
:1085600000923022FEF7D2FE0346002B06D107F51B
:108570008C73A3F584731B68002B01D11B2372E25B
:10858000D7F8142107F58C73A3F584731B68134483
:10859000C7F81431D7F814311B78002B01D01B23F6
:1085A00061E207F1540207F1B40107F1E40007F1B9
:1085B000140301936023009313462C4A00F03AFD04
:1085C0000346002B01D11B234DE207F58C73A3F565
:1085D0008A731B685A6807F1B4031146184606F0FF
:1085E000DEF807F58C73A3F58A731B685B68194680
:1085F0001F4806F0D4F807F58C73A3F58A731B683F
:108600005A6807F154031146184606F0C8F807F5F2
:108610008C73A3F58A731B685B681946154806F0CE
:10862000BEF800231FE200BFA83901002443010067
:1086300034430100CC42010064240100882401007D
:10864000544301007C43010090430100C0430100FA
:10865000D8430100FC4301001444010034440100EC
:10866000B8390100484401005C440100A83B010006
:108670006C4401008441010007F58C73A3F58673F7
:108680001022B849186809F048FB0346002B40F057
:10869000C28007F58C73A3F588731B6801221A70DA
:1086A00007F58C73A3F586731B681033C7F8143174
:1086B000D7F8140107F1100307F114010022019209
:1086C000002200924022FEF721FE0346002B06D135
:1086D00007F58C73A3F584731B68002B01D11B2352
:1086E000C1E1D7F8142107F58C73A3F584731B68D7
:1086F0001344C7F8143107F58A73184607F0BAF81F
:10870000D7F8140107F1100307F1E40100220192E8
:10871000002200923022FEF7F9FD0346002B06D11D
:1087200007F58C73A3F584731B68002B01D11B2301
:1087300099E1D7F8142107F58C73A3F584731B68AE
:108740001344C7F8143107F58A73184607F092F8F6
:10875000D7F8140107F1100307F1B40100220192C8
:10876000002200923022FEF7D1FD0346002B06D1F5
:1087700007F58C73A3F584731B68002B01D11B23B1
:1087800071E1D7F8142107F58C73A3F584731B6886
:108790001344C7F8143107F58A73184607F06AF8CE
:1087A000D7F8140107F1100307F1540100220192D8
:1087B000002200926022FEF7A9FD0346002B06D19D
:1087C00007F58C73A3F584731B68002B01D11B2361
:1087D00049E1D7F8142107F58C73A3F584731B685E
:1087E0001344C7F81431D7F814311B78002B01D08B
:1087F0001B2338E107F1140307F1540207F1B40118
:1088000007F1E40000F08AFD0346002B01D11B2391
:1088100029E1002327E107F58C73A3F58673112264
:108820005149186809F079FA0346002B40F09E8000
:1088300007F58C73A3F588731B6801221A7007F57E
:108840008C73A3F586731B681133C7F81431D7F8FE
:10885000140107F1100307F1140100220192002214
:1088600000924022FEF752FD0346002B06D107F589
:108870008C73A3F584731B68002B01D11B23F2E0DA
:10888000D7F8142107F58C73A3F584731B68134480
:10889000C7F8143107F58A73184606F0EBFFD7F8CE
:1088A000140107F1100307F1E401002201920022F4
:1088B00000923022FEF72AFD0346002B06D107F571
:1088C0008C73A3F584731B68002B01D11B23CAE0B2
:1088D000D7F8142107F58C73A3F584731B68134430
:1088E000C7F8143107F58A73184606F0C3FFD7F8A6
:1088F000140107F1100307F1B401002201920022D4
:1089000000923022FEF702FD0346002B06D107F548
:108910008C73A3F584731B68002B01D11B23A2E089
:10892000D7F8142107F58C73A3F584731B681344DF
:10893000C7F81431D7F814311B78002B01D01B2352
:1089400091E007F1140307F1B40107F1E4000022FC
:1089500000F0E4FC0346002B01D11B2383E000233D
:1089600081E000BF704401008444010007F58C736E
:10897000A3F5867311223E49186809F0CEF9034623
:10898000002B6FD107F58C73A3F588731B68012248
:108990001A7007F58C73A3F586731B681133C7F83B
:1089A0001431D7F8140107F1100307F11401002264
:1089B0000192002200924022FEF7A8FC0346002B01
:1089C00006D107F58C73A3F584731B68002B01D1C6
:1089D0001B2348E0D7F8142107F58C73A3F58473A3
:1089E0001B681344C7F8143107F58A73184606F05C
:1089F00041FFD7F8140107F1100307F1E401002249
:108A00000192002200923022FEF780FC0346002BE8
:108A100006D107F58C73A3F584731B68002B01D175
:108A20001B2320E0D7F8142107F58C73A3F584737A
:108A30001B681344C7F81431D7F814311B78002B86
:108A400001D01B230FE007F1140307F1E40000221B
:108A5000002100F063FC0346002B01D11B2302E040
:108A6000002300E00023184607F58C77BD4680BD43
:108A70009844010080B582B000AF78603960102260
:108A80000021386809F02BF83B684FF4FF221A6088
:108A90003B681B6803F118023B685A603B681B681F
:108AA0001B68104A934201D0002316E03B681B6804
:108AB00004337968184609F016F90346002B01D0F3
:108AC00000230AE03B685A683B689A603B680122D1
:108AD0005A733B6801221A73012318460837BD46B2
:108AE00080BD00BFBEBAEDFE80B582B000AF786039
:108AF000396010220021386808F0F1FF4FF400625D
:108B00000021154808F0EBFF3B68134A1A603B68E8
:108B10001B6803F118023B685A603B681B680F4AE8
:108B20001A603B681B6804337A681021184606F007
:108B30002AFA3B681B6800225A613B685A683B6806
:108B40009A603B6801225A733B6800221A73012322
:108B500018460837BD4680BDB8040020BEBAEDFEF9
:108B600080B584B000AF786039603B681B7B002B18
:108B700001D001233AE0786809F0C7F8F8601D4A8F
:108B80003B689B68D31ABB603B689B687A68B9688E
:108B9000184606F0F8F93B689A68FB681A443B6887
:108BA0009A603B689A683B681B6803F500639A42C9
:108BB00007D33B681B6803F500623B689A6000239B
:108BC00014E03B689A683B6859683B681B685B69BE
:108BD0000B449A4209D33B689A683B685B68D21A97
:108BE0003B681B685A61012300E0012318461037D7
:108BF000BD4680BDB80C002080B584B000AF786061
:108C00003960786806F022FF0346002B25D0154B0B
:108C1000FB60FB6804337968184609F064F8034682
:108C2000002B01D0002319E0FB6804333A681021BF
:108C3000184606F0A8F94FF400620A494FF4FF20E5
:108C400006F0BDFE0346002B01D0002306E04FF4E2
:108C500000620021034808F042FF01231846103744
:108C6000BD4680BDB804002080B590B000AFF8606C
:108C7000B9607A601821B86806F077FE034683F081
:108C80000103DBB2002B0FD007F110032C4A302177
:108C9000184606F078F9FB685A6807F11003194680
:108CA000786805F0C5FF48E007F11003254A302138
:108CB000184606F068F9BB681A6807F110033021FE
:108CC000184606F055FB07F110031F4A30211846DD
:108CD00006F07EF9BB681B681C4A934217D1BB683B
:108CE0001A1D07F110033021184606F071F907F13B
:108CF0001003174A3021184606F06AF9BB685A6912
:108D000007F110033021184606F068FB06E007F172
:108D10001003104A3021184606F05AF907F11003E3
:108D20000D4A3021184606F053F9FB685A6807F1DE
:108D300010031946786805F07BFF4037BD4680BDBB
:108D4000AC440100C8440100D4440100BEBAEDFEA9
:108D5000D8440100E04401008441010080B58EB098
:108D600000AF78607B685B681A463349334805F08A
:108D70005FFF07F10803324A3021184606F003F975
:108D800007F108034FF4FF223021184606F0F0FAED
:108D900007F108032B4A3021184606F019F907F1AC
:108DA00008034FF400623021184606F074FA07F108
:108DB0000803254A3021184606F00AF907F108038E
:108DC00001223021184606F0FDF907F108031F4A79
:108DD0003021184606F0FCF87B685A6807F1080352
:108DE00019461B4805F024FF07F108034FF4006201
:108DF00030211846FEF716FA07F10803154A30210C
:108E0000184606F0E5F87B685A6807F1080319462A
:108E1000114805F00DFF114A4FF4FF217868FFF764
:108E200023FF0F4A0F497868FFF71EFF00231846FB
:108E30003837BD4680BD00BFEC440100004501004D
:108E400004450100104501001C450100844101005A
:108E500024450100743901002C450100384501000A
:108E600040450100B804002080B586B000AF7860AE
:108E70004FF4FF23BB60244AB9687868FFF7F4FE1B
:108E8000BB681B68214A934216D1BB6818337B61CB
:108E900000233B610BE07B685B687A6912781046BF
:108EA00098477B6901337B613B6901333B61BB6858
:108EB0005B693A699A42EED3154BBB60154AB968B3
:108EC0007868FFF7D1FEBB681B68104A934216D141
:108ED000BB6818337B610023FB600BE07B685B6839
:108EE0007A691278104698477B6901337B61FB6889
:108EF0000133FB60BB685B69FA689A42EED30023DA
:108F000018461837BD4680BD70340100BEBAEDFE6C
:108F1000B80400204845010080B584B000AFF86077
:108F2000B9607A603549F86808F0DDFE0346002B29
:108F300006D03349F86808F0D6FE0346002B20D14E
:108F40007B685B681A462F492F4805F05FFE7B68F7
:108F50005B681A462D492E4805F058FE7B685B6811
:108F60001A462C492C4805F051FE7B685B681A466E
:108F70002A492B4805F04AFEBB6801221A700023DB
:108F800037E02849F86808F0AEFE0346002B06D00B
:108F90002549F86808F0A7FE0346002B07D1BB68F7
:108FA00001221A707868FFF7D9FE034621E01F49B5
:108FB000F86808F098FE0346002B07D1BB68012231
:108FC0001A707868FFF750FF034612E01849F868F6
:108FD00008F089FE0346002B0AD1BB6801221A70F3
:108FE0004FF400614FF4FF20FEF740FF034600E01E
:108FF000002318461037BD4680BD00BFA8390100C8
:109000004C45010054410100004501006424010069
:109010008824010058450100704501007845010091
:1090200094450100B83901009C450100A8450100A4
:10903000B445010080B58EB004AFF860B9607A60C5
:109040003B6000237B623B68002B05D03B6B002B11
:1090500002DDBB68002B01D1002331E007F11403CE
:109060001946786BFFF706FD0346002B16D007F173
:109070001400002303933B6B02933B6801934FF072
:10908000FF3300934FF0FF33BA68F96806F046FFEC
:10909000786207F11403184606F0F3FC7B6A002B94
:1090A0000AD17B68002B01D0796800E006493A6B51
:1090B0000023386806F00AFE386808F026FE0346EA
:1090C00018462837BD4680BDA83B010080B598B042
:1090D00002AFF860B9607A603B6007F110023B684C
:1090E0000193402300931346194AB968F868FFF7C3
:1090F000A1FF78657B6D002B25D07B6D012B19DDE1
:109100007B7C3B653B6D0133124A13441B7803F0B3
:109110000303022B02D13B6D203B00E03B6D582B3B
:1091200008D107F1100310220021184603F00AFFAE
:10913000034609E007F110030A220021184603F054
:1091400001FF034600E07B6818465837BD4680BDE6
:10915000A83B01007146010080B586B000AFF86001
:10916000B9607A60BB68002B24D0B86808F0CDFDE8
:109170000346002B1ED0FB685B221A70FB68581C4C
:1091800000233C22B96806F0A1FD0021F86808F030
:109190009DFD78617B695A1C7A615D221A700749CE
:1091A000786908F0AAFD7B68002B03D07968F8681D
:1091B000FFF7D6FC00BF1837BD4680BD84410100D3
:1091C00080B586B000AFF860B9607A603B607868BF
:1091D00006F0C2FF0346FB7500233D22B968F8681C
:1091E00006F074FD0021F86808F070FD38613B69F5
:1091F0005A1C3A613D221A703A69FB68D31AC3F1CE
:109200003E031A46FB7D7968386906F05FFD002150
:10921000F86808F05BFD38610749386908F06DFDB2
:109220003B68002B03D03968F868FFF799FC00BF52
:109230001837BD4680BD00BF8441010080B588B0AD
:1092400000AFF860B9607A603B60334808F05DFDBC
:1092500003467B610023FB614FF0FF33BB61B96ABA
:10926000786806F083FCFB6800221A701AE0FB693C
:10927000BB61FB69FA68D018FB69C3F140037A68E7
:10928000194606F02BFC02E0FB690133FB61BB6869
:109290001B68FA699A4205DAFB69FA6813441B787D
:1092A000002BF1D1BB681B68FA699A4203DAFA69AC
:1092B000BB699A42DBD1FB681B78002B0ED0FB699F
:1092C000402B02D1FB69013BFB61FB69FA68134447
:1092D00000221A703968F868FFF742FCB96A7868AA
:1092E00006F030FCBB6800221A60FA697B699A427A
:1092F0000DDDFA697B69D31AFA68134406491846EA
:1093000008F0F1FC0346002B01D1012300E000230B
:1093100018462037BD4680BD8441010090B5A9B0F4
:1093200004AFF860B9607A603B6007F16C031946DE
:109330003868FFF79FFB0346002B27D1BB68002B43
:1093400022D07B68002B1FD007F15C0319463868D8
:10935000FFF7CAFB0346002B01D10023FAE207F115
:109360005C0207F11403F9681846FFF7F5FE07F1F0
:109370005C0307F114007A68B968FFF721FF07F171
:109380005C03184606F07DFB0123E3E2BB68002B7B
:109390002BD07B68002B28D007F16C0007F1540319
:1093A00003934023029307F1140301934FF0FF331B
:1093B00000934FF0FF33BA68F96806F0AFFDC7F8C5
:1093C0008800D7F88830002B34D007F1140379686F
:1093D000184608F088FC0346002B2BD107F16C03DC
:1093E000184606F04EFB0123B4E2BB68002B22D0E6
:1093F0007B68002B1FD107F16C00002303934023EF
:10940000029307F1140301934FF0FF3300934FF0E1
:10941000FF33BA68F96806F081FDC7F88800D7F80D
:109420008830002B07D107F16C03184606F029FBA2
:1094300001238FE200BF07F16C03184606F021FB01
:1094400007F1140340223968184606F06CFE07F154
:109450005C0207F1140311461846FFF745FB03466B
:10946000002B01D1002375E207F16C03194638681F
:10947000FFF700FB0346002B16D107F15C0207F152
:109480001403F9681846FFF767FE07F15C0307F15C
:1094900014007A68B968FFF793FE07F15C03184679
:1094A00006F0EFFA012355E207F1580207F16C03C9
:1094B0001146184606F046FB00233B61FB68002B73
:1094C00004D0F86808F021FC034600E00023C7F848
:1094D0008430D7F88430002B40F3C28007F16C024F
:1094E00007F114034021184606F0F8FA0346002B52
:1094F00038D107F15C0407F16C0207F1100107F1A4
:10950000140007F1580300932346FFF797FEF8670E
:10951000BB68002B1BD07B68002B18D0FB6F002B87
:1095200005D107F15C031946C248FFF719FB07F1A3
:109530005C0207F11403F9681846FFF70DFE07F106
:109540005C0307F114007A68B968FFF739FE07F188
:10955000140307F15C0107F16C003A6806F04CFE59
:109560000346F7E107F11403184606F064FBC7F859
:1095700080005D21D7F8800008F0E3FBC7F88C007D
:10958000D7F880301B785B2B05D1D7F88C30002BB7
:1095900001D0012300E00023C7F88830D7F88830D5
:1095A000002B28D0D7F880300133184606F043FB53
:1095B000C7F88000D7F88010D7F88C0006F052FB6F
:1095C000C7F88C00D7F88C20D7F88030D31AD7F89A
:1095D00084209A420CD1D7F884301A46F968D7F81B
:1095E000800006F0F6FA0346002B01D1012300E0CB
:1095F0000023C7F88830D7F88830002B02D0BB682A
:10960000002B28D007F1100107F11403402218465F
:1096100006F0D3FD0346002B1DD107F15C0407F1D2
:109620006C0207F1100107F1140007F158030093D1
:109630002346FFF703FE07F16C0207F114034021F4
:10964000184606F04BFA07F1100107F11403402207
:10965000184606F0B2FDD7F88830002B3FF43EAF35
:1096600007F15C0407F16C0207F1100107F1140027
:1096700007F1580300932346FFF7E0FDBB68002B7A
:109680000FD107F16C0207F114034021184606F0D0
:1096900025FA07F1580207F16C031146184606F047
:1096A00051FABB68002B04D0B86808F02EFB0346C3
:1096B00000E00023C7F8843007F16C0207F11403BF
:1096C0004021184606F00AFA0346002B30D107F174
:1096D0005C0407F16C0207F1100107F1140007F1B7
:1096E000580300932346FFF7A9FDF867BB68002BDA
:1096F00013D07B68002B10D0FB6F002B05D107F136
:109700005C0319464B48FFF72BFA07F15C0307F19E
:1097100014007A68B968FFF753FD07F1140307F1E5
:109720005C0107F16C003A6806F066FD034611E142
:1097300007F11403184606F07EFAC7F880003D21B1
:10974000D7F8800008F0C2FAC7F88C00D7F88C3040
:10975000002B06D13A21D7F8800008F0B7FAC7F8F5
:109760008C00D7F88C30002B1ED0D7F88430002B1B
:109770001ADDD7F88010D7F88C0006F073FA02468D
:10978000D7F88030D31AD7F884209A420CD1D7F872
:1097900084301A46B968D7F8800006F01AFA0346F2
:1097A000002B01D1012300E00023C7F88830BB68FB
:1097B000002B03D0D7F88830002B3DD1D7F880306C
:1097C0001B785B2B38D0BB68002B08D107F15802FF
:1097D00007F16C031146184606F0B4F96CE707F17F
:1097E000100107F114034022184606F0E6FC034678
:1097F000002B7FF461AF07F15C0407F16C0207F105
:10980000100107F1140007F1580300932346FFF7F6
:1098100015FD07F16C0207F114034021184606F00C
:109820005DF907F1100107F114034022184606F014
:10983000C4FC41E784410100D7F880301B785B2BE2
:109840000CBF01230023DBB2FB6707F15C0407F1C7
:109850006C0207F1100107F1140007F1580300939F
:109860002346FFF7EBFCBB68002B0AD07B68002B7C
:1098700007D007F15C0307F114007A68B968FFF7B5
:109880009FFC07F16C0207F114034021184606F013
:1098900025F9FB6F002B08D007F1100107F1140325
:1098A0004022184606F089FC31E007F1580207F122
:1098B0006C031146184606F045F928E007F110013F
:1098C00007F114034022184606F077FC0346002BEC
:1098D0001DD107F15C0407F16C0207F1100107F1DB
:1098E000140007F1580300932346FFF7A7FC07F184
:1098F0006C0207F114034021184606F0EFF807F157
:10990000100107F114034022184606F056FC07F137
:109910006C0207F114034021184606F0DFF80346F5
:10992000002BCBD107F15C0407F16C0207F11001A9
:1099300007F1140007F1580300932346FFF77EFC5C
:1099400007F1140307F15C0107F16C003A6806F0B7
:1099500053FC034618469437BD4690BD80B586B08B
:1099600000AF7860396000237B617B683B617A6877
:10997000204B83FB02139910D317C91A0B469B0087
:109980000B445B00D31AFB60FB68002B05DAFB6815
:10999000DBB2C3F13003DBB203E0FB68DBB2303390
:1099A000DBB27A69511C796111463A680A44137036
:1099B0007B68104A82FB03129210DB17D31A7B607C
:1099C0007B68002BD3D13B69002B07DA7B695A1CDB
:1099D0007A611A463B6813442D221A707B693A68F3
:1099E000134400221A70386806F021FC00BF1837B3
:1099F000BD4680BD6766666680B582B000AF1F4B0E
:109A00007B607B6803221A617B6803225A617B6852
:109A10001B4A9A617B681B4ADA617B684FF480625B
:109A20001A627B6800229A627B6800225A627B6815
:109A30000022DA627B68124A1A667B68124A5A660A
:109A40007B6896229A667B6800221A677B680022F0
:109A5000DA667B6800225A677B6807330B49184631
:109A600008F04BF97B680A49184608F046F97B680C
:109A700020229A7100BF0837BD4680BDB80C002077
:109A8000C0450100600D002060110020CC450100A0
:109A9000D045010080B58CB000AFF860B9607A6045
:109AA0003E4B3B623B6A1B78DBB2002B01D1FFF7D8
:109AB000A3FFFA6813465B001344DB006033374AA8
:109AC0001344FB61BB687B62FB691B69BB62FB697A
:109AD000DB68BB610023FB62BA6ABB699A422BD97F
:109AE000FB699A68BB6AD31A7B617A697B68934287
:109AF00028BF13467B61FB695A68BB6A13443B610C
:109B00007A693969786A07F0DCFFFA6A7B6913447D
:109B1000FB627A6A7B6913447B627A687B69D31A39
:109B20007B60BA6A7B691344BB62FB699B68BA6A53
:109B30009A4201D10023BB62BA69BB6AD31A7B6126
:109B40007A697B68934228BF13467B617B69002B4F
:109B500019D0FB695A68BB6A13443B617A69396959
:109B6000786A07F0AEFFFA6A7B691344FB627A6A8F
:109B70007B6913447B627A687B69D31A7B60BA6A1B
:109B80007B691344BB62FB6A002B02D0FB69BA6A93
:109B90001A61FB6A18463037BD4680BDB80C0020FC
:109BA00080B588B000AFF860B9607A60BB68BB610F
:109BB000FB685A1C13465B001344DB001F4A134426
:109BC0007B617B695B69022B29D0022B2ED8002B8D
:109BD00002D0012B13D029E0786906F00EFC386121
:109BE0003A697B689A4202D20023FB6121E07B68DC
:109BF000FB617A68B969786906F0BBFB19E078699E
:109C000006F0FBFB38617A683B69934228BF134634
:109C1000FB61FA69B969786906F0ABFB09E07A681B
:109C2000B969786906F04AFBF86102E00023FB613C
:109C300000BFFB6918462037BD4680BDB80C002028
:109C400080B588B000AFF860B9607A600E4BFB61F8
:109C5000FB691B78DBB2002B01D1FFF7CDFEEFF3E0
:109C600011834FF0500181F31188BB617A68B968A4
:109C7000F868FFF795FF7861BB6983F311887B690A
:109C800018462037BD4680BDB80C002080B584B092
:109C900000AF0E4BBB60BB681B78DBB2002B01D161
:109CA000FFF7AAFE0A4B7B607B681B693B607B6801
:109CB000DB683A689A4202D00123FB6001E000238E
:109CC000FB60FB6818461037BD4680BDB80C00200D
:109CD000180D002080B586B000AF7860114B7B6115
:109CE0007B691B78DBB2002B01D1FFF785FEEFF318
:109CF00011834FF0500181F311883B617B685A1C3E
:109D000013465B001344DB00064A1344184606F072
:109D100074FBF8603B6983F31188FB6818461837B9
:109D2000BD4680BDB80C002080B586B000AF78601D
:109D30000023FB6000F012FD564B1B68002B01D185
:109D400000F01AF9544B1A687B681340002B40F05E
:109D50008A807B68002B18D0504B1B687A681344AC
:109D60007B607B6803F00703002B0ED07B6823F039
:109D7000070308337B607B6803F00703002B04D0E4
:109D80004FF0500080F31188FEE77B68002B6AD00B
:109D9000434B1B687A689A4265D8424B3B61414B02
:109DA0001B687B6104E07B693B617B691B687B61AD
:109DB0007B695B687A689A4203D97B691B68002BD0
:109DC000F1D1344B1B687A699A424CD03B691A68CE
:109DD000324B1B681344FB607B691A683B691A604D
:109DE0007B695A687B68D21A2C4B1B685B009A42CD
:109DF00019D97A697B681344BB60BB6803F0070319
:109E0000002B04D04FF0500080F31188FEE77B69EF
:109E10005A687B68D21ABB685A607B697A685A6054
:109E2000B86800F00FF91E4B1A687B695B68D31A9B
:109E30001B4A13601A4B1A681B4B1B689A4203D2C9
:109E4000174B1B68184A13607B695A68124B1B68D2
:109E50001A437B695A607B6900221A60134B1B68A6
:109E60000133124A136000F087FCFB68002B01D11C
:109E700007F0B4FDFB6803F00703002B04D04FF09C
:109E8000500080F31188FEE7FB6818461837BD467E
:109E900080BD00BF00120020141200201C00002012
:109EA00004120020F8110020081200200C120020DB
:109EB00080B584B000AF78607B68FB607B68002B66
:109EC00042D0234B1B685B42FA681344FB60FB687B
:109ED000BB60BB685A681F4B1B681340002B04D142
:109EE0004FF0500080F31188FEE7BB681B68002B21
:109EF00004D04FF0500080F31188FEE7BB685A6829
:109F0000144B1B681340002B1ED0BB681B68002B32
:109F10001AD1BB685A680F4B1B68DB431A40BB68F9
:109F20005A6000F01BFCBB685A680B4B1B6813445B
:109F3000094A1360B86800F085F8084B1B680133C4
:109F4000064A136000F018FC00BF1037BD4680BD04
:109F50001C00002014120020041200201012002007
:109F600080B400AF034B1B681846BD465DF8047B08
:109F7000704700BF0412002080B485B000AF4FF4DA
:109F8000C043BB60284BFB60FB6803F00703002B5A
:109F90000CD0FB680733FB60FB6823F00703FB6012
:109FA000BA68FB68D31A204A1344BB60FB687B6025
:109FB0001E4A7B6813601D4B00225A607B68BA689A
:109FC0001344FB601A4B1B68FA68D31AFB60FB68EA
:109FD00023F00703FB60FB68164A1360154B1B68F0
:109FE00000225A60134B1B6800221A607B683B609A
:109FF0003B68FA68D21A3B685A600E4B1A683B6895
:10A000001A603B685B680C4A13603B685B680B4AEC
:10A0100013600B4B4FF000421A6000BF1437BD466F
:10A020005DF8047B704700BF0000FF1FF81100209F
:10A030001C00002000120020081200200412002042
:10A040001412002080B485B000AF7860284BFB600C
:10A0500002E0FB681B68FB60FB681B687A689A4239
:10A06000F7D8FB68BB60FB685B68BA6813447A6822
:10A070009A4208D1FB685A687B685B681A44FB689F
:10A080005A60FB687B607B68BB607B685B68BA6812
:10A090001A44FB681B689A4218D1FB681A68154B72
:10A0A0001B689A420DD07B685A68FB681B685B6826
:10A0B0001A447B685A60FB681B681A687B681A60E0
:10A0C00008E00C4B1A687B681A6003E0FB681A68AA
:10A0D0007B681A60FA687B689A4202D0FB687A68EB
:10A0E0001A6000BF1437BD465DF8047B704700BF9F
:10A0F000F81100200012002080B400AF0E4B1B6846
:10A100000D4A43F0704313600C4B06221A600C4B4F
:10A110001B680C4AA2FB03239B090B4A013B1360FB
:10A120000A4B00221A60054B07221A6000BFBD4689
:10A130005DF8047B704700BF20ED00E010E000E018
:10A1400018000020D34D621014E000E018E000E099
:10A1500080B400AF034B07221A6000BFBD465DF814
:10A16000047B704710E000E080B400AF034B062290
:10A170001A6000BFBD465DF8047B704710E000E048
:10A1800080B400AF054B1B68044A43F470031360AE
:10A1900000BFBD465DF8047B704700BF88ED00E05E
:10A1A00080B584B000AF294BFB60FB681B78DBB245
:10A1B000BB60FB68FF221A70FB681B78DBB2FB7187
:10A1C000FB79DBB203F05003DAB2214B1A70214B5A
:10A1D00007221A6009E01F4B1B68013B1D4A1360F0
:10A1E000FB79DBB25B00DBB2FB71FB79DBB203F026
:10A1F0008003802BEFD0174B1B681B02154A13609E
:10A20000144B1B6803F4E063124A1360BB68DAB2B4
:10A21000FB681A70104B1B680F4A43F470031360FD
:10A220000E4B00221A60FFF767FFFFF791FFFFF761
:10A23000A7FF0B4B1B680A4A43F04043136000F032
:10A240005FF8002318461037BD4680BD00E400E0EB
:10A25000EE1300201812002020ED00E02000002066
:10A2600034EF00E080B400AF4FF0500080F311886D
:10A270000D4B1B6801330C4A13600B4B1B68012B01
:10A2800009D10A4B1B68DBB2002B04D04FF0500001
:10A2900080F31188FEE7BFF34F8FBFF36F8F00BFCE
:10A2A000BD465DF8047B70472000002004ED00E00F
:10A2B00080B400AF084B1B68013B074A1360064B94
:10A2C0001B68002B03D14FF0000080F3118800BF02
:10A2D000BD465DF8047B70472000002080B400AFCD
:10A2E000064B4FF080521A60BFF34F8FBFF36F8F52
:10A2F00000BFBD465DF8047B704700BF04ED00E081
:10A3000080B483B000AF134B1B68DBB2FB71124B00
:10A310001B78DBB2002B00D1FEE7104B1B78642BBF
:10A3200000D9FEE74FF060404FF46D4140EA010074
:10A330004FF0080140EA01000068006880F30888D7
:10A3400062B600DF00BF00BF0C37BD465DF8047B7E
:10A35000704700BFF8370100E44501007046010076
:10A36000054B19680868B0E8F04F80F309884FF092
:10A37000000080F3118870474412002000BF00BF26
:10A38000EFF30980114B1A681EF0100F08BF20ED83
:10A39000108A20E9F04F10602DE908404FF050007E
:10A3A00080F3118800F080FB4FF0000080F31188EB
:10A3B000BDE8084019680868B0E8F04F1EF0100FBB
:10A3C00008BFB0EC108A80F309887047441200205F
:10A3D00000BF00BF80B483B000AFEFF305837B60A4
:10A3E0007B680F2B0ED9114A7B6813441B78FB70D6
:10A3F0000F4B1B78FA789A4204D24FF0500080F34A
:10A400001188FEE70B4B1B6803F4E0620A4B1B68E4
:10A410009A4204D94FF0500080F31188FEE700BF44
:10A420000C37BD465DF8047B704700BFF0E300E0E9
:10A43000EE1300200CED00E01812002080B485B06F
:10A4400000AF786039600023FB6014E00F4AFB68BE
:10A4500052F83330002B0BD10C49FB683A6841F8B5
:10A4600033200A4AFB68DB0013447A685A6006E02E
:10A47000FB680133FB60FB68042BE7D900BF00BF1A
:10A480001437BD465DF8047B704700BF1C120020E6
:10A4900080B485B000AF78600023FB6016E0104AFE
:10A4A000FB68DB0013445B687A689A420BD10C4A64
:10A4B000FB68002142F83310094AFB68DB001344B3
:10A4C00000225A6006E0FB680133FB60FB68042B46
:10A4D000E5D900BF00BF1437BD465DF8047B704767
:10A4E0001C12002080B582B000AF7860FFF7BAFE82
:10A4F0002A4B1B680133294A1360294B1B68002B28
:10A5000009D1274A7B681360244B1B68012B10D1AB
:10A5100000F08EFC0DE0234B1B68002B09D1204B73
:10A520001B68DA6A7B68DB6A9A4202D81C4A7B683D
:10A5300013601D4B1B6801331B4A13601A4B1A68CA
:10A540007B685A647B68DA6A184B1B689A4203D9A5
:10A550007B68DB6A154A13607B68DA6A13469B00E6
:10A5600013449B00124A1A447B6804331946104670
:10A5700006F010F8FFF79CFE0A4B1B68002B08D072
:10A58000074B1B68DA6A7B68DB6A9A4201D2FFF7E5
:10A59000A5FE00BF0837BD4680BD00BF30130020B8
:10A5A000441200203C1300204C13002038130020DC
:10A5B0004812002080B584B000AF78600023FB60B3
:10A5C0007B68002B11D00D4B1B68002B04D04FF083
:10A5D000500080F31188FEE700F0C0F80021786891
:10A5E00000F098FE00F0C8F8F860FB68002B01D17D
:10A5F000FFF774FE00BF1037BD4680BD5813002022
:10A6000080B588B000AF78607B687B617B69002B88
:10A6100004D14FF0500080F31188FEE7294B1B68EE
:10A620007A699A4202D10023FB7745E0FFF71AFED0
:10A630007B695B693B61244B1B68FB60234B1B6898
:10A64000BB60FFF735FE3A69FB689A4203D03A696E
:10A65000BB689A4202D10223FB772DE03B691C4A7A
:10A6600093421DD17B699B6A002B16D10323FB7794
:10A670000023BB610DE07A69BB6913445C331B782E
:10A68000DBB2012B02D10223FB7715E0BB6901335A
:10A69000BB61BB69002BEEDD0EE00223FB770BE014
:10A6A0003B690C4A934202D03B69002B02D1042340
:10A6B000FB7701E00123FB77FB7F18462037BD467F
:10A6C00080BD00BF44120020E8120020EC120020E0
:10A6D0001C1300200413002080B584B002AF194B76
:10A6E0000193002300930023C8221749174806F05E
:10A6F000FFFF78607B68012B02D100F0DBFE786001
:10A700007B68012B10D14FF0500080F31188104B63
:10A710004FF0FF321A600F4B01221A600E4B0022DD
:10A720001A60FFF73DFD08E07B68B3F1FF3F04D1FD
:10A730004FF0500080F31188FEE700BF0837BD4698
:10A7400080BD00BF54130020D84501000DAE0000AD
:10A75000501300203C1300203413002080B400AFBD
:10A76000044B1B680133034A136000BFBD465DF80C
:10A77000047B70475813002080B584B000AF0023DD
:10A78000FB600023BB603C4B1B68002B04D14FF0E7
:10A79000500080F31188FEE7FFF764FD364B1B681D
:10A7A000013B354A1360344B1B68002B5CD1334BA3
:10A7B0001B68002B58D02FE0314BDB68DB68FB6057
:10A7C000FB681833184605F042FFFB68043318464F
:10A7D00005F03DFFFB68DA6A2A4B1B689A4203D9F1
:10A7E000FB68DB6A274A1360FB68DA6A13469B0042
:10A7F00013449B00244A1A44FB680433194610464C
:10A8000005F0C8FEFB68DA6A204B1B68DB6A9A42D7
:10A8100002D31F4B01221A60194B1B68002BCBD1AE
:10A82000FB68002B01D000F0D7FB1A4B1B687B6044
:10A830007B68002B10D000F07BF80346002B02D081
:10A84000134B01221A607B68013B7B607B68002B05
:10A85000F1D1104B00221A600D4B1B68002B03D066
:10A860000123BB60FFF73AFDFFF722FDBB681846E6
:10A870001037BD4680BD00BF5813002030130020A4
:10A88000F01200203813002048120020441200204B
:10A89000441300204013002080B483B000AF054B68
:10A8A0001B687B607B6818460C37BD465DF8047BEF
:10A8B000704700BF3413002080B582B000AFFFF7AF
:10A8C00089FD00237B60044B1B683B603B68184696
:10A8D0000837BD4680BD00BF3413002080B400AFF0
:10A8E000034B1B681846BD465DF8047B704700BFEC
:10A8F0003013002080B485B000AF78607B68002BF7
:10A9000002D10A4B1B6800E07B68FB60FB68002BF0
:10A9100004D14FF0500080F31188FEE7FB68343318
:10A9200018461437BD465DF8047B7047441200207A
:10A9300080B586B000AF00237B61504B1B68002BB5
:10A9400040F08F804E4B1B6801333B614C4A3B69A2
:10A9500013603B69002B1AD14A4B1B681B68002B04
:10A9600004D04FF0500080F31188FEE7454B1B6880
:10A97000FB60454B1B68434A1360434AFB68136006
:10A98000424B1B680133414A136000F025FB404BEA
:10A990001B683A699A4249D33A4B1B681B68002BE3
:10A9A00004D13B4B4FF0FF321A603FE0354B1B6840
:10A9B000DB68DB68BB60BB685B687B603A697B68AF
:10A9C0009A4203D2324A7B6813602FE0BB6804339B
:10A9D000184605F03CFEBB689B6A002B04D0BB68A0
:10A9E0001833184605F033FEBB68DA6A294B1B683A
:10A9F0009A4203D9BB68DB6A264A1360BB68DA6AED
:10AA000013469B0013449B00234A1A44BB6804333B
:10AA10001946104605F0BEFDBB68DA6A1F4B1B687D
:10AA2000DB6A9A42B8D301237B61B5E71B4B1B68F5
:10AA3000DA6A194913469B0013449B000B441B68B8
:10AA4000012B01D901237B61154B1B68002B01D120
:10AA500006F0CCFF134B1B68002B09D001237B6150
:10AA600006E00F4B1B6801330D4A136006F0BEFF72
:10AA70007B6918461837BD4680BD00BF58130020BB
:10AA800034130020E8120020EC12002048130020AC
:10AA900050130020381300204812002044120020D8
:10AAA000401300204413002080B582B000AF394B22
:10AAB0001B68002B03D0384B01221A6065E0364B2F
:10AAC00000221A60FFF7F8FE0346344A1360334B46
:10AAD0001A68334B1B689A4209D9324B1B68596D6F
:10AAE0002E4A10682E4A1268821A0A445A652B4B65
:10AAF0001B682B4A13602B4B1B681A68294B1B6879
:10AB00001B6B9A4208D8274B1A68264B1B683433B4
:10AB10001946104606F057FF234B1B687B600AE07E
:10AB20007B68002B04D14FF0500080F31188FEE7C2
:10AB30007B68013B7B601D497A6813469B00134488
:10AB40009B000B441B68002BEAD07A6813469B00DD
:10AB500013449B00154A13443B603B685B685A688A
:10AB60003B685A603B685A683B6808339A4204D194
:10AB70003B685B685A683B685A603B685B68DB68A7
:10AB8000084A1360084A7B68136000BF0837BD4657
:10AB900080BD00BF58130020441300206013002024
:10ABA0005C130020441200203813002048120020BB
:10ABB00080B582B000AF786039607B68002B04D12B
:10ABC0004FF0500080F31188FEE7074B1B681833E5
:10ABD0001946786805F002FD0121386800F09AFBFB
:10ABE00000BF0837BD4680BD4412002080B584B048
:10ABF00000AFF860B9607A60FB68002B04D14FF0B9
:10AC0000500080F31188FEE70A4B1B681833194681
:10AC1000F86805F0BFFC7B68002B02D04FF0FF33D3
:10AC2000BB607968B86800F075FB00BF1037BD469F
:10AC300080BD00BF4412002080B584B000AF7860B2
:10AC40007B68DB68DB68BB60BB68002B04D14FF01E
:10AC5000500080F31188FEE7BB681833184605F0F2
:10AC6000F6FC1E4B1B68002B1DD1BB680433184635
:10AC700005F0EDFCBB68DA6A194B1B689A4203D9F0
:10AC8000BB68DB6A164A1360BB68DA6A13469B002E
:10AC900013449B00134A1A44BB68043319461046F8
:10ACA00005F078FC05E0BB68183319460E4805F03E
:10ACB00071FCBB68DA6A0D4B1B68DB6A9A4205D9E6
:10ACC0000123FB600A4B01221A6001E00023FB60B4
:10ACD000FB6818461037BD4680BD00BF58130020E2
:10ACE0003813002048120020F012002044120020E7
:10ACF0004413002080B483B000AF7860064B1A681C
:10AD00007B681A60054B1A687B685A6000BF0C3775
:10AD1000BD465DF8047B70474813002034130020C3
:10AD200080B586B000AF786039607B68002B04D1B5
:10AD30004FF0500080F31188FEE73B68002B04D1F0
:10AD40004FF0500080F31188FEE7FFF78BFA264B97
:10AD50001B683B617B685B683A69D31AFB60234BD5
:10AD60001B6893F85D30002B07D0204B1B68002236
:10AD700083F85D2001237B612EE03B681B68B3F103
:10AD8000FF3F02D100237B6126E07B681A68184BE5
:10AD90001B689A420AD07B685B683A699A4205D37D
:10ADA00001237B613B6800221A6015E03B681B6849
:10ADB000FA689A420BD23B681A68FB68D21A3B6861
:10ADC0001A607868FFF796FF00237B6104E03B6818
:10ADD00000221A6001237B61FFF76AFA7B6918463B
:10ADE0001837BD4680BD00BF341300204412002038
:10ADF0004813002080B400AF034B01221A6000BF4B
:10AE0000BD465DF8047B70474413002080B582B0D6
:10AE100000AF786000F04CF8044B1B68012B01D99F
:10AE2000FFF75CFA06F0E9FDF4E700BF48120020E6
:10AE300080B582B000AF00237B600CE07A681346D7
:10AE40009B0013449B00124A1344184605F075FBFF
:10AE50007B6801337B607B68052BEFD90D4805F0DB
:10AE60006CFB0D4805F069FB0C4805F066FB0C48CF
:10AE700005F063FB0B4805F060FB0B4B054A1A60BD
:10AE80000A4B054A1A6000BF0837BD4680BD00BFA7
:10AE900048120020C0120020D4120020F01200201E
:10AEA000041300201C130020E8120020EC120020E4
:10AEB00080B582B000AF19E0FFF7D4F9104BDB6822
:10AEC000DB687B607B680433184605F0C0FB0D4BE4
:10AED0001B68013B0B4A13600B4B1B68013B0A4A82
:10AEE0001360FFF7E5F9786806F0F9FC064B1B687C
:10AEF000002BE1D100BF00BF0837BD4680BD00BFB9
:10AF000004130020301300201813002080B586B0F1
:10AF100000AFF860B9607A60FB70FB68002B02D16B
:10AF20002C4B1B6800E0FB687B61BB687A691A6088
:10AF30007B6903F13402BB685A607B69DA6ABB68DB
:10AF40001A617B691A6BBB68DA617B695A6CBB68F2
:10AF50009A607B69DA6CBB685A617B695A6DBB6821
:10AF60009A61FB78052B1AD01A4B1B687A699A42B2
:10AF700003D1BB6800221A7318E0BB68FA781A7311
:10AF8000FB78032B12D1FFF7E9FB7B699B6A002B4F
:10AF900002D0BB6802221A73FFF7EEFB06E0786965
:10AFA000FFF72EFB03461A46BB681A737B68002B1B
:10AFB00009D07B691B6B184606F075FC03461A46E0
:10AFC000BB681A8402E0BB6800221A8400BF1837ED
:10AFD000BD4680BD4412002080B400AF0A4B1B6800
:10AFE0001B68002B04D1094B4FF0FF321A6005E0BB
:10AFF000054B1B68DB681B68044A136000BFBD4635
:10B000005DF8047B704700BFE81200205013002059
:10B0100080B483B000AF054B1B687B607B6818462B
:10B020000C37BD465DF8047B704700BF441200201A
:10B0300080B483B000AF0B4B1B68002B02D10123FF
:10B040007B6008E0084B1B68002B02D102237B6069
:10B0500001E000237B607B6818460C37BD465DF835
:10B06000047B70473C1300205813002080B584B047
:10B0700000AF78607B68BB600023FB607B68002BBF
:10B0800051D0BB68DA6A2A4B1B68DB6A9A4241D20C
:10B09000BB689B69002B06DB254B1B68DB6AC3F191
:10B0A0000602BB689A61BB685969BB68DA6A1346D5
:10B0B0009B0013449B001F4A1344994222D1BB6852
:10B0C0000433184605F0C3FA194B1B68DA6ABB68EB
:10B0D000DA62BB68DA6A184B1B689A4203D9BB680C
:10B0E000DB6A154A1360BB68DA6A13469B00134497
:10B0F0009B00104A1A44BB6804331946104605F0F9
:10B1000049FA04E00A4B1B68DA6ABB68DA62012379
:10B11000FB6008E0BB68DA6C054B1B68DB6A9A428F
:10B1200001D20123FB60FB6818461037BD4680BD85
:10B1300044120020481200203813002080B584B04B
:10B1400000AF78607B68BB600023FB607B68002BEE
:10B150004AD0284B1B68BA689A4204D04FF050007E
:10B1600080F31188FEE7BB681B6D002B04D14FF004
:10B17000500080F31188FEE7BB681B6D5A1EBB6848
:10B180001A65BB68DA6ABB68DB6C9A422CD0BB6874
:10B190001B6D002B28D1BB680433184605F057FA05
:10B1A000BB68DA6CBB68DA62BB68DB6AC3F10602B3
:10B1B000BB689A617B68DA6A0F4B1B689A4203D9B5
:10B1C0007B68DB6A0C4A13607B68DA6A13469B0073
:10B1D00013449B00094A1A447B68043319461046FD
:10B1E00005F0D8F90123FB60FB6818461037BD460F
:10B1F00080BD00BF441200203813002048120020F8
:10B2000080B586B000AF786039607B683B61012310
:10B21000FB607B68002B5ED03B691B6D002B04D16B
:10B220004FF0500080F31188FEE73B69DB6C3A6811
:10B230009A4202D93B687B6102E03B69DB6C7B612F
:10B240003B69DB6A7A699A4245D03B691B6DFA68B3
:10B250009A4240D1224B1B683A699A4204D14FF07E
:10B26000500080F31188FEE73B69DB6ABB603B69F5
:10B270007A69DA623B699B69002B04DB7B69C3F165
:10B2800006023B699A613B695969BA6813469B009B
:10B2900013449B00134A134499421CD13B69043365
:10B2A000184605F0D4F97B68DA6A0F4B1B689A429E
:10B2B00003D97B68DB6A0C4A13607B68DA6A134641
:10B2C0009B0013449B00074A1A447B6804331946C9
:10B2D000104605F05FF900BF1837BD4680BD00BFBE
:10B2E00044120020481200203813002080B400AF20
:10B2F000074B1B68002B04D0054B1B681A6D0132ED
:10B300001A65034B1B681846BD465DF8047B704701
:10B310004412002080B584B000AF78603960244BBF
:10B320001B68FB60234B1B68002283F85D20214BC8
:10B330001B680433184605F08AF97B68B3F1FF3FB8
:10B340000AD13B68002B07D01A4B1B6804331946FF
:10B35000194805F01FF926E0FA687B681344BB60C2
:10B36000144B1B68BA685A60BA68FB689A4209D2E3
:10B37000124B1A680F4B1B6804331946104605F030
:10B380002DF910E00E4B1A680A4B1B68043319465E
:10B39000104605F023F90B4B1B68BA689A4202D29B
:10B3A000084ABB68136000BF1037BD4680BD00BFB0
:10B3B00034130020441200201C130020EC12002043
:10B3C000E81200205013002080B584B000AF7860F0
:10B3D00039600623FB600023BB60FFF7BFF9FB6801
:10B3E000013BFB60FA6813469B0013449B00184A1C
:10B3F000981807F108033A68796806F080FAFB6844
:10B40000002BECD1134B186807F108033A687968F0
:10B4100006F075FA104B186807F108033A68796866
:10B4200006F06DFA07F108033A6879680B4806F0F0
:10B4300066FA07F108033A687968094806F05FFA86
:10B44000FFF79AF9BB6818461037BD4680BD00BFAC
:10B4500048120020E8120020EC1200201C130020EB
:10B460000413002080B586B000AFF860B9607A6040
:10B470003B60FEF7F7FEFB68002B02D10C4B1B680C
:10B4800000E0FB687B617B691A6CBB681A607B69B2
:10B490001A6B7B681A607B691A683B681A603B6AA2
:10B4A00000221A70FEF704FF00BF1837BD4680BDAA
:10B4B0004412002080B584B002AF00237B6000F00E
:10B4C000ADFA0E4B1B68002B0AD00D4B01930523E0
:10B4D00000930023C8220B490B4806F009F9786055
:10B4E0007B68002B04D14FF0500080F31188FEE7F9
:10B4F0007B6818460837BD4680BD00BF9413002006
:10B5000098130020FC450100A319010080B58AB002
:10B5100000AFF860B9607A603B6000237B62FB6833
:10B52000002B04D14FF0500080F31188FEE71A4B36
:10B530001B68002B2AD0BB687B617B68BB61FB6802
:10B54000FB61BB68052B18DCFFF772FD0346022B7D
:10B5500009D1114B186807F1140100233A6B05F06B
:10B56000F4F9786212E00C4B186807F1140100231B
:10B57000002205F0EAF9786208E0074B186807F145
:10B58000140100233A6805F0C8FA78627B6A18460D
:10B590002837BD4680BD00BF9413002080B586B01B
:10B5A00002AF786039601F4B1B68DB68DB68FB60AB
:10B5B000FB680433184605F04AF8FB6893F8283016
:10B5C00003F00403002B1CD0FB689A697B68D11838
:10B5D0007B683A68F86800F0B1F80346002B19D090
:10B5E0000023009300237A680021F868FFF78EFF9C
:10B5F000B860BB68002B0DD14FF0500080F311886C
:10B60000FEE7FB6893F8283023F00103DAB2FB6809
:10B6100083F82820FB681B6AF868984700BF10373A
:10B62000BD4680BD8C13002080B584B000AF78602B
:10B630003960FFF793F807F10803184600F05EF849
:10B64000F860BB68002B2AD13B68002B0AD17A68CE
:10B65000FB689A4206D8FFF78FF8F9687868FFF719
:10B660009DFF1EE03B68002B08D0104B1B681B6839
:10B67000002B01D1012300E000233B600C4B186834
:10B680007A68FB68D31A3A68194605F0A7FFFFF7F6
:10B6900073F80346002B04D1FEF720FE01E0FFF70C
:10B6A0006BF800BF1037BD4680BD00BF901300206F
:10B6B0009413002080B485B000AF78600E4B1B68F7
:10B6C0001B68002B01D1012200E000227B681A6078
:10B6D0007B681B68002B05D1074B1B68DB681B6868
:10B6E000FB6001E00023FB60FB6818461437BD4691
:10B6F0005DF8047B704700BF8C13002080B584B0D8
:10B7000000AF7860FFF7C8F8F8600B4B1B68FA6869
:10B710009A4205D200F024F97B6801221A6002E007
:10B720007B6800221A60044AFB681360FB681846B5
:10B730001037BD4680BD00BF9C13002080B586B089
:10B7400000AFF860B9607A603B6000237B61FB6802
:10B75000BA685A60FB68FA681A61BA687B689A42EC
:10B7600012D87A683B68D21AFB689B699A4202D366
:10B7700001237B611BE0104B1A68FB6804331946F8
:10B78000104604F02BFF12E07A683B689A4206D21A
:10B79000BA683B689A4202D301237B6107E0074BFA
:10B7A0001A68FB6804331946104604F017FF7B69DA
:10B7B00018461837BD4680BD901300208C1300201A
:10B7C00080B58CB002AFB8E0BB68002B13DA07F18C
:10B7D000080304337B627B6A002B04D14FF05000D6
:10B7E00080F31188FEE77B6A1B687A6A50687A6A80
:10B7F000926811469847BB68002BC0F29D803B6958
:10B800003B623B6A5B69002B04D03B6A04331846F9
:10B8100004F01DFF3B1D1846FFF770FFF861BB6881
:10B82000092B00F28A8001A252F823F055B80000DB
:10B8300055B8000055B80000BDB80000D1B80000F0
:10B840000FB9000055B8000055B80000BDB80000A1
:10B85000D1B800003B6A93F8283043F00103DAB214
:10B860003B6A83F82820FA683B6A9B69D118FB6819
:10B87000FA69386AFFF762FF0346002B5DD03B6A26
:10B880001B6A386A98473B6A93F8283003F0040330
:10B89000002B52D0FA683B6A9B691A44002300933C
:10B8A00000230021386AFFF731FEB861BB69002B25
:10B8B00043D14FF0500080F31188FEE73B6A93F8C4
:10B8C000283023F00103DAB23B6A83F8282034E001
:10B8D0003B6A93F8283043F00103DAB23B6A83F8FD
:10B8E0002820FA683B6A9A613B6A9B69002B04D165
:10B8F0004FF0500080F31188FEE73B6A9A69FB69BC
:10B90000D118FB69FA69386AFFF718FF15E03B6A3E
:10B9100093F8283003F00203002B03D1386AFEF7B6
:10B92000C7FA0AE03B6A93F8283023F00103DAB241
:10B930003B6A83F8282000E000BF084B1B6807F132
:10B9400008010022184605F00EFA0346002B7FF48A
:10B950003BAF00BF00BF2837BD4680BD9413002019
:10B9600080B588B002AF42E02A4B1B68DB681B68D9
:10B970003B61284B1B68DB68DB68FB60FB680433BA
:10B98000184604F064FEFB681B6AF8689847FB6879
:10B9900093F8283003F00403002B28D0FB689B6940
:10B9A0003A691344BB60BA683B699A420ED9FB6896
:10B9B000BA685A60FB68FA681A61164B1A68FB6825
:10B9C00004331946104604F009FE10E000230093EA
:10B9D00000233A690021F868FFF798FD78607B68DA
:10B9E000002B04D14FF0500080F31188FEE7094B83
:10B9F0001B681B68002BB7D1064B1B687B61064B8D
:10BA00001B68044A1360044A7B69136000BF18373F
:10BA1000BD4680BD8C1300209013002080B500AF80
:10BA2000FEF720FC124B1B68002B1DD1114804F0BF
:10BA300084FD114804F081FD104B0E4A1A60104B32
:10BA40000D4A1A60002210210A2004F084FE0346E9
:10BA5000074A1360064B1B68002B05D0044B1B687C
:10BA600008491846FEF7EAFCFEF722FC00BF80BD3D
:10BA70009413002064130020781300208C130020FE
:10BA8000901300200446010081F0004102E000BF55
:10BA900083F0004330B54FEA41044FEA430594EA8E
:10BAA000050F08BF90EA020F1FBF54EA000C55EAC9
:10BAB000020C7FEA645C7FEA655C00F0E2804FEA9A
:10BAC0005454D4EB5555B8BF6D420CDD2C4480EA7C
:10BAD000020281EA030382EA000083EA010180EAAC
:10BAE000020281EA0303362D88BF30BD11F0004FFA
:10BAF0004FEA01314FF4801C4CEA113102D0404230
:10BB000061EB410113F0004F4FEA03334CEA13336A
:10BB100002D0524263EB430394EA050F00F0A78082
:10BB2000A4F10104D5F1200E0DDB02FA0EFC22FA7D
:10BB300005F2801841F1000103FA0EF2801843FA71
:10BB400005F359410EE0A5F120050EF1200E012A62
:10BB500003FA0EFC28BF4CF0020C43FA05F3C018A0
:10BB600051EBE37101F0004507D54FF0000EDCF119
:10BB7000000C7EEB00006EEB0101B1F5801F1BD3C2
:10BB8000B1F5001F0CD349085FEA30004FEA3C0CC6
:10BB900004F101044FEA445212F5800F80F09A80BC
:10BBA000BCF1004F08BF5FEA500C50F1000041EBC0
:10BBB000045141EA050130BD5FEA4C0C404141EBC4
:10BBC0000101013C28BFB1F5801FE9D291F0000FBF
:10BBD00004BF01460020B1FA81F308BF2033A3F16E
:10BBE0000B03B3F120020CDA0C3208DD02F1140C65
:10BBF000C2F10C0201FA0CF021FA02F10CE002F1A0
:10BC00001402D8BFC2F1200C01FA02F120FA0CFC98
:10BC1000DCBF41EA0C019040E41AA2BF01EB0451E1
:10BC2000294330BD6FEA04041F3C1CDA0C340EDCDF
:10BC300004F11404C4F1200220FA04F001FA02F322
:10BC400040EA030021FA04F345EA030130BDC4F1E0
:10BC50000C04C4F1200220FA02F001FA04F340EAD5
:10BC60000300294630BD21FA04F0294630BD94F086
:10BC7000000F83F4801306BF81F480110134013D6D
:10BC80004EE77FEA645C18BF7FEA655C29D094EADE
:10BC9000050F08BF90EA020F05D054EA000C04BF5C
:10BCA0001946104630BD91EA030F1EBF0021002047
:10BCB00030BD5FEA545C05D14000494128BF41F0E6
:10BCC000004130BD14F580043CBF01F5801130BD4A
:10BCD00001F0004545F0FE4141F470014FF00000D5
:10BCE00030BD7FEA645C1ABF194610467FEA655C86
:10BCF0001CBF0B46024650EA013406BF52EA033528
:10BD000091EA030F41F4002130BD00BF90F0000F15
:10BD100004BF0021704730B54FF4806404F1320451
:10BD20004FF000054FF0000150E700BF90F0000F0A
:10BD300004BF0021704730B54FF4806404F1320431
:10BD400010F0004548BF40424FF000013EE700BF01
:10BD500042004FEAE2014FEA31014FEA02701FBF91
:10BD600012F07F4393F07F4F81F06051704732F0C3
:10BD70007F4208BF704793F07F4F04BF41F400211A
:10BD8000704730B54FF4607401F0004521F0004178
:10BD90001CE700BF50EA010208BF704730B54FF002
:10BDA00000050AE050EA010208BF704730B511F003
:10BDB000004502D5404261EB41014FF4806404F13B
:10BDC00032045FEA915C3FF4D8AE4FF003025FEAC1
:10BDD000DC0C18BF03325FEADC0C18BF033202EB45
:10BDE000DC02C2F1200300FA03FC20FA02F001FA9F
:10BDF00003FE40EA0E0021FA02F11444BDE600BF42
:10BE000070B54FF0FF0C4CF4E06C1CEA11541DBFF0
:10BE10001CEA135594EA0C0F95EA0C0F00F0DEF8BB
:10BE20002C4481EA030621EA4C5123EA4C5350EAA0
:10BE3000013518BF52EA033541F4801143F48013F1
:10BE400038D0A0FB02CE4FF00005E1FB02E506F082
:10BE50000042E0FB03E54FF00006E1FB03569CF0D7
:10BE6000000F18BF4EF0010EA4F1FF04B6F5007FDD
:10BE700064F5407404D25FEA4E0E6D4146EB06064F
:10BE800042EAC62141EA55514FEAC52040EA5E50D8
:10BE90004FEACE2EB4F1FD0C88BFBCF5E06F1ED882
:10BEA000BEF1004F08BF5FEA500E50F1000041EBB9
:10BEB000045170BD06F0004646EA010140EA020066
:10BEC00081EA0301B4EB5C04C2BFD4EB0C0541EA88
:10BED000045170BD41F480114FF0000E013C00F39D
:10BEE000AB8014F1360FDEBF002001F0004170BDC1
:10BEF000C4F10004203C35DA0C341BDC04F11404DA
:10BF0000C4F1200500FA05F320FA04F001FA05F265
:10BF100040EA020001F0004221F0004110EBD37032
:10BF200021FA04F642EB06015EEA430E08BF20EA5E
:10BF3000D37070BDC4F10C04C4F1200500FA04F301
:10BF400020FA05F001FA04F240EA020001F0004193
:10BF500010EBD37041F100015EEA430E08BF20EA06
:10BF6000D37070BDC4F1200500FA05F24EEA020E4E
:10BF700020FA04F301FA05F243EA020321FA04F07D
:10BF800001F0004121FA04F220EA020000EBD37034
:10BF90005EEA430E08BF20EAD37070BD94F0000F34
:10BFA0000FD101F00046400041EB010111F4801F68
:10BFB00008BF013CF7D041EA060195F0000F18BF19
:10BFC000704703F00046520043EB030313F4801F55
:10BFD00008BF013DF7D043EA0603704794EA0C0F0F
:10BFE0000CEA135518BF95EA0C0F0CD050EA410625
:10BFF00018BF52EA4306D1D181EA030101F00041A2
:10C000004FF0000070BD50EA410606BF10461946C9
:10C0100052EA430619D094EA0C0F02D150EA0136D5
:10C0200013D195EA0C0F05D152EA03361CBF104616
:10C0300019460AD181EA030101F0004141F0FE41B5
:10C0400041F470014FF0000070BD41F0FE4141F439
:10C05000780170BD70B54FF0FF0C4CF4E06C1CEA39
:10C0600011541DBF1CEA135594EA0C0F95EA0C0FEE
:10C0700000F0A7F8A4EB050481EA030E52EA0335A9
:10C080004FEA013100F088804FEA03334FF08055CA
:10C0900045EA131343EA12634FEA022245EA1115F7
:10C0A00045EA10654FEA00260EF000419D4208BFA8
:10C0B000964244F1FD0404F5407402D25B084FEA55
:10C0C0003202B61A65EB03055B084FEA32024FF401
:10C0D00080104FF4002CB6EB020E75EB030E22BF5E
:10C0E000B61A754640EA0C005B084FEA3202B6EB1E
:10C0F000020E75EB030E22BFB61A754640EA5C00CD
:10C100005B084FEA3202B6EB020E75EB030E22BF5C
:10C11000B61A754640EA9C005B084FEA3202B6EB5D
:10C12000020E75EB030E22BFB61A754640EADC001C
:10C1300055EA060E18D04FEA051545EA16754FEA7E
:10C1400006164FEAC30343EA52734FEAC2025FEA9C
:10C150001C1CC0D111F4801F0BD141EA00014FF02B
:10C1600000004FF0004CB6E711F4801F04BF0143FC
:10C170000020B4F1FD0C88BFBCF5E06F3FF6AFAE18
:10C18000B5EB030C04BFB6EB020C5FEA500C50F1A8
:10C19000000041EB045170BD0EF0004E4EEA11312B
:10C1A00014EB5C04C2BFD4EB0C0541EA045170BD32
:10C1B00041F480114FF0000E013C90E645EA060E76
:10C1C0008DE60CEA135594EA0C0F08BF95EA0C0FA4
:10C1D0003FF43BAF94EA0C0F0AD150EA01347FF4EC
:10C1E00034AF95EA0C0F7FF425AF104619462CE7C3
:10C1F00095EA0C0F06D152EA03353FF4FDAE104626
:10C20000194622E750EA410618BF52EA43067FF476
:10C21000C5AE50EA41047FF40DAF52EA43057FF406
:10C22000EBAE12E74FF0FF3C06E000BF4FF0010C11
:10C2300002E000BF4FF0010C4DF804CD4FEA410C75
:10C240007FEA6C5C4FEA430C18BF7FEA6C5C1BD042
:10C2500001B050EA410C0CBF52EA430C91EA030FC3
:10C2600002BF90EA020F0020704710F1000F91EA20
:10C27000030F58BF994208BF90422CBFD8176FEAEE
:10C28000E37040F0010070474FEA410C7FEA6C5CBC
:10C2900002D150EA013C07D14FEA430C7FEA6C5CC3
:10C2A000D6D152EA033CD3D05DF8040B704700BFEF
:10C2B0008446104662468C461946634600E000BF3D
:10C2C00001B5FFF7B7FF002848BF10F1000F01BD0F
:10C2D0004DF808EDFFF7F4FF0CBF012000205DF8DA
:10C2E00008FB00BF4DF808EDFFF7EAFF34BF01205F
:10C2F00000205DF808FB00BF4DF808EDFFF7E0FFF8
:10C3000094BF012000205DF808FB00BF4DF808ED48
:10C31000FFF7CEFF94BF012000205DF808FB00BFAF
:10C320004DF808EDFFF7C4FF34BF012000205DF891
:10C3300008FB00BF4FEA410212F5001215D211D5D9
:10C340006FF47873B3EB625212D94FEAC12343F012
:10C35000004343EA505311F0004F23FA02F018BF94
:10C36000404270474FF00000704750EA013005D15D
:10C3700011F0004008BF6FF0004070474FF0000020
:10C38000704700BF4A0011D212F5001211D20DD52C
:10C390006FF47873B3EB62520ED44FEAC12343F0CB
:10C3A000004343EA505323FA02F070474FF0000075
:10C3B000704750EA013002D14FF0FF3070474FF024
:10C3C00000007047024B0A460146186805F08FBB13
:10C3D00024000020014B1868704700BF2400002093
:10C3E0008A892DE9F041054610070C4658D44B6860
:10C3F000002B05DC0B6C002B02DC0020BDE8F0817B
:10C40000E66A002EF9D0002312F480522F682B60C8
:10C4100032D0606DA3895A0705D56368C01A636B73
:10C420000BB1236CC01A00230246E66A216A284633
:10C43000B047431CA38906D129681D292CD82A4A54
:10C44000CA40D60728D500226260D904226922603A
:10C4500004D5421C01D12B6803B96065616B2F6064
:10C460000029CAD004F14403994202D0284600F0C2
:10C4700089F900206063C1E7216A01232846B0479B
:10C48000411CC7D12B68002BC4D01D2B01D0162B0B
:10C4900001D12F60B1E7A38943F04003A381ADE749
:10C4A0000F69002FA9D093070E6808BF4B690F6072
:10C4B00018BF0023A6EB07088B60B8F1000F9CDDC6
:10C4C000216AA66A43463A462846B047002806DC59
:10C4D000A38943F04003A3814FF0FF308EE7074468
:10C4E000A8EB0008E9E700BF0100402038B50B6960
:10C4F00005460C4613B90025284638BD18B1836996
:10C500000BB900F071F8144B9C421BD16C68B4F964
:10C510000C30002BEFD0626ED00704D4990502D402
:10C52000A06D05F0A7FA28462146FFF759FF636E74
:10C53000DA070546E0D4A3899B05DDD4A06D05F09C
:10C540009AFAD9E7054B9C4201D1AC68DFE7044B6E
:10C550009C4208BFEC68DAE72C4601004C4601001B
:10C560000C460100002310B50446C0E90033C0E9C1
:10C570000433836081814366C28183611946082246
:10C580005C3005F0ACFA054B6362054BA362054BCA
:10C59000E362054B2462236310BD00BF471C01000A
:10C5A000691C0100A11C0100C51C0100014905F026
:10C5B00041BA00BFEDC40000014805F05BBA00BFFE
:10C5C000F0130020014805F056BA00BFF013002018
:10C5D000014805F04FBA00BFF1130020014805F0F3
:10C5E0004ABA00BFF113002010B50446FFF7F0FF70
:10C5F000A3691BB1BDE81040FFF7F0BFC4E91233D7
:10C600002365134B134A1B68A262A34204BF012394
:10C61000A361204600F020F86060204600F01CF87E
:10C62000A060204600F018F80022E0600421606855
:10C63000FFF798FFA06801220921FFF793FFE06848
:10C6400002221221FFF78EFF0123A361D2E700BF70
:10C650006C460100ADC50000F8B50746FFF7ACFF1A
:10C660001E4B1E68B36913B93046FFF7BDFF48364D
:10C67000D6E90134013B03D533680BB33668F7E7DD
:10C68000B4F90C50D5B9164BE36004F15800656657
:10C6900005F0EFF9FFF796FFC4E90155C4E9045529
:10C6A0002560A5610822294604F15C0005F017FA0F
:10C6B000C4E90D55C4E912552046F8BD6834D9E7E0
:10C6C0000421384605F0A0F9044630600028D5D191
:10C6D000FFF778FF0C233B60EEE700BF6C460100DC
:10C6E0000100FFFF8B8973B59D0706460C4607D5F1
:10C6F00004F14703236023610123636102B070BD2D
:10C7000001AB6A4605F0B8F900990546304600F0DD
:10C71000A5F848B9B4F90C309A05EFD423F0030317
:10C7200043F00203A381E3E70D4BB362A3892060CA
:10C7300043F08003A381009B6361019B20615BB197
:10C74000B4F90E10304600F0FBFC28B1A38923F0A9
:10C75000030343F00103A381A0890543A581CDE72D
:10C76000ADC50000024B0146186800F077B800BF65
:10C7700024000020024B0146186800F003B800BFF7
:10C780002400002037B5002944D051F8043C019022
:10C79000002BA1F10404B8BFE41800F0F3FC1E4A1A
:10C7A0000198136833B96360146003B0BDE830408A
:10C7B00000F0EEBCA34208D9256861198B4201BF85
:10C7C00019685B6849192160EDE71A465B680BB18F
:10C7D000A342FAD911685518A5420BD12468214407
:10C7E0005418A3421160E0D11C685B685360214477
:10C7F0001160DAE702D90C230360D6E725686119D6
:10C800008B4204BF19685B68636004BF49192160EB
:10C810005460CAE703B030BDA013002070B50E4EBF
:10C820000C463168054611B900F0FAFA306021462D
:10C83000284600F0F5FA431C0AD0C41C24F0030477
:10C84000A04207D0211A284600F0EAFA013001D1AF
:10C850004FF0FF34204670BDA41300202DE9F041B5
:10C86000CD1C25F0030508350C2D38BF0C25002DF7
:10C87000074601DBA94205D90C233B600026304660
:10C88000BDE8F0812E4E00F07DFC33681C4634BBC1
:10C8900029463846FFF7C2FF431C04464DD1346891
:10C8A0002646002E40D123683146384604EB030863
:10C8B00000F0B6FA80453AD1216803356D1A25F0AB
:10C8C000030508350C2D38BF0C2529463846FFF7DF
:10C8D000A5FF01302BD023682B4423600EE0226893
:10C8E000521B1ED40B2A16D96119A342256018BF0A
:10C8F0005960636808BF316062514B60384604F18B
:10C900000B0600F045FC26F00706231DF21AB6D0F0
:10C910009B1BA350B3E76268A3420CBF32605A600E
:10C92000ECE723466468B2E734467668B9E70C233F
:10C930003B60384600F02CFCA1E72560DEE700BF35
:10C94000A01300202DE9F04F0D469DB014469846E7
:10C95000064618B183690BB9FFF746FE894B9D4225
:10C960001BD175686B6ED90705D4AB899A0502D4C3
:10C97000A86D05F07FF8AB891B0701D52B69EBB9D2
:10C980002946304600F04CFBC0B16B6EDC070ED57B
:10C990004FF0FF301DB0BDE8F08F7B4B9D4201D1C1
:10C9A000B568DFE7794B9D4208BFF568DAE7AB89E8
:10C9B0009805EDD4A86D05F05EF8E9E7002309932A
:10C9C00020238DF82930CDF80C803023DFF8C0818A
:10C9D0008DF82A304FF0010923469A4613F8012BAF
:10C9E0000AB1252AF9D1BAEB040B0BD05B462246DB
:10C9F0002946304605F0A8F8013000F0AA80099ACF
:10CA00005A4409929AF80030002B00F0A2800023CB
:10CA10004FF0FF32CDE905230AF1010A0493079391
:10CA20008DF853301A935446052214F8011B5848C8
:10CA3000F3F7EEFC049AD8B9D10644BF20238DF851
:10CA40005330130744BF2B238DF853309AF800302E
:10CA50002A2B15D0079A544600204FF00A0C214685
:10CA600011F8013B303B092B4ED9B0B1079214E0CD
:10CA7000A0EB080309FA03F313430493A246D2E799
:10CA8000039B191D1B680391002BBBBF5B4242F047
:10CA9000020207930793B8BF049223782E2B0CD180
:10CAA00063782A2B35D1039B1A1D1B680392002B38
:10CAB000B8BF4FF0FF3302340593DFF8E4A02178CC
:10CAC00003225046F3F7A4FC40B14023A0EB0A0038
:10CAD00003FA00F0049B03430134049314F8011B90
:10CAE0002C488DF828100622F3F792FC00283FD03E
:10CAF000294B1BBB039B073323F007030833039326
:10CB0000099B3B44099367E70CFB02320C4601206A
:10CB1000A5E700230134059319464FF00A0C20467F
:10CB200010F8012B303A092A03D9002BC5D0059102
:10CB3000C3E70CFB012104460123F0E703AB00939C
:10CB40002A46164B04A93046AFF300800746781CEE
:10CB5000D6D16B6ED90705D4AB899A0502D4A86DDE
:10CB600004F089FFAB895B063FF512AF099811E726
:10CB700003AB00932A46094B04A9304600F012F893
:10CB8000E4E700BF2C4601004C4601000C460100C2
:10CB9000724701007C47010000000000491B0100B2
:10CBA000784701002DE9FF470F7E0C9D782F9146B5
:10CBB00080460C469A4601F1430207D8622F0AD8F4
:10CBC000002F00F0D880582F00F0A38004F1420518
:10CBD00084F842703AE0A7F16303152BF6D801A15F
:10CBE00051F823F03DCC000051CC0000CDCB00002B
:10CBF000CDCB0000CDCB0000CDCB000051CC000050
:10CC0000CDCB0000CDCB0000CDCB0000CDCB0000C4
:10CC10005DCD000081CC00003FCD0000CDCB0000F9
:10CC2000CDCB00007FCD0000CDCB000081CC00003B
:10CC3000CDCB0000CDCB000047CD00002B681A1DE6
:10CC40001B682A6004F1420584F842300123A3E006
:10CC500020682968060601F104030AD50E682B60D6
:10CC6000002E03DA2D23764284F843305E480A23EF
:10CC700019E00E682B6010F0400F18BF36B2EFE7D6
:10CC80002B682068191D2960010601D51E6802E085
:10CC90004606FBD51E8854486F2F0CBF08230A2375
:10CCA000002184F843106568A560002DA2BF2168AB
:10CCB00021F0040121600EB9002D4DD01546B6FBC0
:10CCC000F3F103FB1167C75D05F8017D3746BB42F1
:10CCD0000E46F4D9082B0BD12368DE0708D523694B
:10CCE00061689942DEBF302305F8013C05F1FF354C
:10CCF000521B2261CDF800A04B4603AA21464046B4
:10CD000004F034FF01304CD14FF0FF3004B0BDE8E7
:10CD1000F087354881F845702968236851F8046B1D
:10CD200029601D0614D5DF0744BF43F020032360AC
:10CD30001EB9236823F0200323601023B0E7236883
:10CD400043F0200323607823284884F84530E3E744
:10CD5000590648BFB6B2E6E71546BBE72B6826681A
:10CD60006169181D286035061B6801D5196002E04D
:10CD70007006FBD51980002323611546BAE72B689E
:10CD80001A1D2A601D68626800212846F3F740FBDF
:10CD900008B1401B606063682361002384F843305E
:10CDA000A8E723692A4649464046D0470130ABD020
:10CDB00023689B0713D4E068039B9842B8BF1846CA
:10CDC000A4E70123324649464046D04701309BD074
:10CDD0000135E36803995B1AAB42F2DCEBE700250F
:10CDE00004F11906F5E700BF8347010094470100ED
:10CDF0000FB40A4B13B51C6824B1A36913B92046BC
:10CE0000FFF7F2FB05AB049AA16801932046FFF7F8
:10CE100099FD02B0BDE8104004B070472400002026
:10CE200038B5064D0023044608462B6000F0C8F9CB
:10CE3000431C02D12B6803B1236038BDA813002026
:10CE4000012B2DE9F04701D0242B06D9FFF7C2FAB8
:10CE5000162303600020BDE8F087DFF8E4C00D462C
:10CE60002E4615F8014B14F80C7017F00807F7D18F
:10CE70002D2C32D12C780127B51C002B5BD0102B28
:10CE800009D1302C07D12C7804F0DF04582C4DD177
:10CE90006C781023023507F1004808F1FF384FF095
:10CEA000000CB8FBF3F9664603FB198AA4F1300EB7
:10CEB000BEF1090F16D87446A34224DDBCF1000F61
:10CEC0001EDBB1451CD301D1A24519DB06FB03468D
:10CED0004FF0010C15F8014BE8E72B2C04BF2C7820
:10CEE000B51CCAE7A4F1410EBEF1190F01D8373CB9
:10CEF000E2E7A4F1610EBEF1190F04D8573CDBE75D
:10CF00004FF0FF3CE6E7BCF1000F05DA2223036097
:10CF1000464642B930469EE707B17642002AF9D02C
:10CF2000BCF1000F00D0691E1160F3E73024002B24
:10CF3000B1D10823AFE7302CA5D00A23ABE700BF5F
:10CF40007246010013460A46014602480068FFF790
:10CF500077BF00BF24000020F8B50E4614460546F2
:10CF600018B183690BB9FFF73FFB214B9C422BD1D2
:10CF70006C68A369A360A3891A072FD523696BB3D3
:10CF800023692068C01A6369F6B28342374604DC1D
:10CF900021462846FFF7AAFA30BBA368013BA360ED
:10CFA00023685A1C22601E7063690130834204D0DA
:10CFB000A389DB0706D50A2E04D121462846FFF7B0
:10CFC00095FA88B93846F8BD0A4B9C4201D1AC6845
:10CFD000CFE7094B9C4208BFEC68CAE721462846C8
:10CFE00000F01EF80028CBD04FF0FF37EAE700BF73
:10CFF0002C4601004C4601000C46010038B5074D97
:10D0000004460846114600222A601A4604F039FFF9
:10D01000431C02D12B6803B1236038BDA813002044
:10D02000324B70B51D6806460C4625B1AB6913B985
:10D030002846FFF7D9FA2E4B9C420FD16C68A38982
:10D04000B4F90C2019072CD4DD0611D40923336060
:10D0500042F04003A3814FF0FF303EE0254B9C425D
:10D0600001D1AC68EBE7244B9C4208BFEC68E6E7D3
:10D07000580712D5616B41B104F14403994202D0C3
:10D080003046FFF77FFB00236363A38923F024036B
:10D09000A3810023636023692360A38943F008030D
:10D0A000A38123694BB9A38903F42073B3F5007FEF
:10D0B00003D021463046FFF715FBA089B4F90C20B8
:10D0C00010F001030AD00023A36063695B42A361EF
:10D0D000236943B910F08000BAD170BD810758BFF1
:10D0E0006369A360F4E70020F7E700BF2400002095
:10D0F0002C4601004C4601000C46010038B5064D97
:10D100000023044608462B6000F0E2F8431C02D1DD
:10D110002B6803B1236038BDA813002038B5074D34
:10D1200000230446084611462B6004F0FAFE431C17
:10D1300002D12B6803B1236038BD00BFA8130020C3
:10D1400038B5064D0023044608462B6004F0F7FE70
:10D15000431C02D12B6803B1236038BDA813002003
:10D1600038B5074D04460846114600222A601A4683
:10D1700004F075FE431C02D12B6803B1236038BD57
:10D18000A8130020014804F075BC00BFEF13002075
:10D19000014804F070BC00BFEF13002038B5074D04
:10D1A00004460846114600222A601A4604F000FE92
:10D1B000431C02D12B6803B1236038BDA8130020A3
:10D1C00070B50C4D2B680BB90B4B2B6003302E68E0
:10D1D00020F003043444204600F0A0F810B92C607D
:10D1E000304670BDFFF7F6F80C2303604FF0FF36B2
:10D1F000F6E700BFAC130020F41300202DE9FF4731
:10D20000DFF89490CDF804900327002303970124BE
:10D21000029301AE20463146ABBE0546DFF87C8066
:10D22000CDF8049004230397C8F8005002932046D9
:10D230003146ABBE8246144DCDF8049008230397C7
:10D24000C5F800A0029320463146ABBE04460F4904
:10D2500028680C60013404BF2B680B600C4B096814
:10D260004FF0FF329A611A62D8F800201A6000224B
:10D27000C3E90202C3E904125A60064B01221A6094
:10D2800004B0BDE8F08700BFBC130020B413002039
:10D29000C0130020B0130020A5470100B8130020E0
:10D2A000042810B5044601D9002010BD064B1B68A8
:10D2B0000BB9FFF7A3FF054850F834200132F3D033
:10D2C00000EBC400F1E700BFB0130020C013002042
:10D2D00038B50546FFF7E4FF044630B9FFF77AF8A2
:10D2E000092303604FF0FF3038BD013D012D09D8FF
:10D2F000094B9A681B699A4204D14FF0FF330360CF
:10D300000020F1E7206804F0DEFD0028ECD14FF0AA
:10D31000FF332360E8E700BFC0130020044B23B1B4
:10D32000984234BF0020012070471846704700BF64
:10D33000F423002008B5F2F772FF08BD08B5F2F734
:10D340006EFF08BD08B5F2F76AFF08BD08B5F2F731
:10D3500066FF08BD08B5F2F762FF08BD08B5F2F731
:10D360005EFF08BD08B5F2F75AFF08BD08B5F2F731
:10D3700056FF08BD08B5F2F752FF08BD08B5F2F731
:10D380004EFF08BD08B5F2F74AFF08BD08B5F2F731
:10D3900046FF08BD08B5F2F742FF08BD08B5F2F731
:10D3A0003EFF08BD08B5F2F73AFF08BD08B5F2F731
:10D3B00036FF08BD08B5F2F732FF08BD08B5F2F731
:10D3C0002EFF08BD08B5F2F72AFF08BD08B5F2F731
:10D3D00026FF08BD08B5F2F722FF08BD08B5F2F731
:10D3E0001EFF08BD08B5F2F71AFF08BD08B5F2F731
:10D3F00016FF08BD08B5F6F7A1FD08BD08B5F6F79C
:10D40000ABFD08BD08B5F6F747FA08BD08B5F6F755
:10D4100063FA08BD08B5F2F702FF08BD08B5F2F7D8
:10D42000FEFE08BD08B5F2F7FAFE08BD08B500F02B
:10D43000C0FF08BD08B5F2F7F2FE08BD08B500F060
:10D44000C1FF08BD08B5F2F7EAFE08BD08B5F2F75E
:10D45000E6FE08BD08B5F2F7E2FE08BD08B5F2F732
:10D46000DEFE08BD08B5F2F7DAFE08BD08B5F2F732
:10D47000D6FE08BD08B5F2F7D2FE08BD08B5F2F732
:10D48000CEFE08BD08B5F2F7CAFE08BD08B5F2F732
:10D49000C6FE08BD08B5F2F7C2FE08BD08B5F2F732
:10D4A000BEFE08BD08B5F2F7BAFE08BD08B5F2F732
:10D4B000B6FE08BD08B5F2F7B2FE08BD08B5F2F732
:10D4C000AEFE08BD08B5F2F7AAFE08BD08B5F2F732
:10D4D000A6FE08BD08B5F2F7A2FE08BD08B5F2F732
:10D4E0009EFE08BD08B5F2F79AFE08BD08B5F2F732
:10D4F00096FE08BD08B5F2F792FE08BD08B5F2F732
:10D500008EFE08BD08B5F2F78AFE08BD08B5F2F731
:10D5100086FE08BD08B5F2F782FE08BD08B5F2F731
:10D520007EFE08BD08B5F2F77AFE08BD08B5F2F731
:10D5300076FE08BD08B5F2F772FE08BD08B5F2F731
:10D540006EFE08BD08B5F2F76AFE08BD08B5F2F731
:10D5500066FE08BD08B5F2F762FE08BD08B5F2F731
:10D560005EFE08BD08B5F2F75AFE08BD08B5F2F731
:10D5700056FE08BD80B500AF0C20FFF7F3F8034658
:10D58000184680BD80B584B000AF786039607B6894
:10D59000FB600EE0FB681B683968184604F0A3FBCB
:10D5A0000346002B02D1FB685B6806E0FB689B68C2
:10D5B000FB60FB68002BEDD1002318461037BD46F9
:10D5C00080BD80B584B000AF786039607B681B682F
:10D5D000FB600023BB6031E0FB681B6839681846BC
:10D5E00004F081FB0346002B23D1FB689B68002BD2
:10D5F0000CD0BB68002B04D1FB689A687B681A606A
:10D600000EE0FB689A68BB689A6009E0BB68002B73
:10D6100003D0BB6800229A6002E07B6800221A6097
:10D62000FB681B681846FFF7A5F8F868FFF7A2F833
:10D6300007E0FB68BB60FB689B68FB60FB68002B36
:10D64000CAD11037BD4680BD80B586B000AFF86046
:10D65000B9607A60FB681B68002B03D0B968F86872
:10D66000FFF7AFFF0C20FFF77DF803467B61B8683A
:10D6700004F04BFB034601331846FFF773F80346EB
:10D680001A467B691A607B691B68B968184604F002
:10D6900034FB7B697A685A60FB681A687B699A6018
:10D6A000FB687A691A6000BF1837BD4680BD80B438
:10D6B00000AF00BFBD465DF8047B704780B400AF8B
:10D6C00000BFBD465DF8047B704780B400AF00BF6B
:10D6D000BD465DF8047B704780B485B000AF7860CC
:10D6E0007B681B0C03F1804303F58E23FB60FB6812
:10D6F00019687B689BB201229A40FB680A431A6052
:10D7000000BF1437BD465DF8047B704780B500AF9D
:10D7100001F00EF800F092F9F7F762FDF8F7E4FE79
:10D7200001F09FFA01F02EF801F0E9FB00F0CBFFC9
:10D7300000F0A4FFF9F7E0FE00F0FAFF00F0D1FFDF
:10D7400002F078F902F06FF9FFF7B8FF00BF80BD73
:10D7500080B582B000AF0023FB71FB1D1846F3F7C4
:10D760001FFC0346002B01D1FB7900E00023184683
:10D770000837BD4680BD80B483B000AF0346FB715F
:10D7800000BF0C37BD465DF8047B704780B483B0A2
:10D7900000AF78607B6800221A7000BF0C37BD466E
:10D7A0005DF8047B704780B400AF00231846BD4687
:10D7B0005DF8047B704780B485B000AF78600B469D
:10D7C000FB701346BB70BB78FB7300237B7327E0B1
:10D7D0007B7B7A6813441B783B730023BB7319E08F
:10D7E000FA7B3B7B5340DBB203F00103002B08D0F4
:10D7F000FB7B5B08FB73FB7B83F07303DB43FB73F7
:10D8000002E0FB7B5B08FB733B7B5B083B73BB7BF2
:10D810000133BB73BB7B072BE2D97B7B01337B736B
:10D820007A7BFB789A42D3D3FB7B18461437BD46EC
:10D830005DF8047B704790B585B000AF786000223A
:10D8400007217868FFF7B7FF0346FB737B6803F196
:10D8500009047B680933184604F057FA0346DBB223
:10D86000FA7B19462046FFF7A6FF0346FB73FB7BB6
:10D8700018461437BD4690BD80B487B000AFF8603D
:10D88000B9601346FB710023FB7504E0FB681B685D
:10D890005A1CFB681A60FB681B681B78202BF5D0AC
:10D8A000FB681B681B78FB754FE097F90730DBB20C
:10D8B000013BDBB2FB71FB7D392B09D8FB7D2F2BA4
:10D8C00006D9FA7DBB681A60BB680433BB6033E0DD
:10D8D000FB7D402B02D9FB7D5A2B05D9FB7D602BAC
:10D8E00015D9FB7D7A2B12D8FB7D602B08D9FB7DE7
:10D8F0007A2B05D8FB7DA3F12002BB681A6002E0F9
:10D90000FA7DBB681A60BB680433BB6014E0FB7D22
:10D91000212B08D0FB7D3F2B05D0FB7D3A2B02D07D
:10D92000FB7D202B06D1FA7DBB681A60BB680433EF
:10D93000BB6001E0022310E0FB681B685A1CFB6817
:10D940001A60FB681B681B78FB75FB7D002B03D0FE
:10D9500097F90730002BA8DC002318461C37BD467A
:10D960005DF8047B704780B487B000AFF8600B4669
:10D970007A60FB720023FB7545E0FB7D9B00FA6833
:10D9800013441B687F2B06DCFB7D9B00FA68134465
:10D990001B68002B01DA02233BE0FB7D9B00FA6849
:10D9A00013441B68DAB27B681A707B681B78002B03
:10D9B00001D100232DE07B681B78392B03D87B68CD
:10D9C0001B782F2B19D87B681B78402B03D97B68D9
:10D9D0001B785A2B11D97B681B78212B0DD07B68C3
:10D9E0001B783F2B09D07B681B783A2B05D07B68CE
:10D9F0001B78202B01D002230BE07B6801337B6076
:10DA0000FB7D0133FB75FA7D97F90B309A42B4DB4D
:10DA1000002318461C37BD465DF8047B704780B56F
:10DA200082B000AF786039603B685B6819467868FF
:10DA300000F0B5FE00BF0837BD4680BD80B400AF22
:10DA400000BFBD465DF8047B704780B483B000AF73
:10DA500078607B6801221A7500BF0C37BD465DF8FF
:10DA6000047B704780B582B000AF78607B689B68AC
:10DA7000184600F093FD034618460837BD4680BDA2
:10DA800080B582B000AF78607B685B68184601F0B3
:10DA90002AFA034618460837BD4680BD80B483B0D5
:10DAA00000AF78607B681B7D18460C37BD465DF87B
:10DAB000047B704780B582B000AF78607B68DB681C
:10DAC0001421184602F011FF0346012B01D0002358
:10DAD00000E0012318460837BD4680BD80B500AF81
:10DAE000F5F7A4FA0346184680BD80B582B000AFB2
:10DAF000F5F762FB3860F5F7FBFC0346DB083A6894
:10DB00009A4205D83B68002B02D03B687B6001E05D
:10DB100000237B607B6818460837BD4680BD80B512
:10DB200082B000AF03463A60FB710B46BB71B97916
:10DB3000FB793A681846F5F72DFE03461846083774
:10DB4000BD4680BD80B485B000AF78600023FB7314
:10DB50007B681B68002B01DA0123FB73FB7B1846F3
:10DB60001437BD465DF8047B704780B483B000AFC6
:10DB700078607A6892F84C3043F0010382F84C30B8
:10DB80007A6892F84C3043F0020382F84C307B689C
:10DB90001022A3F860207B681322A3F862207B6820
:10DBA00000225A657B68082283F851207B68002296
:10DBB00083F850207B684FF48072A3F8522000BF96
:10DBC0000C37BD465DF8047B704780B487B000AF6A
:10DBD000F860B9607A60FB7066237B61FB78013B7B
:10DBE000DBB21A46BB681340002B07D1FB78013B20
:10DBF000DBB21A467B681340002B01D0652311E08D
:10DC0000FB689B68BA689A420BD3BA687B681A446F
:10DC1000FB689968FB68DB680B449A4201D80023D3
:10DC20007B617B6918461C37BD465DF8047B7047F5
:10DC300080B487B000AF786000237B617B683B6174
:10DC40003B6903F00303002B03D13B691B687B6135
:10DC500015E00023FB600FE03B691B781A46FB6868
:10DC6000DB0002FA03F37A6913437B613B690133FA
:10DC70003B61FB680133FB60FB68032BECD97B69DC
:10DC800018461C37BD465DF8047B704780B584B0EC
:10DC900000AF78607B68002B01D1042347E00023AC
:10DCA000FB7340E0FB7B7A68642101FB03F31344C0
:10DCB00000221A70FB7B7A68642101FB03F3134492
:10DCC0000133FA7B1A70FB7B642202FB03F37A6850
:10DCD0001344184600F0BFF8FB7B1946786800F043
:10DCE000E2F8FB7B7A68642101FB03F313441B79A0
:10DCF000C3F30013DBB2002B04D0FB7B194678681A
:10DD0000F6F764F8FB7B1946786800F051F9FB7B65
:10DD1000642202FB03F37A6813441846F5F7FCFD0E
:10DD2000FB7B0133FB73FB7B002BBBD0002318462E
:10DD30001037BD4680BD80B586B000AFF860B960D1
:10DD40007A603B6007F113037A68B968F86800F0FD
:10DD50007CF978617B69002B01D07B6917E0FB7C43
:10DD60001A46642302FB03F3FA681344B9681846A1
:10DD700000F0B3F9FB7C1A46642302FB03F3FA6854
:10DD8000D0183B687A68B968F5F7E8FD034618468D
:10DD90001837BD4680BD80B586B000AFF860B96069
:10DDA0007A603B6007F113033A68B968F86800F0DD
:10DDB0004CF978617B69002B01D07B6917E0FB7C13
:10DDC0001A46642302FB03F3FA681344B968184641
:10DDD00000F083F9FB7C1A46642302FB03F3FA6824
:10DDE000D0183B687A68B968F5F718FE03461846FC
:10DDF0001837BD4680BD80B586B000AFF860B96009
:10DE00007A60FB7007F113037A68B968F86800F06C
:10DE10001CF978617B69002B01D07B6917E0FB7CE2
:10DE20001A46642302FB03F3FA681344B9681846E0
:10DE300000F053F9FB7C1A46642302FB03F3FA68F3
:10DE4000D018FB787A68B968F5F752FE0346184691
:10DE50001837BD4680BD80B483B000AF78607A6863
:10DE6000137943F0010313717A68137943F00203C5
:10DE700013717A68137943F0080313717A68137980
:10DE800043F0200313717A68137943F0040313718C
:10DE90007A68137943F01003137100BF0C37BD4645
:10DEA0005DF8047B704790B58DB000AF78600B468D
:10DEB000FB700023FB624FF48023BB6202237B6272
:10DEC0004FF400633B620423FB610823BB6108231A
:10DED0007B614FF070633B611823FB60FB787A68CD
:10DEE000642101FB03F313440833FA6A1A60FB78D8
:10DEF0007A68642101FB03F3134414337A6A1A60CD
:10DF0000FB787A68642101FB03F3134410333A6A07
:10DF10001A60FC78FB683A69B96A786AF5F77EFF9F
:10DF200001467A68642304FB03F313440C3319603D
:10DF3000FB78FA69D0B27A68642101FB03F31344D9
:10DF4000393302461A70FB78BA69D0B27A68642114
:10DF500001FB03F31344343302461A70FB787A69E9
:10DF6000D0B27A68642101FB03F3134435330246CF
:10DF70001A70FB787A68642101FB03F3134436338B
:10DF800004221A70FB787A68642101FB03F31344BE
:10DF9000373304221A70FB787A68642101FB03F39B
:10DFA0001344383300221A7000BF3437BD4690BD89
:10DFB00080B584B000AF78600B46FB702023FB6017
:10DFC000FB78642202FB03F320337A6813440433A2
:10DFD000BB60FB787A68642101FB03F313440833C8
:10DFE0001A68BB681A60BB68FA689A60FB787A683E
:10DFF000642101FB03F313440C331A68BB689B686C
:10E000001946104600F007F80246BB685A6000BF88
:10E010001037BD4680BD80B485B000AF78603960F0
:10E020003B689B027A689A4205D97A683B68B2FBE2
:10E03000F3F3FB6002E04FF48063FB60FB6818467B
:10E040001437BD465DF8047B704790B486B000AFCE
:10E05000F860B9607A603B60FB68002B01D1042353
:10E0600036E00023FB752FE0FB7DFA68642101FB9D
:10E0700003F3134408331B68BA689A4221D3BA6881
:10E080007B681A44FB7DF968642000FB03F30B44B2
:10E0900008331968FB7DF868642404FB03F3034428
:10E0A0000C331B680B449A420BD8FB7DFA68642141
:10E0B00001FB03F3134401331A783B681A70002301
:10E0C00006E0FB7D0133FB75FB7D002BCCD0662386
:10E0D00018461837BD4690BC704780B483B000AF77
:10E0E000786039607B683A681A6300BF0C37BD46B8
:10E0F0005DF8047B704780B485B000AFF860B9600C
:10E100001346FB71FB79002B05D10122BB689A40B5
:10E11000FB689A6004E00122BB689A40FB685A6081
:10E1200000BF1437BD465DF8047B704780B485B0EE
:10E1300000AF78607B681B0C03F1804303F58E23EE
:10E14000FB60FB6819687B689BB201229A40FB6800
:10E150000A431A6000BF1437BD465DF8047B704760
:10E1600080B485B000AF78607B685B78FB73FB7B25
:10E1700023F06003FB737B68FA7B5A700023184618
:10E180001437BD465DF8047B704780B485B000AF9E
:10E1900078607B685B78FB73FB7B23F06003FB7329
:10E1A000FB7B43F06003FB737B68FA7B5A700023B0
:10E1B00018461437BD465DF8047B704780B485B0BF
:10E1C00000AF78607B681B0C03F1804303F58E235E
:10E1D000FB60FB6819687B689BB201229A40FB6870
:10E1E0000A431A6000BF1437BD465DF8047B7047D0
:10E1F00080B485B000AF78607B681B79DBB2FB60D0
:10E200007B685B79DBB21B02FA681343FB607B68B7
:10E210001B7BDBB21B04FA681343FB607B689B7CAF
:10E22000DBB21B06FA681343FB60FB681846143721
:10E23000BD465DF8047B704780B584B000AF786060
:10E2400039607B685B79FB72FB7A03F03F03FB72FA
:10E250003B681B0ADAB2FB7A1343DAB27B685A7165
:10E260003B681B0EDAB27B689A743B6803F01F03AD
:10E27000002B0ED07B681B797B68DB797B680122E1
:10E280009A747B685B7CDBB243F04003DAB27B6854
:10E290005A747868FFF7ACFF02463B681340002BC6
:10E2A00003D040F2EE33FB6001E00023FB60FB682B
:10E2B00018461037BD4680BD80B485B000AFF86009
:10E2C000B9607A600CE000BFFB681B79DBB25BB21F
:10E2D000002BF9DABB685A1CBA601A78FB68DA714D
:10E2E0007B685A1E7A60002BEDD100BFFB681B795A
:10E2F000DBB203F04003002BF8D00023184614379C
:10E30000BD465DF8047B704780B485B000AF78608F
:10E310000B46FB700023FB730023BB737B689B7C65
:10E32000FB737B68DB78DBB203F00C03BB73FB7B16
:10E3300003F04003002B35D07B68DB78DBB223F0A1
:10E340000C03DAB27B68DA707B685B7CDBB263F06B
:10E350003F03DAB27B685A74FB78002B08D07B68E5
:10E360001B7CDBB243F00803DAB27B681A7407E067
:10E370007B681B7CDBB223F00803DAB27B681A747B
:10E380007B685B7CDBB263F03F03DAB27B685A7474
:10E390007B68DB78DAB2BB7B1343DAB27B68DA7076
:10E3A000002300E0012318461437BD465DF8047BC6
:10E3B000704780B500AFF6F74DFABFF34F8F00BF3F
:10E3C00000BF80BD80B500AFF6F758FABFF34F8F9E
:10E3D00000BF00BF80BD80B400AF00BFBD465DF888
:10E3E000047B704780B400AF00BFBD465DF8047B7E
:10E3F000704780B483B000AF47F230537B6000E0D9
:10E4000000BF7B685A1E7A60002BF9D100BF00BFA5
:10E410000C37BD465DF8047B704780B500AFF6F75A
:10E420008DFA00BF80BD80B400AF00BFBD465DF86F
:10E43000047B704780B500AFFFF7F5FF00BF80BDDC
:10E4400080B485B000AF78607B681B0C03F180431B
:10E4500003F58E23FB60FB6819687B689BB2012281
:10E460009A40FB680A431A6000BF1437BD465DF846
:10E47000047B704780B485B000AFF860B960134684
:10E48000FB71FB68BA6853F8223023F4E062FB7931
:10E490001B0203F4E06342EA0301FB68BA6843F835
:10E4A000221000BF1437BD465DF8047B704780B56D
:10E4B00000AFF6F765FA00BF80BD80B483B000AF4F
:10E4C000786039607B683A685A6000BF0C37BD4697
:10E4D0005DF8047B704780B483B000AF786039602A
:10E4E0007B683A689A6000BF0C37BD465DF8047BD4
:10E4F000704780B483B000AF786039607B681A6978
:10E500003B6822FA03F303F0010318460C37BD46BB
:10E510005DF8047B704780B485B000AFF860B960E7
:10E520001346FB71FB68BA6853F8223023F4E062AB
:10E53000FB791B0203F4E06342EA0301FB68BA685B
:10E5400043F8221000BF1437BD465DF8047B7047C6
:10E5500080B584B000AF78600B46FB701346BB708B
:10E5600007F10C0302220021184603F0B8FAFB78E9
:10E57000002B02D000233B7301E001233B73BB78E7
:10E580007B737B6858687B68DB6807F10C0219466F
:10E59000F5F770FC00BF1037BD4680BD80B582B076
:10E5A00000AF78607868F6F7D5FA0346002B14BF01
:10E5B00001230023DBB283F00103DBB203F001038C
:10E5C000DBB218460837BD4680BD80B485B000AFC9
:10E5D00078600B46FB707B68FB60FB68FA781A7406
:10E5E000FB78002B12D1FB689B68FA68D26853F85D
:10E5F000223023F0807323F00303FA689268F968ED
:10E60000C96843F0030342F821302AE0FB78012B6C
:10E6100012D1FB689B68FA68D26853F8223023F065
:10E62000807323F00303FA689268F968C96843F0BD
:10E63000030342F8213014E0FB78022B11D1FB6870
:10E640009B68FA68D26853F8223023F0807323F075
:10E650000303FA689268F968C96843F0020342F854
:10E66000213000BF1437BD465DF8047B704780B48D
:10E6700000AF00BFBD465DF8047B704780B400AFBB
:10E6800000BFBD465DF8047B704704207146084218
:10E6900002D0EFF3098001E0EFF3088081690A8876
:10E6A0004BF6AB639A4201D0F6F77CBA0231816136
:10E6B00020210160704700BF80B400AF00BFBD469D
:10E6C0005DF8047B704780B400AF00BFBD465DF8C5
:10E6D000047B704780B400AF00BFBD465DF8047B8B
:10E6E000704780B400AF00BFBD465DF8047B704743
:10E6F00080B584B000AFF860B9607A6008E0FB686C
:10E700001A78BB68114678689847FB680133FB604C
:10E71000FB681B78002BF2D100BF00BF1037BD464D
:10E7200080BD80B500AF72B6FBF71EFD00BF80BD97
:10E7300080B400AF00BFBD465DF8047B704780B574
:10E7400000AFFBF7A3FA0346002B14BF01230023FD
:10E75000DBB2184680BD80B584B000AF786001F0B0
:10E760008AFEF860FB68B3F1FF3F03D17B680022AB
:10E770001A7003E0FB68DAB27B681A7000BF1037CA
:10E78000BD4680BD80B400AF00BFBD465DF8047BD0
:10E79000704780B500AF01F087FE00BF80BD80B537
:10E7A00082B000AF786039603B68002B0CD006E087
:10E7B0007B685A1C7A601A783B68104698477B68D9
:10E7C0001B78002BF4D100E000BF0837BD4680BDA8
:10E7D00080B586B000AF7860396007F10C037A68C5
:10E7E0000B211846F8F71EFD07F10C03396818468F
:10E7F000FFF7D5FF00BF1837BD4680BD80B485B098
:10E8000000AFB9607A603B600346FB733B6800224F
:10E810001A70002318461437BD465DF8047B704714
:10E8200080B586B000AFF860B9607A603B603B6845
:10E83000DB6898470346002B53D00023FB753B68E9
:10E840001B6807F1170210469847FB7D002B40D04C
:10E85000FB7D082B02D0FB7D7F2B0DD1BA68FB68B6
:10E860009A4235D9BB68013BBB60BB6800221A7075
:10E870007B6801337B602BE0F87DBA68FB68D31AB4
:10E880001A4607F11603F968FFF7B8FF0346002B95
:10E890000CD007E00023FB753B681B6807F11702EB
:10E8A00010469847FB7D002BF4D1C6E7FA7DBB6884
:10E8B0001A70BB680133BB607B68013B7B60FB7DEA
:10E8C0000D2B09D0FB7D0A2B06D07B68012B02D9CA
:10E8D000B3E700BF00E000BFBB6800221A7001234D
:10E8E00000E0002318461837BD4680BD80B586B0CD
:10E8F00000AFF860B9607A603B600023FB753B684D
:10E90000002B01D11B2317E07B68002B0FD11B23A9
:10E9100012E03B681B687A68B968F8689847034654
:10E92000002B01D01B23FB753B6804333B603B6825
:10E930001B68002BEDD1FB7D18461837BD4680BD06
:10E9400080B586B000AFF860B9607A60FB700023D4
:10E95000FB750023BB75BB68002B01D11B233CE07A
:10E96000FB681B78002B01D1002336E0FB681B7885
:10E97000232B0CBF01230023BB75BB7D002B02D0D2
:10E98000FB680133FB6000237B7507F115017B6891
:10E99000BA68F868FFF7AAFF0346FB757B7D83F032
:10E9A0000103DBB2002B02D1FB7D002B05D0B9683F
:10E9B000F868F7F78BFA1B23FB75BB7D83F0010327
:10E9C000DBB2002B08D0FB7883F00103DBB2002B15
:10E9D00002D0B868F7F7ECF9FB7D18461837BD464A
:10E9E00080BD80B586B000AFF860B9607A603B60EA
:10E9F0000023FB757B68002B01D11B235AE0F868CC
:10EA000003F083F93861FA683B69D118BA683B6949
:10EA1000D21A7B68F868FFF703FF0346002B48D043
:10EA2000F86803F072F938613B69002B01D11B23B0
:10EA300040E03B69012B0AD1FB681B780A2B03D00D
:10EA4000FB681B780D2B02D1FB6800221A70BB6893
:10EA5000013B3A699A420CD397F820303A687968BA
:10EA6000F868FFF76DFFFB6800221A700423FB753E
:10EA70001FE03B69013BFA6813441B780A2B06D060
:10EA80003B69013BFA6813441B780D2B11D13B699C
:10EA9000013BFA68134400221A7097F820303A6854
:10EAA0007968F868FFF74CFF0346FB75FB680022A6
:10EAB0001A70FB7D18461837BD4680BD80B586B0FC
:10EAC00000AFF860B9607A607B68002B01D11B232E
:10EAD00048E0F86803F019F97861FA687B69D118A1
:10EAE000BA687B69D21A7B68F868FFF799FE03461B
:10EAF000002B36D0F86803F008F978617B69002BA9
:10EB000001D11B232EE07B69012B0AD1FB681B7806
:10EB10000A2B03D0FB681B780D2B02D1FB68002267
:10EB20001A70BB68013B7A699A4204D3FB680022E1
:10EB30001A70042316E07B69013BFA6813441B78C2
:10EB40000A2B06D07B69013BFA6813441B780D2B16
:10EB500007D17B69013BFA68134400221A70002335
:10EB600000E0082318461837BD4680BD80B586B042
:10EB700002AFF860B9607A603B60002300933B68A5
:10EB80007A68B968F868FFF72CFF03461846103713
:10EB9000BD4680BD80B584B000AFF860B960114655
:10EBA0001A460B46FB711346BB71FB68002B18D04D
:10EBB00009E0FB685A1CFA601A78BB69104698474E
:10EBC000BB79013BBB71FB681B78002B09D0BB797B
:10EBD000002BEED105E0BB6920209847BB79013BB3
:10EBE000BB71BB79002BF6D1FA79BB691046984707
:10EBF000BB6920209847BB68002B03D0B969B8686F
:10EC0000FFF7CDFD00BF1037BD4680BD80B586B093
:10EC100002AFF860B9607A607B6800931A233B22E8
:10EC2000B968F868FFF7B6FF00BF1037BD4680BD72
:10EC300080B586B002AFF860B9607A607B680093F7
:10EC40000D233A22B968F868FFF7A4FF00BF103718
:10EC5000BD4680BD80B400AF00BFBD465DF8047BFB
:10EC6000704780B400AF00BFBD465DF8047B7047BD
:10EC700080B485B000AF78607B681B0C03F18043E3
:10EC800003F58E23FB60FB6819687B689BB2012249
:10EC90009A40FB680A431A6000BF1437BD465DF80E
:10ECA000047B704780B584B000AF0346FB7100233E
:10ECB000FB6097F9073013F1800F02D10123FB604D
:10ECC00004E097F907301846F7F77EFAFB68184614
:10ECD0001037BD4680BD80B483B000AF78607B68DC
:10ECE000DB68DBB218460C37BD465DF8047B704725
:10ECF00080B485B000AFF860B9601346FB71FB6863
:10ED0000BA6853F8223023F4E062FB791B0203F463
:10ED1000E06342EA0301FB68BA6843F8221000BFCF
:10ED20001437BD465DF8047B704780B500AF042002
:10ED3000F7F70AFB00BF80BD80B485B000AF7860F4
:10ED400039607B68FB60FB683A681A61FB680022E7
:10ED50001A75FB6800225A7500BF1437BD465DF86E
:10ED6000047B704780B584B000AF786039600023C1
:10ED7000FB600FE07A68FB6806339B001344586819
:10ED8000FB683A6813441B781946F5F7ADFEFB683B
:10ED90000133FB60FB68032BECDD00BF00BF1037C5
:10EDA000BD4680BD80B584B000AF78600B46FB7077
:10EDB0007B68FB60FB681B7D002B1AD0FB685B7DCA
:10EDC000002B07D0FB685B7D013BDAB2FB685A750C
:10EDD000002321E0FB681B7D013BDAB2FB681A755A
:10EDE000FB681B695B68FA68127D13441A78FB683C
:10EDF0005A75FB78002B04D001217868F7F75CFC8A
:10EE000003E000217868F7F757FCFB689B79002B3B
:10EE10000CBF01230023DBB218461037BD4680BD6E
:10EE200080B485B000AF78607B68FB60FB681B69CD
:10EE30001B78013BDAB2FB681A75FB681B695A68DC
:10EE4000FB681B691B78013B13441A78FB685A75F1
:10EE500000BF1437BD465DF8047B704780B485B0B1
:10EE600000AF78607B68FB60FB6800221A75FB6866
:10EE700000225A7500BF1437BD465DF8047B704709
:10EE800080B584B000AF78607B68FB60FB681B686E
:10EE90000133BB6001217868F7F70EFCFB681B7932
:10EEA000022B03D10220FBF785FB02E00420FBF7D5
:10EEB00081FBFB681B68BA689A42EBD100BF00BFB8
:10EEC0001037BD4680BD80B485B000AF7860396032
:10EED0007B68FB60FB683A681A6000BF1437BD4668
:10EEE0005DF8047B704780B483B000AF78607B68C6
:10EEF0001B6818460C37BD465DF8047B704780B42C
:10EF000000AF00BFBD465DF8047B704780B400AF22
:10EF100000BFBD465DF8047B704780B584B000AF8C
:10EF20000346FB710023FB6097F9073013F1800F54
:10EF300002D10123FB6004E097F907301846F7F788
:10EF400031FCFB6818461037BD4680BD80B483B0E5
:10EF500000AF78607B68DB79DBB218460C37BD46C2
:10EF60005DF8047B704780B582B000AF7860786848
:10EF700002F0CBFE034619467868F7F77DFC00BF28
:10EF80000837BD4680BD80B485B000AFF860B96079
:10EF90007A60BB68013BBB600AE07A68531C7B6007
:10EFA000FB68591CF96012781A70BB68013BBB60A2
:10EFB000BB68002B03D07B681B78002BEDD1FB686E
:10EFC00000221A7000BF1437BD465DF8047B7047FD
:10EFD00080B485B000AFF860B9607A60BB68013B6F
:10EFE000BB6005E0FB680133FB60BB68013BBB60B5
:10EFF000BB68002B0FD0FB681B78002BF2D10AE016
:10F000007A68531C7B60FB68591CF96012781A708F
:10F01000BB68013BBB60BB68002B03D07B681B78DF
:10F02000002BEDD1FB6800221A7000BF1437BD46DB
:10F030005DF8047B704780B485B000AFF860B960BC
:10F040001346FB71BB68013BBB6005E0FB68013305
:10F05000FB60BB68013BBB60BB68002B03D0FB6857
:10F060001B78002BF2D1BB68002B04D0FB685A1C24
:10F07000FA60FA791A70FB6800221A7000BF143720
:10F08000BD465DF8047B704780B584B000AFF86082
:10F09000B9601346FB71FB799BB21A46B968F868F0
:10F0A000F7F7AAFF00BF1037BD4680BD80B485B01A
:10F0B00000AF78600B46FB701346BB700023BB7338
:10F0C00005E097F90E30DBB20133DBB2BB7397F981
:10F0D0000E307A6813441B78002BF2D1BB78FB7397
:10F0E00097F90F2097F90E309A4231D097F90F20F7
:10F0F00097F90E309A422BDD15E097F90E307A68B9
:10F100001A4497F90F3079680B4412781A7097F9FE
:10F110000F30DBB2013BDBB2FB7397F90E30DBB291
:10F12000013BDBB2BB7397F90E30002BE5DA0BE045
:10F1300097F90F307A681344FA781A7097F90F30FC
:10F14000DBB2013BDBB2FB7397F90F30002BEFDA38
:10F1500000BF1437BD465DF8047B704780B584B0AE
:10F1600000AFF860B96011461A460B46FB801346A3
:10F170007B71FB881A46B968F868F7F73DFF3A7E5D
:10F180007B791946F868FFF791FF00BF1037BD463D
:10F1900080BD80B586B000AFF860B9601346FB71E2
:10F1A000FA7907F1140304211846FFF76DFF07F100
:10F1B00014031A46B968F868FFF70AFF00BF18374A
:10F1C000BD4680BD80B586B000AFF860B96013461B
:10F1D000FB80FA8807F1100306211846F7F70CFFA9
:10F1E00007F110031A46B968F868FFF7F1FE00BF8F
:10F1F0001837BD4680BD80B588B002AFF860B960F1
:10F2000011461A460B46FB8013467B717979FA88C2
:10F2100007F1100097F8203000930B46B968FFF70C
:10F220009DFF07F110031A46B968F868FFF7D0FE92
:10F2300000BF1837BD4680BD80B586B000AFF8600E
:10F24000B9601346FB710023BB75FB7903F00F0314
:10F25000FB75FB7D092B01D8302200E03722FB7DB6
:10F260001344DBB27B75FB791B09FB75FB7D092B16
:10F2700001D8302200E03722FB7D1344DBB23B751E
:10F2800007F114031A46B968F868FFF7A1FE00BF3A
:10F290001837BD4680BD80B586B000AFF860B96054
:10F2A0001346FB8000233B750323FB75FB88DBB211
:10F2B00003F00F03BB75BB7D092B01D8302100E0A3
:10F2C000372197F91730BA7D0A44D2B218333B443C
:10F2D00003F8082CFB881B09FB8097F91730DBB279
:10F2E000013BDBB2FB7597F91730002BDEDA07F133
:10F2F00010031A46B968F868FFF76AFE00BF1837AE
:10F30000BD4680BD80B588B000AFF860B9607A6056
:10F310000023BB760523FB777B68DBB203F00F038A
:10F32000BB77BB7F092B01D8302100E0372197F94B
:10F330001F30BA7F0A44D2B220333B4403F80C2C6E
:10F340007B681B097B6097F91F30DBB2013BDBB2A6
:10F35000FB7797F91F30002BDEDA07F114031A460A
:10F36000B968F868FFF734FE00BF2037BD4680BD9E
:10F3700080B588B000AFF860B9607A6000233B7751
:10F380000723FB777B68DBB203F00F03BB77BB7F00
:10F39000092B01D8302100E0372197F91F30BA7FBF
:10F3A0000A44D2B220333B4403F80C2C7B681B097F
:10F3B0007B6097F91F30DBB2013BDBB2FB7797F93B
:10F3C0001F30002BDEDA07F114031A46B968F8681B
:10F3D000FFF7FEFD00BF2037BD4680BD80B588B079
:10F3E00000AFF860B9607A6007F114037A680B2106
:10F3F0001846F7F717FF07F114031A46B968F868BB
:10F40000FFF7E6FD00BF2037BD4680BD80B485B064
:10F4100000AF7860396000237B723B6800221A607D
:10F4200004E07B681B685A1C7B681A607B681B6859
:10F430001B78202BF5D07B681B681B78FB72FB7A4E
:10F440002D2B0AD101237B727B681B685A1C7B68B9
:10F450001A607B681B681B78FB72FB7A302B38D1F3
:10F460007B681B685A1C7B681A607B681B681B786A
:10F47000FB72FB7A622B0DD0782B17D11023BB7255
:10F480007B681B685A1C7B681A607B681B681B784A
:10F49000FB7228E00223BB727B681B685A1C7B68E6
:10F4A0001A607B681B681B78FB721CE0FB7A202BC0
:10F4B00002D9FB7A2E2B01D1002351E0FB7A2F2BAE
:10F4C00002D9FB7A392B01D91B2349E00823BB72EF
:10F4D00009E0FB7A2F2B02D9FB7A392B01D91B23A8
:10F4E0003EE00A23BB720023FB6029E0FB7A602B1D
:10F4F00002D9FB7A203BFB72FB7A303BFB72FB7A32
:10F50000102B07D9FB7A073BFB72FB7A092B01D83A
:10F510001B2325E0FA7ABB7A9A4201D31B231FE012
:10F52000BB7AFA6803FB02F2FB7A1344FB607B6848
:10F530001B685A1C7B681A607B681B681B78FB720F
:10F54000FB7A202B02D9FB7A2E2BCFD17B7A002B92
:10F5500002D0FB685B42FB60FA683B681A600023DC
:10F5600018461437BD465DF8047B704780B483B0FD
:10F5700000AF0346FB71FB792F2B02D9FB79392BA6
:10F580000BD9FB79602B02D9FB79662B05D9FB7966
:10F59000402B04D9FB79462B01D8012300E000233E
:10F5A00003F00103DBB218460C37BD465DF8047B5F
:10F5B000704780B485B000AF786039607B681B68A5
:10F5C0001B78FB73FB7B2F2B0ED9FB7B392B0BD8C6
:10F5D000FB7B303BDAB23B681A707B681B685A1CB5
:10F5E0007B681A60002324E0FB7B602B0ED9FB7B39
:10F5F000662B0BD8FB7B573BDAB23B681A707B68F3
:10F600001B685A1C7B681A60002312E0FB7B402BAE
:10F610000ED9FB7B462B0BD8FB7B373BDAB23B6822
:10F620001A707B681B685A1C7B681A60002300E014
:10F630001B2318461437BD465DF8047B704780B520
:10F6400086B000AF786039600223FB757B681B6869
:10F650003B613B6800221A7002E03B6901333B6169
:10F660003B691B78202BF8D03B691B781846FFF7C5
:10F670007DFF034683F00103DBB2002B0DD01B237B
:10F680001DE03B681B781B01DAB2FB7B1344DAB246
:10F690003B681A70FB7D013BFB75FB7D002B0AD09C
:10F6A00007F10F0207F1100311461846FFF781FF1B
:10F6B0000346002BE5D03A697B681A6000231846A0
:10F6C0001837BD4680BD80B487B000AFF860B96020
:10F6D0007A60FB681B687B617B68012B01D11B236F
:10F6E00038E07B68013BBA68134400221A707B68DB
:10F6F000013B7B607B691B78222B01D01B2329E017
:10F700007B6901337B610AE07A69531C7B61BB68CA
:10F71000591CB96012781A707B68013B7B607B6969
:10F720001B78222B06D07B691B78002B02D07B68CC
:10F73000002BE9D17B691B78222B01D01B2309E028
:10F740007B6901337B61BB6800221A70FB687A69B0
:10F750001A60002318461C37BD465DF8047B7047CD
:10F7600080B586B000AFF860B9607A60FB700023A6
:10F770003B61BB68012B4AD9FB687B6105E07B6973
:10F7800001337B613B6901333B617B691B78002B53
:10F79000F5D1FA683B69D018BA683B69D31A7A6820
:10F7A0001946FFF715FCBA683B69D31ABB600AE03B
:10F7B0007B6901337B6197F82030013B87F820306B
:10F7C000BB68013BBB607B691B78002B14D097F8AA
:10F7D0002030002B10D0BB68012BE9D80CE07B69EE
:10F7E0005A1C7A61FA781A7097F82030013B87F832
:10F7F0002030BB68013BBB6097F82030002B02D063
:10F80000BB68012BEBD87B6900221A7000E000BFB7
:10F810001837BD4680BD80B584B000AFF860B960D0
:10F820007A60FB70FB78012B07D17B68DBB21A464C
:10F83000B968F868FFF700FD18E0FB78022B07D1E4
:10F840007B689BB21A46B968F868FFF724FD0DE0A3
:10F85000FB78032B05D17A68B968F868FFF752FD89
:10F8600004E07A68B968F868FFF782FD00BF1037D6
:10F87000BD4680BD80B483B000AF786004E07B6893
:10F880001B685A1C7B681A607B681B681B78202BDE
:10F89000F5D000BF00BF0C37BD465DF8047B704754
:10F8A00080B485B000AF78607B68FB6002E0FB68E5
:10F8B0000133FB60FB681B78002BF8D1FA687B688A
:10F8C000D31A18461437BD465DF8047B704780B5DF
:10F8D00088B000AFF860B9607A603B600023FB61DC
:10F8E0000023BB611BE0BB697A6813441B78FB757E
:10F8F000BB6A002B08D0FB7D602B05D9FB7D7A2BE2
:10F9000002D8FB7D203BFB75FA7DFB681146B86889
:10F910009847FB690133FB61BB690133BB61BA697D
:10F920003B689A42DFDBFB6918462037BD4680BD45
:10F9300080B586B000AFF860B9603B601346FB71DC
:10F9400000237B6107E0FA79FB681146B8689847A5
:10F950007B6901337B613B685A1E3A60002BF2DC05
:10F960007B6918461837BD4680BD80B483B000AFB0
:10F9700078603960012318460C37BD465DF8047B7A
:10F98000704780B485B000AF786039607B68FB60F9
:10F990000BE0FB681B78FF2B01D0002309E0FB681C
:10F9A0000133FB603B68013B3B603B68002BF0D1BF
:10F9B000012318461437BD465DF8047B704780B5B7
:10F9C00084B000AFF860B9607A607A68B968F868A6
:10F9D000F8F70EFA034618461037BD4680BD80B5CD
:10F9E00084B000AFF860B9607A603B60BB6839688A
:10F9F0001846FFF7BAFF034683F00103DBB2002B82
:10FA000006D03A68FF21786802F069F81B2306E007
:10FA1000BB683A681946786802F053F80023184624
:10FA20001037BD4680BD80B400AF00BFBD465DF855
:10FA3000047B704780B500AF00F0BBF800BF80BD0D
:10FA400080B500AF00F0BDF800BF80BD80B584B0C8
:10FA500000AF7860786802F058F9F860FB68002B16
:10FA600001D1002309E0FB68013B7A6813441B784D
:10FA70007E2B01D1012300E0002318461037BD463C
:10FA800080BD80B582B000AF78607B6800225A7379
:10FA90007B681B7B83F00103DBB2002B19D07B68F2
:10FAA0001B6804331846FFF7D1FF034683F00103B8
:10FAB000DBB2002B0DD07B681B684FF40062194647
:10FAC0004FF4FF20FFF77BFF0346002B01D00023FC
:10FAD00000E0012318460837BD4680BD80B586B0DA
:10FAE00000AFF860B9607A60FB6800221A707B682A
:10FAF0009A687B6859687B681B685B690B449A420B
:10FB000009D37B685A687B681B685B691A447B6809
:10FB10009A60002312E07B689B681B78FB757B680A
:10FB20009B685A1C7B689A60FB7D1A46B968F86826
:10FB3000FFF781FAFB7D0A2BD9D10123184618372C
:10FB4000BD4680BD80B483B000AF786039607B680B
:10FB50009A687B685B68D31A1A463B681A6001236F
:10FB600018460C37BD465DF8047B704780B483B0FF
:10FB700000AF786039607B685A683B681B681A443C
:10FB80007B689A607B689A687B681B6803F50063F2
:10FB90009A4207D37B681B6803F500627B689A6012
:10FBA000002300E0012318460C37BD465DF8047BB6
:10FBB000704780B400AF00231846BD465DF8047B53
:10FBC000704780B400AF00231846BD465DF8047B43
:10FBD0007047B0B485B000AFF860B9607A6017E0E4
:10FBE000FB685A1CFA601B781D46602D02DD7A2DD9
:10FBF00000DC203DBB685A1CBA601B781C46602C98
:10FC000002DD7A2C00DC203CA54201D02B1B0DE04C
:10FC10007B685A1E7A60002B07D0FB681B78002B8C
:10FC2000DED1BB681B78002BDAD1002318461437CD
:10FC3000BD46B0BC704780B483B000AF786002E0CE
:10FC40007B6801337B607B681B78002B03D07B686B
:10FC50001B78202BF4D97B6818460C37BD465DF81D
:10FC6000047B704780B483B000AF7860396002E0F5
:10FC70007B68013B7B607A683B689A4209D97B6864
:10FC8000013B1B78002B04D07B68013B1B78202BA9
:10FC9000EED97B6818460C37BD465DF8047B70478B
:10FCA00080B584B000AF78600021786802F00EF86B
:10FCB000034679681846FFF7D5FFF860FB68002215
:10FCC0001A707B6818461037BD4680BD80B487B077
:10FCD00000AFF860B9607A60FB70FB78012B04D14B
:10FCE0007B68022B01D80023FB70FB78022B6CD0C1
:10FCF000022B00F3A480002B02D0012B1FD09EE02A
:10FD000000237B610AE0BA687B691A44F9687B6961
:10FD10000B4412781A707B6901337B617B68013B6D
:10FD20007A699A4205D2BA687B6913441B78002B22
:10FD3000E9D1FA687B69134400221A707FE000233E
:10FD40007B617B695A1C7A61FA68134422221A701B
:10FD500000233B611FE0BA683B6913441B78222BE8
:10FD60000BD17B68033B7A699A4220D27B695A1C8B
:10FD70007A61FA6813445C221A70BA683B691A44C3
:10FD8000F9687B690B4412781A703B6901333B6157
:10FD90007B6901337B61BA683B6913441B78002B94
:10FDA00006D07B68023B7A699A42D4D300E000BF58
:10FDB0007B695A1C7A61FA68134422221A70FA6825
:10FDC0007B69134400221A7039E000233B613B69D0
:10FDD0007B6123E0BA683B6913441B78222B05D072
:10FDE000BA683B6913441B785C2B09D13B6901332A
:10FDF000BA6813441B78222B02D13B6901333B6163
:10FE0000BA683B691A44F9687B690B4412781A7026
:10FE10003B6901333B617B6901337B61BA683B69B4
:10FE200013441B78002B04D07B68013B7A699A420B
:10FE3000D0D3FA687B69134400221A7000BFFB68B4
:10FE400018461C37BD465DF8047B704780B584B00A
:10FE500000AF786039600023FB607B68BB6023E003
:10FE6000BB681B78222B10D1BB6801331B78222B77
:10FE700003D1BB680133BB6013E0FB68002B0CBFF0
:10FE800001230023DBB2FB600BE0BB681B785C2B1B
:10FE900007D1BB6801331B78222B02D1BB68013329
:10FEA000BB60BB680133BB60BB681B78002B0AD00A
:10FEB000BB681B783B2B03D0BB681B78232BCFD1AF
:10FEC000FB68002BCCD1BB6800221A707868FFF762
:10FED000E7FE3B6800221A707B681B78222B18D142
:10FEE0000021786801F0F2FEB860BB68002B10D0EA
:10FEF000BB68013B1B78222B0BD17B6801337B60F5
:10FF0000BB68013BBB60BB6800221A703B680222E1
:10FF10001A707B6818461037BD4680BD80B59AB010
:10FF200000AFF860B9607A603B60BB68002B04D01A
:10FF3000B86801F0EAFE034600E00023FB65FB6DB4
:10FF4000002B02DC3B68002B58DB4FF0FF333B6695
:10FF500007F11403FA6840211846FFF7BFFD034676
:10FF6000002B01D10023DAE007F114031846FFF754
:10FF700062FEB8655D21B86D01F0E3FE7866BB6D89
:10FF80001B785B2BE4D17B6E002BE1D0BB6D013382
:10FF90001846FFF750FEB865B96D786EFFF762FE40
:10FFA00078667A6EBB6DD31AFA6D9A420BD1BB6834
:10FFB000002B08D0FB6D1A46B968B86DFFF709FE33
:10FFC0000346002B06D03B6E01333B663A6E3B681E
:10FFD0009A42BDD13B68002B10DB3A6E3B689A42D7
:10FFE0000AD17B6E00221A70BA6F0023B96D786F48
:10FFF000FFF76CFE012392E0002390E07B68002B6A
:020000021000EC
:1000000004D0786801F081FE034600E00023FB6520
:100010004FF0FF333B66FB6F002B03D0F96FF8689E
:10002000FFF790FD07F11403FA6840211846FFF727
:1000300055FD0346002B09D007F114031846FFF7BE
:10004000FAFDB865BB6D1B785B2B01D1002366E020
:1000500007F114031846FFF7EEFDB8653D21B86DB2
:1000600001F034FE78667B6E002B04D13A21B86D26
:1000700001F02CFE7866BB6D1B783B2BCBD0BB6DA3
:100080001B78232BC7D07B6E002BC4D0FB6D002BBD
:1000900012D0B96D786EFFF7E5FD0246BB6DD31A3D
:1000A000FA6D9A4208D1FB6D1A467968B86DFFF770
:1000B00090FD0346002B06D03B6E01333B663A6E43
:1000C0003B6F9A42A7D13B6F002B13DB3A6E3B6F1D
:1000D0009A420DD17B6E00221A70B86DFFF7E0FDD9
:1000E000BA6F0023B96D786FFFF7F0FD012316E0BA
:1000F000002314E07B6E01331846FFF79CFDB865C2
:1001000007F157031946B86DFFF7A0FEB865BA6F3F
:1001100097F85730B96D786FFFF7D8FD012318466F
:100120006837BD4680BD80B586B000AFF860B96065
:100130007A607A680023B968F868FFF7C7FD002184
:10014000F86801F0C3FD78617B69013B7E221A707B
:1001500000BF1837BD4680BD80B485B000AF786061
:100160007B68FB6002E0FB680133FB60FB681B7887
:10017000002B0BD0FB681B78222B07D0FB681B7869
:100180003B2B03D0FB681B78232BECD1FB681B783F
:10019000002B08D1FA687B689A4206D9FB68013BBC
:1001A0001B78202B01D1012300E00023DBB218468D
:1001B0001437BD465DF8047B704780B586B000AF4C
:1001C000F860B9607A60F86801F09FFD03467B61D2
:1001D000BB681A687B6913447A689A4201DC002381
:1001E00006E0BB681A687B691A44BB681A60012381
:1001F00018461837BD4680BD80B584B000AFF860A2
:10020000B9607A603B60F868FFF73BFCB868FFF7BD
:1002100038FC402279683868FFF785FF79683868CC
:10022000F8F7EAFC012318461037BD4680BD80B5BB
:1002300086B000AF786000237B61786801F065FDCF
:100240000346013B3B6117E07B697A6813441B78E6
:10025000FB733B697A681A447B6979680B441278AE
:100260001A703B697A681344FA7B1A707B69013310
:100270007B613B69013B3B617A693B699A42E3DB05
:1002800000BF00BF1837BD4680BD80B58CB000AF41
:10029000F860B9607A603B6007F11003194678682E
:1002A000F9F75CFB07F110023B68B968F868F9F7E9
:1002B00035F8034618463037BD4680BD80B58AB054
:1002C00000AFF860B9607A6000233B62FB68DB68CE
:1002D000FB61FB681B69BB61BA69FB699A4205D97E
:1002E000BA69FB69D31A013B7B6207E0FB689A6835
:1002F000B969FB69CB1A1344013B7B62FB689A68BE
:10030000FB69D31A7A6A934228BF13467B627A6AE2
:100310007B68934228BF13467B62FB685A68FB697F
:1003200013447B617A6AB968786901F0CAFB3A6A5A
:100330007B6A13443B62BA687B6A1344BB607A6889
:100340007B6AD31A7B60FA697B6A1344FB61FB68A2
:100350009B68FA699A4201D10023FB61FB68FA6944
:10036000DA607B68002BB4D13B6A18462837BD465B
:1003700080BD80B588B000AFF860B9607A60FB6876
:10038000DB68FB61FB689A68FB69D31ABB61BA69D9
:100390007B689A420FD9FB685A68FB6913443B613A
:1003A0007A68B968386901F08CFBFA697B681A448D
:1003B000FB68DA601DE0BB697B61FB685A68FB691A
:1003C00013443B617A69B968386901F07AFB7A684D
:1003D000BB69D31A7B61FB685B683B61BA68BB6928
:1003E00013447A691946386901F06BFBFB687A6936
:1003F000DA6000BF2037BD4680BD80B487B000AF53
:1004000078607B681B693B617B68DB68FB603A69ED
:10041000FB689A4208D87B689A68FB68D21A3B69E5
:100420001344013B7B6104E03A69FB68D31A013B4A
:100430007B617B6918461C37BD465DF8047B7047BD
:1004400080B586B000AFF860B9607A60EFF31183D1
:100450004FF0500181F311887B617A68B968F868C0
:10046000F9F718FB38617B6983F311883B691846FB
:100470001837BD4680BD80B582B000AFFB1C01229D
:1004800019460020FFF7DCFF03467B607B68012BE9
:1004900002D1FB787B6002E04FF0FF337B607B682A
:1004A00018460837BD4680BD80B500AFF9F7A4FAFD
:1004B00000BF80BD80B485B000AFF860B9607A60DD
:1004C000FB68043BFB60FB684FF080721A60FB68BE
:1004D000043BFB60BA68FB681A60FB68043BFB6086
:1004E000FB6800221A60FB68143BFB607A68FB68BB
:1004F0001A60FB68043BFB60FB686FF002021A6045
:10050000FB68203BFB60FB6818461437BD465DF86E
:10051000047B704780B500AF4FF0500080F3118826
:10052000FAF706FA0346002B01D0F9F7D7FE4FF091
:10053000000080F3118800BF80BD80B483B000AF9D
:1005400078607B6803F108027B685A607B684FF033
:10055000FF329A607B6803F108027B68DA607B688F
:1005600003F108027B681A617B6800221A6000BFF1
:100570000C37BD465DF8047B704780B483B000AF94
:1005800078607B6800221A6100BF0C37BD465DF8B9
:10059000047B704780B485B000AF786039607B68B9
:1005A0005B68FB603B68FA685A60FB689A683B6866
:1005B0009A60FB689B683A685A60FB683A689A6080
:1005C0003B687A681A617B681B685A1C7B681A60F2
:1005D00000BF1437BD465DF8047B704780B485B01A
:1005E00000AF786039603B681B68BB60BB68B3F1E3
:1005F000FF3F03D17B681B69FB600CE07B6808331D
:10060000FB6002E0FB685B68FB60FB685B681B6883
:10061000BA689A42F6D2FB685A683B685A603B68EF
:100620005B683A689A603B68FA689A60FB683A6867
:100630005A603B687A681A617B681B685A1C7B6841
:100640001A6000BF1437BD465DF8047B704780B464
:1006500085B000AF78607B681B69FB607B685B6876
:100660007A6892689A607B689B687A6852685A6078
:10067000FB685B687A689A4203D17B689A68FB687A
:100680005A607B6800221A61FB681B685A1EFB686F
:100690001A60FB681B6818461437BD465DF8047B7A
:1006A000704780B584B000AF786039607B68FB60CC
:1006B000FB68002B04D14FF0500080F31188FEE757
:1006C000F9F7D0FDFB681A68FB68DB6BF968096C09
:1006D00001FB03F31A44FB689A60FB6800229A63EB
:1006E000FB681A68FB685A60FB681A68FB68DB6B7A
:1006F000013BF968096C01FB03F31A44FB68DA60FB
:10070000FB68FF2283F84420FB68FF2283F8452022
:100710003B68002B0ED1FB681B69002B14D0FB68D3
:1007200010331846FAF788FA0346002B0CD0F9F775
:10073000D5FD09E0FB6810331846FFF7FEFEFB68A5
:1007400024331846FFF7F9FEF9F7B2FD01231846E6
:100750001037BD4680BD80B58AB002AFF860B96081
:100760001346FB71FB68002B04D14FF0500080F35F
:100770001188FEE7FB68BA6802FB03F3FB61BB6804
:10078000002B06D0FA69BB68B2FBF3F3FA689A4211
:1007900001D1012300E00023002B04D14FF05000D1
:1007A00080F31188FEE7FB6954331846F9F7BCFA69
:1007B000B861BB69002B0DD0BB697B617B69543389
:1007C0007B61FA79BB69009313467A69B968F86866
:1007D00000F005F8BB6918462037BD4680BD80B5DE
:1007E00084B000AFF860B9607A60FB70BB68002B22
:1007F00003D1BB69BA691A6002E0BB697A681A6002
:10080000BB69FA68DA63BB69BA681A640121B8691E
:10081000FFF747FFBB69FA7883F85020BB690022D5
:100820009A6400BF1037BD4680BD80B582B000AF6E
:1008300078607B68002B0ED07B6800229A607B6812
:1008400000221A607B680022DA6000230022002167
:10085000786800F07AF800BF0837BD4680BD80B5E3
:1008600086B000AF0346FB7101237B6100233B612F
:10087000FB791A4639697869FFF76DFFF860F86807
:10088000FFF7D3FFFB6818461837BD4680BD90B50B
:1008900085B000AF78607B68BB60BB68002B04D17B
:1008A0004FF0500080F31188FEE7BB689C68FAF7B0
:1008B000AFFB03469C4211D1BB68DB685A1EBB6884
:1008C000DA60BB68DB68002B05D100230022002121
:1008D000B86800F03AF80123FB6001E00023FB60F8
:1008E000FB6818461437BD4690BD90B585B000AF83
:1008F000786039607B68BB60BB68002B04D14FF027
:10090000500080F31188FEE7BB689C68FAF780FB13
:1009100003469C4207D1BB68DB685A1CBB68DA609F
:100920000123FB600CE03968B86800F0DBFAF8607E
:10093000FB68002B04D0BB68DB685A1CBB68DA601C
:10094000FB6818461437BD4690BD80B58AB000AF2D
:10095000F860B9607A603B6000237B62FB683B62B1
:100960003B6A002B04D14FF0500080F31188FEE762
:10097000BB68002B03D13B6A1B6C002B01D1012308
:1009800000E00023002B04D14FF0500080F31188C9
:10099000FEE73B68022B03D13B6ADB6B012B01D1E5
:1009A000012300E00023002B04D14FF0500080F31E
:1009B0001188FEE7FAF73CFB0346002B02D17B6867
:1009C000002B01D1012300E00023002B04D14FF0C4
:1009D000500080F31188FEE7F9F744FC3B6A9A6BFC
:1009E0003B6ADB6B9A4202D33B68022B33D13B6AF2
:1009F0009B6BFB613A68B968386A00F0D2FCB86159
:100A00003B6A9B6C002B0ED03B68022B02D1FB692A
:100A1000002B1CD1386A00F015FE0346002B16D0BF
:100A2000F9F75CFC13E03B6A5B6A002B0AD03B6A77
:100A300024331846FAF700F90346002B07D0F9F7DC
:100A40004DFC04E0BB69002B01D0F9F747FCF9F736
:100A50002FFC01235DE07B68002B03D1F9F728FC14
:100A6000002356E07B6A002B06D107F110031846DD
:100A7000FAF740F901237B62F9F71AFCF9F76EFEE9
:100A8000F9F7F0FB3B6A93F844305BB2B3F1FF3FF8
:100A900003D13B6A002283F844203B6A93F8453037
:100AA0005BB2B3F1FF3F03D13B6A002283F84520DC
:100AB000F9F7FEFB3A1D07F1100311461846FAF745
:100AC0002FF90346002B1ED1386A00F06FFD034654
:100AD000002B12D03B6A10337A6811461846FAF799
:100AE00067F8386A00F0EDFCF9F746FE0346002B84
:100AF0007FF472AFF9F7F2FB6EE7386A00F0E1FCC1
:100B0000F9F73AFE68E7386A00F0DBFCF9F734FEE3
:100B1000002318462837BD4680BD80B58AB000AF97
:100B2000F860B9607A603B60FB683B623B6A002B0F
:100B300004D14FF0500080F31188FEE7BB68002B12
:100B400003D13B6A1B6C002B01D1012300E0002381
:100B5000002B04D14FF0500080F31188FEE73B6872
:100B6000022B03D13B6ADB6B012B01D1012300E097
:100B70000023002B04D14FF0500080F31188FEE7D2
:100B8000F9F728FC0023FB614FF0500080F3118837
:100B90003B6A9A6B3B6ADB6B9A4202D33B68022B3F
:100BA0004DD13B6A93F84530FB763B6A9B6B7B618A
:100BB0003A68B968386A00F0F4FB97F91B30B3F172
:100BC000FF3F29D13B6A9B6C002B12D03B68022B64
:100BD00002D17B69002B2FD1386A00F033FD034628
:100BE000002B29D07B68002B26D07B6801221A605D
:100BF00022E03B6A5B6A002B1ED03B6A2433184616
:100C0000FAF71AF80346002B16D07B68002B13D096
:100C10007B6801221A600FE097F91B307F2B04D10B
:100C20004FF0500080F31188FEE7FB7E0133DBB20A
:100C30005AB23B6A83F8452001237B6201E000231E
:100C40007B624FF0000080F311887B6A18462837DA
:100C5000BD4680BD80B588B000AF786039607B68E4
:100C6000BB61BB69002B04D14FF0500080F31188A9
:100C7000FEE7BB691B6C002B04D04FF0500080F3E3
:100C80001188FEE7BB691B68002B03D1BB699B6819
:100C9000002B01D1012300E00023002B04D14FF0F1
:100CA000500080F31188FEE7F9F794FB00237B6185
:100CB0004FF0500080F31188BB699B6B3B61BB69AF
:100CC000DB6B3A699A4243D2BB6993F84530FB73B8
:100CD0003B695A1CBB699A6397F90F30B3F1FF3F28
:100CE00023D1BB699B6C002B0CD0B86900F0AAFC27
:100CF0000346002B29D03B68002B26D03B680122FD
:100D00001A6022E0BB695B6A002B1ED0BB692433EA
:100D10001846F9F791FF0346002B16D03B68002BCD
:100D200013D03B6801221A600FE097F90F307F2B38
:100D300004D14FF0500080F31188FEE7FB7B0133B4
:100D4000DBB25AB2BB6983F845200123FB6101E0A5
:100D50000023FB614FF0000080F31188FB69184607
:100D60002037BD4680BD80B58AB000AFF860B9605D
:100D70007A6000237B62FB683B623B6A002B04D1F4
:100D80004FF0500080F31188FEE7BB68002B03D1C1
:100D90003B6A1B6C002B01D1012300E00023002BD8
:100DA00004D14FF0500080F31188FEE7FAF740F9C4
:100DB0000346002B02D17B68002B01D1012300E008
:100DC0000023002B04D14FF0500080F31188FEE780
:100DD000F9F748FA3B6A9B6BFB61FB69002B19D062
:100DE000B968386A00F047FBFB695A1E3B6A9A6390
:100DF0003B6A1B69002B09D03B6A10331846F9F790
:100E00001BFF0346002B01D0F9F768FAF9F750FAF7
:100E1000012363E07B68002B03D1F9F749FA002333
:100E20005CE07B6A002B06D107F114031846F9F742
:100E300061FF01237B62F9F73BFAF9F78FFCF9F7C1
:100E400011FA3B6A93F844305BB2B3F1FF3F03D130
:100E50003B6A002283F844203B6A93F845305BB23A
:100E6000B3F1FF3F03D13B6A002283F84520F9F735
:100E70001FFA3A1D07F1140311461846F9F750FFFF
:100E80000346002B1DD1386A00F07AFB0346002B85
:100E900011D03B6A24337A6811461846F9F788FE68
:100EA000386A00F00EFBF9F767FC0346002B8FD180
:100EB000F9F714FA8CE7386A00F003FBF9F75CFCE9
:100EC00086E7386A00F0FDFAF9F756FC386A00F058
:100ED00057FB0346002B3FF47BAF0023184628370F
:100EE000BD4680BD80B58AB000AF78603960002310
:100EF0007B627B68FB6100233B62FB69002B04D1B2
:100F00004FF0500080F31188FEE7FB691B6C002B4B
:100F100004D04FF0500080F31188FEE7FAF788F80C
:100F20000346002B02D13B68002B01D1012300E0D6
:100F30000023002B04D14FF0500080F31188FEE70E
:100F4000F9F790F9FB699B6BBB61BB69002B1ED065
:100F5000BB695A1EFB699A63FB691B68002B04D1AD
:100F6000FAF7C4F90246FB699A60FB691B69002B1A
:100F700009D0FB6910331846F9F75EFE0346002BD3
:100F800001D0F9F7ABF9F9F793F901238BE03B684E
:100F9000002B0BD13B6A002B04D04FF0500080F3A4
:100FA0001188FEE7F9F784F900237CE07B6A002BC7
:100FB00006D107F10C031846F9F79CFE01237B626A
:100FC000F9F776F9F9F7CAFBF9F74CF9FB6993F8E9
:100FD00044305BB2B3F1FF3F03D1FB69002283F8D9
:100FE0004420FB6993F845305BB2B3F1FF3F03D176
:100FF000FB69002283F84520F9F75AF93A4607F1D0
:101000000C0311461846F9F78BFE0346002B2CD132
:10101000F86900F0B5FA0346002B20D0FB691B6885
:10102000002B09D1F9F71EF9FB699B681846FAF7FE
:101030001DF83862F9F73CF9FB6924333A68114628
:101040001846F9F7B5FDF86900F03BFAF9F794FB9B
:101050000346002B7FF474AFF9F740F970E7F869A5
:1010600000F02FFAF9F788FB6AE7F86900F029FA2F
:10107000F9F782FBF86900F083FA0346002B3FF48E
:101080005FAF3B6A002B0DD0F9F7ECF8F86900F080
:1010900070F97861FB699B6879691846FAF7B0F8CE
:1010A000F9F706F9002318462837BD4680BD80B5FC
:1010B0008AB000AFF860B9607A6000237B62FB6899
:1010C0003B623B6A002B04D14FF0500080F3118843
:1010D000FEE7BB68002B03D13B6A1B6C002B01D1E0
:1010E000012300E00023002B04D14FF0500080F3D7
:1010F0001188FEE7F9F79CFF0346002B02D17B68BD
:10110000002B01D1012300E00023002B04D14FF07C
:10111000500080F31188FEE7F9F7A4F83B6A9B6B57
:10112000FB61FB69002B1BD03B6ADB68BB61B968C4
:10113000386A00F0A0F93B6ABA69DA603B6A5B6A18
:10114000002B09D03B6A24331846F9F775FD034696
:10115000002B01D0F9F7C2F8F9F7AAF8012363E0F0
:101160007B68002B03D1F9F7A3F800235CE07B6ACE
:10117000002B06D107F110031846F9F7BBFD012338
:101180007B62F9F795F8F9F7E9FAF9F76BF83B6A3A
:1011900093F844305BB2B3F1FF3F03D13B6A0022C6
:1011A00083F844203B6A93F845305BB2B3F1FF3FCC
:1011B00003D13B6A002283F84520F9F779F83A1DFC
:1011C00007F1100311461846F9F7AAFD0346002B54
:1011D0001DD1386A00F0D4F90346002B11D03B6AC8
:1011E00024337A6811461846F9F7E2FC386A00F0B1
:1011F00068F9F9F7C1FA0346002B8DD1F9F76EF8BB
:101200008AE7386A00F05DF9F9F7B6FA84E7386AD8
:1012100000F057F9F9F7B0FA386A00F0B1F903466F
:10122000002B3FF479AF002318462837BD4680BD18
:1012300080B58AB000AFF860B9607A60FB683B6245
:101240003B6A002B04D14FF0500080F31188FEE779
:10125000BB68002B03D13B6A1B6C002B01D101231F
:1012600000E00023002B04D14FF0500080F31188E0
:10127000FEE7F9F7AFF80023FB614FF0500080F371
:1012800011883B6A9B6BBB61BB69002B36D03B6A04
:1012900093F84430FB75B968386A00F0ECF8BB6924
:1012A0005A1E3B6A9A6397F91730B3F1FF3F12D188
:1012B0003B6A1B69002B1ED03B6A10331846F9F7B6
:1012C000BBFC0346002B16D07B68002B13D07B6839
:1012D00001221A600FE097F917307F2B04D14FF0ED
:1012E000500080F31188FEE7FB7D0133DBB25AB278
:1012F0003B6A83F8442001237B6201E000237B6288
:101300004FF0000080F311887B6A18462837BD46ED
:1013100080BD80B584B000AF78607B68002B04D1BD
:101320004FF0500080F31188FEE7F8F79BFF7B68D1
:101330009B6BFB60F8F7BCFFFB6818461037BD4697
:1013400080BD80B584B000AF78607B68FB60FB68CF
:10135000002B04D14FF0500080F31188FEE7F868AD
:10136000F9F796F8F868F8F7A3FD00BF1037BD4607
:1013700080BD80B485B000AF78607B685B6A002B6D
:1013800006D07B681B6B1B68C3F10603FB6001E0A2
:101390000023FB60FB6818461437BD465DF8047BEC
:1013A000704780B586B000AFF860B9607A600023FE
:1013B0007B61FB689B6B3B61FB681B6C002B0DD159
:1013C000FB681B68002B4DD1FB689B681846F9F73A
:1013D000B5FE7861FB6800229A6043E07B68002BD1
:1013E00019D1FB685868FB681B6C1A46B96800F095
:1013F00068FBFB685A68FB681B6C1A44FB685A6000
:10140000FB685A68FB689B689A422BD3FB681A6892
:10141000FB685A6026E0FB68D868FB681B6C1A46BC
:10142000B96800F04EFBFB68DA68FB681B6C5B4236
:101430001A44FB68DA60FB68DA68FB681B689A424A
:1014400007D2FB689A68FB681B6C5B421A44FB6816
:10145000DA607B68022B05D13B69002B02D03B6927
:10146000013B3B613B695A1CFB689A637B691846E8
:101470001837BD4680BD80B582B000AF7860396056
:101480007B681B6C002B18D07B68DA687B681B6C50
:101490001A447B68DA607B68DA687B689B689A42EA
:1014A00003D37B681A687B68DA607B68D9687B68DD
:1014B0001B6C1A46386800F004FB00BF0837BD46B5
:1014C00080BD80B584B000AF7860F8F7CBFE7B6854
:1014D00093F84530FB731EE07B689B6C002B08D0B3
:1014E000786800F0AFF80346002B10D0F9F782FCC3
:1014F0000DE07B685B6A002B12D07B6824331846B2
:10150000F9F79AFB0346002B01D0F9F773FCFB7B3C
:10151000013BDBB2FB7397F90F30002BDCDC00E002
:1015200000BF7B68FF2283F84520F8F7C1FEF8F77B
:1015300099FE7B6893F84430BB7311E07B681B69AC
:10154000002B12D07B6810331846F9F775FB034661
:10155000002B01D0F9F74EFCBB7B013BDBB2BB7328
:1015600097F90E30002BE9DC00E000BF7B68FF221A
:1015700083F84420F8F79CFE00BF1037BD4680BDBD
:1015800080B584B000AF7860F8F76CFE7B689B6B29
:10159000002B02D10123FB6001E00023FB60F8F780
:1015A00087FEFB6818461037BD4680BD80B584B005
:1015B00000AF7860F8F756FE7B689A6B7B68DB6B50
:1015C0009A4202D10123FB6001E00023FB60F8F79F
:1015D0006FFEFB6818461037BD4680BD80B586B0EB
:1015E00000AFF860B9607A60FB687B61F8F73AFE9B
:1015F0007B6993F844305BB2B3F1FF3F03D17B6961
:10160000002283F844207B6993F845305BB2B3F144
:10161000FF3F03D17B69002283F84520F8F748FE9D
:101620007B699B6B002B06D17B6924337A68B96890
:101630001846F9F7DBFA7869FFF743FF00BF183760
:10164000BD4680BD80B586B000AF78607B689B6C7E
:101650003B6100237B613B69002B04D14FF05000BC
:1016600080F31188FEE73B699A6B3B69DB6B9A421A
:1016700004D34FF0500080F31188FEE73B699A6B6A
:101680003B69DB6B9A422ED23B6993F84530FB7382
:101690003B1D002219463869FFF783FE786197F9F0
:1016A0000F30B3F1FF3F0ED13B695B6A002B1AD0BC
:1016B0003B6924331846F9F7BFFA0346002B12D0D2
:1016C00001237B610FE097F90F307F2B04D14FF09E
:1016D000500080F31188FEE7FB7B0133DBB25AB286
:1016E0003B6983F845207B6918461837BD4680BDA5
:1016F00080B58CB004AFF860B9603B601346FB80E6
:10170000FB889B001846F8F70FFB78617B69002B7C
:101710000ED06020F8F708FBF861FB69002B03D0BE
:10172000FB697A691A6305E07869F8F7C1FB01E0A3
:101730000023FB61FB69002B13D0FA88002303937D
:10174000FB690293FB6A0193BB6A00933B68B9682B
:10175000F86800F00EF8F869F8F7C4FE0123BB61E1
:1017600002E04FF0FF33BB61BB6918462037BD462E
:1017700080BD80B586B000AFF860B9607A603B602C
:10178000BB6A186B7B689B001A46A52100F0A7F97D
:10179000BB6A1A6B7B6803F18043013B9B001344D7
:1017A0003B613B6923F007033B613B6903F007039F
:1017B000002B04D04FF0500080F31188FEE7BB6A85
:1017C0003A691A64BB68002B1FD000237B6112E0CA
:1017D000BA687B6913441978BA6A7B691344343355
:1017E0000A461A70BA687B6913441B78002B06D02E
:1017F0007B6901337B617B690B2BE9D900E000BF7A
:10180000BB6A002283F83F2003E0BB6A002283F812
:1018100034203B6A052B01D905233B62BB6A3A6A37
:10182000DA62BB6A3A6ADA64BB6A00221A65BB6A8A
:1018300004331846FEF7A1FEBB6A18331846FEF7BC
:101840009CFEBB6ABA6A1A613B6AC3F10602BB6AB4
:101850009A61BB6ABA6A5A62BB6A00225A65BB6A5D
:10186000583304220021184600F039F9BB6A5C3372
:1018700001220021184600F032F9BB6A002283F8E9
:101880005D203A68F9683869FEF714FE0246BB6AC3
:101890001A607B6A002B02D07B6ABA6A1A6000BFAA
:1018A0001837BD4680BD80B485B000AF7860002396
:1018B000FB6005E07B6801337B60FB680133FB6004
:1018C0007B681B78A52BF5D0FB689B08FB60FB6849
:1018D0009BB218461437BD465DF8047B704780B54F
:1018E00082B000AF78607B681B6B1846F8F7E0FAAF
:1018F0007868F8F7DDFA00BF0837BD4680BD80B4D0
:1019000089B000AFF860B9607A603B60FB681B6823
:10191000002B40D0FB68FB61FB695B685A68FB6980
:101920005A60FB695A68FB6908339A4204D1FB6923
:101930005B685A68FB695A60FB695B68DB68BB617E
:10194000FB687B617B695B685A687B695A607B696D
:101950005A687B6908339A4204D17B695B685A688C
:101960007B695A607B695B68DB683B613B681B682D
:101970007A689A4206D93B681B689B00BA68134490
:101980003A691A603B681B685A1C3B681A603A69DE
:10199000BB699A42D4D100BF2437BD465DF8047BB1
:1019A000704780B584B000AF786007F1080318462F
:1019B000F9F780FEF860BB681946F868F9F734FE5D
:1019C000F9F7FEFEF1E780B483B000AF78603960CC
:1019D0004FF0500080F3118800BEFEE780B400AFE6
:1019E0004FF0500080F3118800BEFEE780B400AFD6
:1019F00000BFBD465DF8047B704780B400AF00BFF8
:101A0000BD465DF8047B704770B568224D1E554396
:101A10000E4605F17401FAF721FF044640B100219A
:101A2000C0E900160C30A06005F1680200F057F81C
:101A3000204670BD2DE9F8430646884600F148046B
:101A40000027D4E90195B9F1010905D52468002CD6
:101A5000F7D13846BDE8F883AB89012B07D9B5F932
:101A60000E30013303D029463046C047074368355E
:101A7000E9E770477047704770B50E46B1F90E1030
:101A8000002996B014461D4608DAB6F90C3000223B
:101A90002A601A0610D44FF480630EE06A46FBF702
:101AA0003DFB0028F1DB019A02F47042A2F50053DD
:101AB0005A425A412A60EEE740230020236016B0C4
:101AC00070BD0A44914200F1FF3300D1704710B558
:101AD00011F8014B03F8014F9142F9D110BD0244B6
:101AE0000346934200D1704703F8011BF9E737B56D
:101AF000A1FB02244CB911460192FAF7AFFE019AFC
:101B0000054630B9284603B030BD0C2202600025DE
:101B1000F8E72146FFF7E3FFF4E79368013B002B6A
:101B200010B4936008DA9469A34201DB0A2903D157
:101B30005DF8044BFBF710BA1368581C106019705D
:101B400008465DF8044B7047F8B506460F46144644
:101B5000D518AC4201D1002007E014F8011B3A4629
:101B60003046FFF7DAFF431CF3D1F8BD2DE9F0470B
:101B7000164699468A680B69DDF820809342B8BF03
:101B80001346336091F8432007460C460AB10133EF
:101B900033602368990642BF336802333360256897
:101BA00015F0060506D104F1190AE36832689B1A9C
:101BB000AB4226DC94F84320131E226818BF012391
:101BC00092062BD404F1430249463846C0470130FF
:101BD0001ED02368E568326803F00603042B08BFB3
:101BE000AD1AA36822690CBF25EAE575002593426A
:101BF000C4BF9B1AED1800261A34B5421AD1002032
:101C000008E00123524649463846C047013003D117
